:100000000C94F3120C94198B0C94EE8A0C94C38A02
:100010000C94988A0C946D8A0C94428A0C94178ADA
:100020000C94EC890C9424130C9424130C94241336
:100030000C9424130C9424130C9424130C94241364
:100040000C9424130C9424130C9424130C94241354
:100050000C9424130C9424130C9424130C94B3B810
:100060000C9424130C94898E0C945F8E0C9424139E
:100070000C9424130C9424130C9424130C94241324
:100080000C9424130C9424130C9424130C94241314
:100090000C9424130C9424130C9424130C945226C3
:1000A0000C9424130C9424130C9424130C942413F4
:1000B0000C9424130C9424130C9424130C942413E4
:1000C0000C9424130C9424130C9424130C942413D4
:1000D0000C9424130C9424130C9424130C942413C4
:1000E0000C94241307634236B79BD8A71A39685675
:1000F00018AEBAAB558C1D3CB7CC5763BD6DEDFD4A
:10010000753EF6177231BF000000803F0800000006
:10011000BE922449123EABAAAA2ABECDCCCC4C3EFC
:1001200000000080BEABAAAAAA3E00000000BF00EB
:100130000000803F0000000000084178D3BB4387E7
:10014000D1133D190E3CC3BD4282AD2B3E68EC82FB
:1001500076BED98FE1A93E4C80EFFFBE01C4FF7F80
:100160003F00000000000C94B8B10C94152F0C94C3
:100170006D1F0C943C810C94761C0C94F3820C94AF
:1001800057840C94AD330C94221D0C9415590C9487
:1001900024330C9447310C94A3560C947A140C9489
:1001A0003BA70C94E06A0C94C7830C94233E0C94F8
:1001B00009A30C9496130C94EDB30C941FA70C9404
:1001C0008B170C9448300C942AAE0C9440130C946A
:1001D00058150C946E500C949B340C94EF320C9484
:1001E0008EB10C9455150C9456310C9446330C94E6
:1001F0003E180C94C6150C94B6340C9433340C94FD
:10020000CC590C9433350C94A83A0C94A5150C9445
:1002100064150C941B180C940A330C9477840C947A
:10022000272F0C94F7360C9453AE0C94CE830C9479
:10023000FE580C9441150C94BA570C9426150C9446
:10024000E7B30C94A6170C9470140C94EC130C9454
:1002500013BC0C94EC330C946C810C94EAB30C94A6
:1002600041AE0C94A8590C946F210C9463300C94FB
:10027000CB370C9411A70C94627B0C942C860C94B5
:100280004B130C946F900C94B2560C94B24E0C9489
:1002900083820C94EC570C9488160C947C830C94F9
:1002A0001F2D0C942C1B0C94011A0C9401800C949F
:1002B0004C730C94661D0C948B830C943E810C94AF
:1002C0005A340C9407170C9437AE0C94EF160C9418
:1002D000403C0C94F2A20C940C830C9484160C9465
:1002E000F92F0C94D8160C948F810C941A170C9437
:1002F00094160C940F800C94403A0C947F300C941C
:10030000F0B30C94AF620C94D92E0C9418A70C94F3
:1003100060150C943C330C9408200C9438150C9404
:1003200053150C9473950C94644F0C94FD170C9416
:10033000094F0C94BBB10C941D580C941EAE0C9438
:1003400045590C945E830C94D5810C94FD2E0C942D
:10035000324F0C949D810C94EC4E0C946D170C94C0
:10036000D5340C9408150C94184F0C94E0900C9410
:10037000D2170C94F94D0C94C0820C9426AE0C94B8
:1003800073820C941E340C94C2340C94943A0C94E2
:10039000327A0C9418AE0C9478340C9470190C9436
:1003A000C1490C94DF580C94C1B10C943E900C944C
:1003B00026A70C947C310C9404560C94893B0C9425
:1003C00022820C9464580C9494130C9422AE0C94D6
:1003D000CF390C9431C90C943F810C944F310C945B
:1003E0006C500C94E8790C94CC410C94AE160C949F
:1003F000813A0C94CE160C94F9480C94F93E0C9466
:1004000041800C94DF330C942F310C944BAE0C9440
:100410008B310C947D820C949E3A0C94891C0C9424
:100420007C2F0C94686F0C94574F0C941FB30C9452
:100430000F780C9406690C94A3580C949A210C9490
:1004400027200C94BB190C942E800C94B8130C9498
:100450002DAE0C94A8340C9445150C9468150C948E
:100460002E8D0C9405A30C9458180C94AD860C9406
:1004700041840C945B800C9429150C94C3330C9428
:10048000C1200C94F4160C9458AE0C9417150C94CF
:100490007B810C942D150C9490160C9418B30C942D
:1004A000CE2D0C9453350C945DAE0C9435180C94F1
:1004B00060170C9475310C94F4490C946E3A0C94BA
:1004C000371F0C94FC7F0C942E3A0C9481990C9459
:1004D000DB840C94F5B30C94D01B0C944F900C94CB
:1004E00027330C9425150C9442A70C949A150C9460
:1004F000C3410C9468630C9484800C94A5590C94AB
:10050000D2410C9446340C9433AE0C9481340C9448
:100510003F430C94EBA20C944A170C94E92F0C94D3
:10052000FE340C9482310C94A3970C943D810C946E
:1005300049150C94544F0C948C160C9472500C94D6
:10054000EA620C942E1B0C947F920C94BD560C9472
:10055000B0150C944FAE0C9434A70C9428A30C94B3
:10056000C0560C9498160C948F840C94333D0C94C4
:1005700042A30C94672B0C943F210C949C160C9472
:100580008C560C943E420C94CB680C94373A0C94E5
:1005900026130C9412180C94FD7E0C948C580C9419
:1005A0007F490C9438990C942A130C94834E0C9424
:1005B00045AE0C94B5830C94A5130C940E340C9496
:1005C0007A820C9478150C9434580C94F4170C948B
:1005D0000B190C94F2900C94301B0C9469800C94C1
:1005E000A9940C94DB950C94EE760C94EB160C9479
:1005F0003C4E0C94AA3A0C94499C0C945B3A0C9493
:1006000038310C943F190C94BD1B0C942A150C9492
:10061000493A0C94EE330C94CC560C94C4800C9450
:10062000AF560C94C8480C94748D0C943DAE0C9449
:10063000FC340C942B910C9458900C94C7550C944A
:1006400079560C9465560C94D9800C94AB590C9443
:100650005A850C9457990C94C7340C9428290C94FF
:1006600095130C9473140C94BF150C949A310C943C
:10067000BF130C9455680C94F1160C9459AE4E416E
:100680004E494E495459494E46CDCCCC3D0AD7230C
:100690003C17B7D13877CC2B329595E6241FB14F54
:1006A0000A000020410000C84200401C4620BCBE99
:1006B0004CCA1B0E5AAEC59D746364696E6F70732D
:1006C0007578585B00454F46002F00496E3A200070
:1006D000204E6F20656D6974206461746121002073
:1006E000436F756E74657220747970652E20766123
:1006F0006C3D00494E3A0020436F756E7465722060
:10070000747970652E20494E434F52524543542010
:10071000496E74657272757074206E756D62657263
:10072000212121004952513A002D3E002000230092
:100730002D3E00200050656E6465643A2023000061
:100740000020002300260029002C002F003200008A
:100750000100000301060109013D00494E3A003D38
:10076000004C454741435920494E3A00737566662F
:100770006978436F64653A0020666F7220286D7354
:10078000293A004354524C3A205363686564756CAF
:100790006520636D642000206D73203A0041726D06
:1007A000656420666F7220002044697361726D6514
:1007B00064002074696D653A004354524C3A2052EB
:1007C00065733A002054533A0020543A0054484587
:1007D000524D3A00436C65616E696E6720616C61D1
:1007E000726D20003D0050696E3A004354524C3AFD
:1007F00020436F6D6D616E6420626C6F636B656426
:1008000020627920647269766572206F7220636855
:10081000616E6E656C2066726F7A656E004354522D
:100820004C3A204F4E3A416C7265616479204163C5
:10083000746976650A004354524C3A2048414C543E
:100840003A416C726561647920496E6163746976BE
:10085000650A004354524C3A20584F4E3A2044699E
:100860007361626C65640A004354524C3A20584FDD
:100870004E3A416C726561647920416374697665B2
:100880000A004354524C3A20584F464620736B6935
:10089000707065642E205072657620636D643A0036
:1008A0004354524C3A205475726E6564206F6666EC
:1008B0002066726F6D3A004354524C3A2052657371
:1008C000746F7265642066726F6D3A004354524CC7
:1008D0003A2049676E6F7265642C206368616E6EA2
:1008E000656C20636D643D0020457865633A004384
:1008F00054524C3A204163746976653A004354522D
:100900004C3A2048414C543A416C726561647920FC
:10091000496E6163746976650A004354524C3A200B
:10092000584F4E3A2044697361626C65640A004313
:1009300054524C3A20584F4E3A416C72656164797A
:10094000204163746976650A004354524C3A20583A
:100950004F464620736B69707065642E2050726537
:100960007620636D643A004354524C3A20547572B9
:100970006E6564206F66662066726F6D3A00435440
:10098000524C3A20526573746F7265642066726FC0
:100990006D3A004354524C3A204E6F7420656E6F8E
:1009A000756768206D656D6F727920666F7220675C
:1009B000726F7570206F7065726174696F6E004937
:1009C0006E76616C69642061726700496E76616C55
:1009D000696420617267004354524C3A20556E6B33
:1009E0006E6F776E2073756666697800536B6970F9
:1009F00070656420686F6D69652073747566660044
:100A00002000205375623D00204974656D3D004310
:100A100054524C3A2052414D3D004354524C3A20DE
:100A20004F75744F664D656D6F72793A2000282DB1
:100A3000292000282B2920002076616C756520690B
:100A400073200020756E6B6E6F776E0A005D3D003F
:100A50005B0020696E76616C6964002000206F6B1A
:100A6000003A00206661696C6564003A0052657462
:100A70007279696E6720434D440A004354524C2FEB
:100A8000706F6C6C3A204F75744F664D656D6F7268
:100A9000793A2000207365632072656D61696E6923
:100AA0006E67005374617475732064656666657261
:100AB00065640A00444D58000000000000444D5891
:100AC000524742570000444D5852474200000050E0
:100AD000574D0000000000004D42555344494D0061
:100AE00000544845524D4F00000052454C415900BA
:100AF00000000047524F5550000000005643544537
:100B00004D500000004D42555356430000004143F4
:100B1000484149455200005350494C4544000000AB
:100B20004D4F544F52000000005049440000000057
:100B300000004D4255530000000000554152544200
:100B40005244470052454C415950574D00444D586E
:100B500052474257570056454E5453000000004537
:100B60004C455641544F5200434F554E5445520048
:100B70000048554D0000000000004D4552435552BD
:100B800059000020002D3E00436F6E766572746937
:100B90006E6720002D3E0057726F6E6720417373A1
:100BA00069676E6D656E742000524742783A200086
:100BB0004853562064697361626C65640020764C0A
:100BC0006576656C3A0020436F6E76563A00204396
:100BD0006F6E76533A0020486F743A00436F6C642E
:100BE0003A0020436F6E76657274656420563A0051
:100BF000436F6E76657274656420533A002D3E0033
:100C000057726F6E672041737369676E6D656E749E
:100C100020002D3E0057726F6E6720417373696725
:100C20006E6D656E74200020537566663A00204133
:100C3000543A00436F6E666967206368616E67654A
:100C400064206C6F63616C6C792C20706F727461BE
:100C50006C2064697361626C6564002F636F6E66FB
:100C600069672E6A736F6E007265626F6F74200021
:100C7000436D643A20002F636F6D6D616E642F00C9
:100C80002F72616D2F002F6974656D2F002F6974AD
:100C9000656D2F004C6F636174696F6E3A206874E4
:100CA00074703A2F2F6C617A79686F6D652E72754A
:100CB0002F707761003F6D61633D002669703D00D4
:100CC00026706F72743D00266E616D653D002F00C9
:100CD00020004D5154543A20436F6D706C6574651B
:100CE0002E2052656D6F766520746F7069632000E9
:100CF00024636F6D6D616E6400536B697070696E13
:100D0000672E2E004D5154543A20436C65616E5548
:100D1000702072657461696E656420746F706963B8
:100D20002000220022004F75744F664D656D6F7272
:100D30007921005D20003A5B004D5154543A005D2A
:100D400000456D7074793A205B000A003A004D410D
:100D5000433A00554450205379736C6F6720696E95
:100D6000697469616C697A65642E0A005379736CE1
:100D70006F6720706172616D733A00476F7420492C
:100D80005020616464726573733A00276970205B58
:100D900069705B2C646E735B2C67775B2C73756278
:100DA0006E65745D5D5D5D27202D20736574207315
:100DB00074617469632049500A004661696C656416
:100DC00020746F20636F6E66696775726520457465
:100DD0006865726E6574207573696E672044484358
:100DE000502E20596F752063616E207365742069E1
:100DF00070206D616E75616C6C792100204D4153DE
:100E00004B3A002047573A0020444E533A004C6F6B
:100E1000616465642066726F6D20666C6173682022
:100E200049503A000A7573657320444843500A00DC
:100E30005374617274696E67206C616E0041424345
:100E40004445464748494A4B4C4D4E4F50515253EA
:100E50005455565758595A616263646566676869A4
:100E60006A6B6C6D6E6F707172737475767778796A
:100E70007A303132333435363738392B2F3D004212
:100E80006173696320003A004F544120696E6974B0
:100E900069616C697A65640A0044454641554C5461
:100EA0002070617373776F726420666F72204F5485
:100EB00041204150492E20557365206F7461707731
:100EC0006420636F6D6D616E6420746F2073657450
:100ED0000070617373776F7264004D5154543A20FF
:100EE00074727969796E67206E656E7874206272AB
:100EF0006F6B6572004D5154543A20546F6F206DE2
:100F0000616E7920636F6E6E656374696F6E2065C4
:100F100072726F72732E2052657374617274204CFA
:100F2000414E002074727920616761696E20696E9C
:100F30002035207365636F6E6473004D5154543ACD
:100F4000206661696C65642C2072633D004D5154CC
:100F5000543A204177616974696E6720666F722028
:100F600072657461696E656420746F706963730083
:100F7000636F6E6E65637465642061732000202E5C
:100F80002E2E0020757365723A003A000A4D5154B6
:100F9000543A20417474656D7074696E6720636F94
:100FA0006E6E656374696F6E20746F200064697380
:100FB000636F6E6E6563746564005573696E672058
:100FC0004D5154542070617373776F726420667250
:100FD0006F6D20636F6E666967004465766963654F
:100FE000204E616D653A004D5154543A20417420B1
:100FF0006C6561737420646576696365206E616DEC
:101000006520616E642062726F6B657220495020AA
:101010006D75737420626520636F6E6669677572A3
:10102000656400757074696D652C667265656865C8
:10103000617000383663303531355F323032342DEF
:1010400030382D3131004C69676874487562200072
:10105000246E616D6500526562696E64207375630C
:10106000636573732E2049502061646472657373E5
:101070003A004572726F723A20726562696E64203E
:101080006661696C0052656E65776564207375638F
:10109000636573732E2049502061646472657373B5
:1010A0003A004572726F723A2072656E65776564B8
:1010B000206661696C000A4E6F206C696E6B00439C
:1010C0006F6E74696E7565207769746820707265DB
:1010D00076696F75736C79206C6F616465642063E9
:1010E0006F6E6669670033307320454550524F4D2F
:1010F000206973206E6F742072656C6F6164656423
:101100002E205265626F6F74004D5154543A204145
:101110006363657074696E6720636F6D6D616E6483
:10112000732E2E2E0A004E6F204D51545420636FA3
:101130006E66696775726564004C6F6164696E679D
:1011400020636F6E6669672066726F6D20706F72C4
:1011500074616C2064697361626C65642E207573C0
:101160006520676574204F4E20746F20656E616244
:101170006C6500436F6E6669672069732076616CE9
:10118000696400436F6E74696E7565207769746871
:101190002070726576696F75736C79206C6F61640D
:1011A000656420636F6E66696700536574757020AF
:1011B0004F5441004D5154543A2073657420666970
:1011C0007273742062726F6B657200437572726520
:1011D0006E74204C414E20636F6E6669672869709B
:1011E0002C646E732C67772C7375626E6574293A64
:1011F000000A55736520746865736520636F6D6DB3
:10120000616E64733A202768656C7027202D207406
:1012100068697320746578740A276D61632064655A
:101220003A61643A62653A65663A66653A303027F3
:101230002073657420616E642073746F7265204D35
:1012400041432D6164647265737320696E20454566
:1012500050524F4D0A276970205B69705B2C646E99
:10126000735B2C67775B2C7375626E65745D5D5D77
:101270005D27202D20736574207374617469632069
:1012800049500A277361766527202D2073617665A2
:101290002063757272656E7420636F6E6669672075
:1012A000696E204E5652414D3B204F4E7C4F464674
:1012B000202D20656E61626C652F64697361626CBC
:1012C00065206175746F736176650A276765742799
:1012D000205B636F6E66696720616464725D2720BE
:1012E0002D2067657420636F6E6669672066726F74
:1012F0006D207072652D636F6E66696775726564C7
:101300002055524C20616E642073746F72652061A9
:101310006464722C204F4E7C4F4646202D20656E13
:1013200061626C652F64697361626C6520646F77BC
:101330006E6C6F6164206F6E20737461727475706F
:101340000A276C6F616427202D206C6F6164206315
:101350006F6E6669672066726F6D204E5652414D02
:101360000A2770776427202D20646566696E6520E2
:10137000616E642073746F7265204D5154542070F7
:10138000617373776F72640A276F74617077642773
:10139000202D20646566696E6520616E642073741B
:1013A0006F72652048545450204150492070617339
:1013B00073776F72640A276C6F67205B736572695D
:1013C000616C5F6C6F676C6576656C5D205B7564E6
:1013D000705F6C6F676C6576656C5D27202D20648F
:1013E0006566696E65206C6F67206C6576656C203C
:1013F00028302E2E37290A276B696C6C27202D2068
:1014000074657374207761746368646F670A276317
:101410006C65617227202D20636C656172204545E3
:1014200050524F4D0A2773656172636827202D2043
:1014300073656172636820312D7769726520646518
:10144000760A277265626F6F7427202D207265629D
:101450006F6F7420636F6E74726F6C6C6572005383
:101460006F6674207265626F6F74696E672E2E2EC0
:1014700000206E65770020697320003157543A00D0
:101480003157543A20536561726368696E6720640E
:1014900065760052414D3D000A5379736C6F6720A9
:1014A000000A312D7769726520000A6D717474200D
:1014B000000A696E7075747320000A6974656D7333
:1014C00020000A436F6E666967757265643A004969
:1014D0006E697469616C697A696E6720496E7075AE
:1014E0007473003157543A207365747570207265B7
:1014F000736F6C7574696F6E20003157543A2044D5
:1015000053323438322D313030206E6F7420707287
:101510006573656E74003157543A20445332343841
:10152000322D3130302049324320726573746F722E
:101530006564003157543A204275732072657365B3
:1015400074206572726F72003157543A204275737D
:1015500020526573657420646F6E65003157543A8C
:10156000204453323438322D31303020707265735C
:10157000656E742C207265736574004572726F72AB
:1015800020312D7720696E6974003157543A204418
:1015900053323438325F3130305F4932435F544F19
:1015A0005F31575F42524944474520696E69740074
:1015B0003B003D0050696E3A003B003D4C4F5700E8
:1015C000546865726D6F3A004F6E65207769726579
:1015D0002052656164790A0042726F6B65727320F4
:1015E000636F6E666967757265643A004170706C0E
:1015F00079696E6720636F6E666967004C6F61641E
:10160000656420455441473A004E6F2073746F72F1
:10161000656420636F6E666967004C6F6164656422
:101620002066726F6D20454550524F4D006C6F61C2
:1016300064206661696C6564004A534F4E2064659E
:10164000746563746564004C6F6164696E67204300
:101650006F6E6669672066726F6D20454550524F08
:101660004D00436F6E666967206175746F736176B4
:10167000653A000A5379736C6F6720646562756719
:10168000206C6576656C3A0053657269616C206404
:1016900065627567206C6576656C3A0053617665A6
:1016A000640A005365742064796E616D6963204932
:1016B000500A004F54412050617373776F72642059
:1016C000757064617465640A004E6F204950206132
:1016D000647265737300205361766564004C6F61BA
:1016E00064696E67204854545020636F6E66696762
:1016F000206F6E20737461727475703A0000000080
:101700000000000000004F4E000000000000004FED
:1017100046460000000000005245535400000000FF
:1017200000544F47474C4500000048414C540000CE
:10173000000000584F4E000000000000584F464681
:101740000000000000494E435245415345004445C6
:1017500043524541534500454E41424C450000002F
:1017600044495341424C450000554E465245455A66
:101770004500465245455A450000004155544F002A
:101780000000000046414E5F4F4E4C59004849470B
:101790004800000000004D454449554D0000004CF4
:1017A0004F57000000000000484541540000000071
:1017B00000434F4F4C00000000004452590000000D
:1017C00000000053544F50000000000052474200F8
:1017D0000000000000485356000000000000636F46
:1017E000756C64206E6F742070617273653A2000AE
:1017F000557064617465640A00454550524F4D2030
:10180000636C65617265640A004D515454205061E7
:101810007373776F726420757064617465640A0015
:101820002B002D00455461673A2000476574204520
:101830005441473A2000485454502F312E3100254E
:10184000733A2025730D0A0020485454502F312E2E
:10185000310D0A486F73743A2025730D0A41636392
:101860006570743A202A2F2A0D0A436F6E6E6563E5
:1018700074696F6E3A20636C6F73650D0A0025738F
:101880000020000D0A00474554006661696C6564DC
:1018900020746F20636F6E6E6563740A0045525248
:1018A0004F523A2053657276657220726574757274
:1018B0006E65642000436F6E666967206E6F7420EA
:1018C0006368616E6765640A00446F6E652E0A0086
:1018D000436F6E6669672070617273696E67206618
:1018E00061696C65640A004765742061626F727497
:1018F000656400676F7420436F6E6669670A0068ED
:1019000074747020726574636F646520006672651C
:10191000652000436F6E666967205552493A20681A
:101920007474703A2F2F002044656661756C7420C2
:10193000636F6E6669672073657276657220757372
:1019400065643A20006C617A79686F6D652E7275F6
:10195000000A282D2943414E000A282D294D4552C1
:1019600043555259000A282D294D554C5449564586
:101970004E54000A282B2950574D5F52454C41596F
:10198000000A282D294D444E53000A282D2955417F
:101990005254425249444745000A282B295359536F
:1019A0004C4F47000A282D29504944000A282D2968
:1019B0004D43503233303137000A282D29415254DB
:1019C0004E4554000A282B294F5441000A282D293E
:1019D000535049204C4544000A282D294D4F544F5F
:1019E0005220435452000A282D294143204841499E
:1019F0004552000A282D29434353383131202620EF
:101A000048444331303830000A282B29524553547A
:101A10004152545F4C414E5F4F4E5F4D5154545FA5
:101A20004552524F5253000A282D294841524452E0
:101A3000455345542C207573696E6720736F667427
:101A4000000A282B29434F554E544552000A282D91
:101A500029444854000A282B294453323438322D63
:101A6000313030000A282B294F57495245000A28A7
:101A70002D2949504D4F44425553000A282D294DD8
:101A80004F44425553000A282D29444D58000A2836
:101A90002B2957697A6E657435783030000A282B07
:101AA000294672656552616D207072696E74696E47
:101AB00067000A282B295741544348444F47006C7C
:101AC000617A79686F6D652E7275000A436F6E6674
:101AD0006967207365727665723A00323031313051
:101AE000334C0020432B2B2076657273696F6E3A5E
:101AF00000383663303531355F323032342D30388E
:101B00002D3131000A4C617A79686F6D652E7275DE
:101B1000204C6967687448756220636F6E74726FD9
:101B20006C6C65722000204F464600204F4E00200E
:101B300042595041535300536176656420746F20BD
:101B4000454550524F4D00536176696E6720636F73
:101B50006E66696720746F20454550524F4D2E2E9A
:101B600000556E6B6E6F776E2073756666697820B0
:101B700000556E6B6E6F776E20636D642000436F4F
:101B8000756E7465723A200020696E697400526542
:101B90006C61792D4F75742023002073746F700071
:101BA00052656C61792D4F75742023003D3E003ADB
:101BB0000070756220616374696F6E200069646CE7
:101BC00065006F66660068656174696E67006661CE
:101BD0006E00647279696E6700636F6F6C696E671F
:101BE0000020697320004F75742000556E6B6E6F76
:101BF000776E207375666669782000556E6B6E6F20
:101C0000776E20636D642000616374696F6E00728B
:101C1000656C61794374723A20005B305D3A200054
:101C2000202D202D202D20EFBBBF003E003E312077
:101C30002D20000000000000636D640000736574D7
:101C4000000076616C000064656C0000485356002B
:101C500000524742000066616E00006D6F646500CF
:101C60006374726C006875650000736174000074C1
:101C7000656D7000726177000020002E00696E00B3
:101C8000735F6F7574006D79686F6D6500435452B2
:101C90004C2F657865633A204F75744F664D656DBE
:101CA0006F72793A2000202D3E20004D5154543A55
:101CB0002000202D3E2000456D69743A203C002014
:101CC0002D3E20004974656D436D643A2000202D3F
:101CD0003E20004974656D3A20003157543A204245
:101CE0007573207265736574206572726F7200314E
:101CF00057543A2042757320526573657420646F9F
:101D00006E65003157543A204453323438322070D3
:101D1000726573656E742C20726573657400493248
:101D20004320526573657400005EBCE2613FDD8351
:101D3000C29C7E20A3FD1F419DC3217FFCA2401EAB
:101D40005F01E3BD3E6082DC237D9FC1421CFEA09B
:101D5000E1BF5D0380DE3C62BEE0025CDF81633D8B
:101D60007C22C09E1D43A1FF4618FAA427799BC57B
:101D700084DA3866E5BB5907DB856739BAE406586B
:101D80001947A5FB7826C49A653BD987045AB8E65B
:101D9000A7F91B45C6987A24F8A6441A99C7257B4B
:101DA0003A6486D85B05E7B98CD2306EEDB3510F3B
:101DB0004E10F2AC2F7193CD114FADF3702ECC922B
:101DC000D38D6F31B2EC0E50AFF1134DCE90722C1B
:101DD0006D33D18F0C52B0EE326C8ED0530DEFB10B
:101DE000F0AE4C1291CF2D73CA947628ABF51749FB
:101DF0000856B4EA6937D58B5709EBB536688AD4EB
:101E000095CB2977F4AA4816E9B7550B88D6346ADA
:101E10002B7597C94A14F6A8742AC896154BA9F7CA
:101E2000B6E80A54D7896B353E3E2000496E76618C
:101E30006C696420636F6D6D616E64003E3E3E00B0
:101E40004E6F204D414320636F6E66696775726502
:101E5000643A20736574206669726D7761726527D4
:101E600073204D41430A00454550524F4D20736940
:101E7000676E6174757265206F6B00496E69746975
:101E8000616C697A696E6720454550524F4D2E004E
:101E90002F64617461002F736B6574636800416324
:101EA000636573732D436F6E74726F6C2D52657121
:101EB000756573742D507269766174652D4E657405
:101EC000776F726B3A207472756500416363657356
:101ED000732D436F6E74726F6C2D416C6C6F772D28
:101EE000486561646572733A202A004163636573D3
:101EF000732D436F6E74726F6C2D416C6C6F772D08
:101F00004D6574686F64733A20504F53542C4745A5
:101F1000542C4F5054494F4E5300416363657373C3
:101F20002D436F6E74726F6C2D416C6C6F772D4307
:101F3000726564656E7469616C733A20747275655C
:101F4000004F5054494F4E530044454C45544500B2
:101F50005055540047455400504F53540061757418
:101F6000686F72697A6174696F6E3A2000417574A6
:101F7000686F72697A6174696F6E3A2000436F6EA0
:101F800074656E742D4C656E6774683A200020721B
:101F9000656164206572726F7220666F7220003E08
:101FA0002000203C003157543A003157543A206EFB
:101FB0006F7420696E6974003157543A204255534A
:101FC000592074696D656F7574003157543A204417
:101FD00053323438325F4552524F525F434F4E4670
:101FE0004947003157543A20312D77697265207383
:101FF000686F72746564007265616479002473743B
:1020000061746500757074696D65006672656568F8
:102010006561700024737461747300204578706981
:102020007265640A00202D746172676574207A6F8E
:102030006E652D0020416C61726D2045787069726B
:1020400065640A0020636D643A00204375723A00AB
:10205000205365743A002054696D65723A00204C33
:102060006F636B733A0052414D3D00000021002424
:102070000027002A002D0030003300010100000479
:102080000107010A0100002200250028002B002E74
:10209000003100340002010000050108010B0105B8
:1020A000050505070508080808020202020A0A08D1
:1020B00008040404040101010101010101030303F7
:1020C0000303030303040707070C0C0C0C0C0C0C94
:1020D0000C0202020206060606060606060B0B0B9B
:1020E0000B0B0B0B0B0102102020080810204010D6
:1020F00020408002010201080402010102040810CC
:1021000020408080402010080402018004020180E9
:102110004020100804020108040201010204081012
:10212000204080010204081020408000000A0B02B9
:10213000090C0D0E08070304010000000000000058
:10214000000000000000000000000000000000008F
:10215000000000000000001211100000000000004C
:10216000000000000000000000000000000000006F
:10217000006F637465742F73747265616D00696DAF
:102180006167652F6A70656700696D6167652F67B4
:10219000696600746578742F68746D6C0061707086
:1021A0006C69636174696F6E2F6A736F6E0074651A
:1021B00078742F706C61696E00436F6E74656E7415
:1021C0002D547970653A2000436F6E6E65637469B3
:1021D0006F6E3A20636C6F73650041636365737360
:1021E0002D436F6E74726F6C2D416C6C6F772D4F39
:1021F000726967696E3A202A00556E6B6E6F776E52
:10220000004E6F74204D6F646966696564004F4BC2
:10221000004D6F766564207065726D616E656E74D9
:102220006C7900496E7465726E616C2053657276CC
:102230006572204572726F72005061796C6F6164D3
:1022400020546F6F204C61726765004E6F7420667A
:102250006F756E64005757572D41757468656E74BD
:1022600069636174653A20426173696320726561D4
:102270006C6D3D2241636365737320726573747284
:1022800069637465642200556E617574686F726964
:102290007A6564005061796C6F61642073697A6556
:1022A0002077726F6E670042616420726571756598
:1022B000737400485454502F312E312000200020D8
:1022C0006973200044656C6574696E6720636F6E86
:1022D000662E2052414D207761733A0053746F701F
:1022E000706564006E6F7468696E6720746F207328
:1022F000746F700053746F7070696E6720636861EB
:102300006E6E656C73202E2E2E0043616E206E6FF4
:102310007420636C65616E202D206C6F636B656447
:10232000000000000000000000004F4E0000000010
:102330000000004F46460000000000005245535484
:102340000000000000544F47474C45000000484142
:102350004C540000000000584F4E000000000000E8
:10236000584F46460000000000494E435245415335
:102370004500444543524541534500454E41424C7A
:102380004500000044495341424C450000554E462B
:102390005245455A4500465245455A4500000041C0
:1023A00055544F000000000046414E5F4F4E4C59BF
:1023B000004849474800000000004D454449554D3C
:1023C0000000004C4F5700000000000048454154F9
:1023D0000000000000434F4F4C000000000044523A
:1023E0005900000000000053544F5000000000004E
:1023F0005247420000000000004853560000000011
:10240000000057726F6E67207061796C6164004DD7
:102410005154543A204354524C2F7478743A204FFC
:1024200075744F664D656D6F72793A2000202D3EB0
:102430002041543A004368616E20747970653A0017
:102440004E6F2073746F7265642076616C7565736E
:10245000202D2064656661756C743A20002D3E0065
:102460005075623A20002D3E005075623A20002DD2
:102470003E005075623A20000000000000636D6469
:102480000000736574000076616C000064656C0088
:10249000004853560000524742000066616E00003B
:1024A0006D6F6465006374726C006875650000731D
:1024B0006174000074656D700072617700002D3EDC
:1024C000005075623A20002D3E005075623A20009F
:1024D00053454E445354415455533A20556E6B6EF8
:1024E0006F776E20636D64200A000000000000001A
:1024F0000000004F4E000000000000004F46460064
:102500000000000000524553540000000000544FEA
:1025100047474C4500000048414C54000000000073
:10252000584F4E000000000000584F464600000083
:102530000000494E435245415345004445435245EE
:1025400041534500454E41424C450000004449532B
:1025500041424C450000554E465245455A450046BD
:102560005245455A450000004155544F00000000B7
:102570000046414E5F4F4E4C5900484947480000C5
:102580000000004D454449554D0000004C4F570098
:102590000000000000484541540000000000434F87
:1025A0004F4C0000000000445259000000000000A1
:1025B00053544F50000000000052474200000000FA
:1025C0000000485356000000000000536176656427
:1025D00020455441473A0053657420455441473AD9
:1025E000200031C913BC11241FBECFEFD1E2DEBFE2
:1025F000CDBF00E00CBF16E0A0E0B2E0E2E4FCEBEF
:1026000001E00BBF02C007900D92AE31B107D9F7C0
:102610002BE0AEE1B6E001C01D92AA37B207E1F7A8
:1026200012E1C2EFD2E100E006C021970109802F3C
:10263000FE010E94F1D5C13FD10780E00807A9F74C
:102640000E9425BC0C940FDE0C940000FC01818DCF
:10265000928D0895CF93DF931F92CDB7DEB7698334
:10266000DC01ED91FC910280F381E02D41E050E02E
:10267000BE016F5F7F4F19950F90DF91CF91089545
:10268000FC019485FB018485981303C081E0983098
:1026900008F080E00895CF93DF931F92CDB7DEB7A7
:1026A0006983DC01ED91FC910280F381E02D41E032
:1026B00050E0BE016F5F7F4F19950F90DF91CF9172
:1026C0000895FC01818191E09093BD088093DE081C
:1026D0001092E4081092E308089520914307260F12
:1026E0003327331F21323105ECF42091B708FC0168
:1026F00090E080E0243069F082E00895A0914307E3
:102700002191AC014D5D584FA40FB52FB11D2C93F5
:102710000196861798F380914307680F60934307EB
:1027200080E0089581E0089508950895E091E60815
:102730008091E508E81730F4F0E0EA59F84F80811D
:1027400090E008958FEF9FEF08959091E6088091B3
:10275000E5082FEF3FEF981748F4E92FF0E0EA592A
:10276000F84F208130E09F5F9093E608C9010895FB
:102770008091E5089091E608891B990B0895CF9206
:10278000DF92EF92FF920F931F93CF93DF937C0121
:10279000CB018A012091BD08222389F0EB016B0156
:1027A000C40ED51ECC15DD0569F06991D701ED91F8
:1027B000FC910190F081E02DC7011995F3CF642FB2
:1027C0000E946D13C801DF91CF911F910F91FF906F
:1027D000EF90DF90CF900895CF93DF931F92CDB706
:1027E000DEB769832091BD082223F9F02091E30828
:1027F000203258F021E030E0FC013383228390E066
:1028000080E00F90DF91CF9108958091E408E82F48
:10281000F0E0E254F74F998190838F5F8093E40852
:102820008093E30881E090E0ECCF61E0CE01019677
:102830000E946D13F7CF90E0FC01E156FF4DE4914B
:10284000F0E0EE0FFF1FEB57FF4DA591B4912C91D7
:102850008B519F4DFC018491822391E009F490E01B
:10286000892F0895FC01DC018D918111FDCF30E0AD
:1028700020E050E040E08AE09191992301F144305A
:1028800051055CF59E3271F42F3F310509F02CF5AE
:10289000DB01A40FB51F12962C934F5F5F4F30E002
:1028A00020E0EACF829FD001839FB00D1124292F11
:1028B000990F330B205331092A0F3B1FDDCF2F3FD8
:1028C000310509F054F4443051053CF4640F751F90
:1028D000FB01228381E090E0089590E080E008957C
:1028E00090E080E00895DC01ED91FC910284F38595
:1028F000E02D1994DF92EF92FF920F931F93CF93E5
:10290000DF93EC010C891D890115110559F01D8A11
:102910001C8AC801DF91CF911F910F91FF90EF901A
:10292000DF900895EC85FD858E859F85DF01A80FDA
:10293000B91F2C91243209F055C011962C912B37D8
:1029400009F050C00296E80FF91FF12CE12CDF01CD
:10295000D190DD2009F446C08DE7D816E9F08FEF5D
:10296000E81AF80AF4CF198A188A2C853D852115B2
:10297000310579F08E859F85280F391FF901208157
:10298000222321F001969F878E873EC01D861C86DC
:10299000C0CF0FEF1FEFBDCFE114F10419F11C926E
:1029A0008E859F8502966C857D85680F791FE881ED
:1029B000F9810684F785E02DCE011995998B888BD6
:1029C0001B8A1A8AEC85FD858E859F85E80FF91F85
:1029D000EE0DFF1DD2828E859F850396E80EF91EAF
:1029E000FF86EE86288939892115310509F4BDCF86
:1029F0008A899B89280F391FF9012081222309F434
:102A0000B2CF01969B8B8A8B022F220F110B81CFA5
:102A1000DC011C96ED91FC911D971E968D919C9169
:102A2000E80FF91F8081082E000C990B0895DC0136
:102A300015968D919C91009739F0DC01ED91FC91F8
:102A40000680F781E02D19940895089583E090E0C1
:102A50000895089584E190E00895DC01ED91FC91E2
:102A60000484F585E02D60E0199581E090E00895FB
:102A70008FE090E090938D0780938C0788EC90E036
:102A80000895FC01848195810895FC01768765870E
:102A90000895DC01ED91FC91068CF78DE02D1995E0
:102AA00091E089270895862F089581E0862708956B
:102AB00021E0FC018485883008F020E0822F089511
:102AC000FC01848595850895FC0184899589089584
:102AD00028EE33E0FC0131832083FB0140895189DA
:102AE00062897389FC0142835383648375830895EB
:102AF000DC01ED91FC91048CF58DE02D1994DC0145
:102B00001196EC911197EF70E150EB3008F03EC058
:102B1000F0E08827E157FA4E8F4F0C94F1D5A515B8
:102B2000A515C6159A159A15BF15B015B015B0158F
:102B30009A159A1514962D913D914D915C91179788
:102B4000A4E6B0E00E94A7D5089514966C9184E69F
:102B5000689FB0011124072E000C880B990B089573
:102B600020E030E048EC52E414966D917D918D9117
:102B70009C9117970E9482D40E94EED608951496D5
:102B80006D917D918D919C911797089560E070E013
:102B9000CB010895FC01A7812A2F2E7FC9F08181E6
:102BA0008F7081508330A0F4A695A150BB0B2BE50C
:102BB00031E00E9408D624E630E040E050E00E9478
:102BC00088D5DA01C90187569F4FAF4FBF4F08958F
:102BD0008FEF9FEF0895FC01A681B781109721F137
:102BE00018969C9118979F708EEF890F823010F085
:102BF00091111AC019964D935D936D937C931C9718
:102C0000A681B78118969C911897907F926018962C
:102C10009C930680F781E02D8085982F907F9036D9
:102C200019F48F70806A80870895FC01238130E059
:102C300090E080E0FC01EE0FFF1FE15BF94FA08107
:102C4000B181A217B30761F4880F991F880F991FEC
:102C5000FC01E55CF94F40835183628373830895DF
:102C6000A081B181AB2B19F420813181EDCF019688
:102C700085309105F9F60895FC01238130E090E05C
:102C800080E0FC01EE0FFF1FE15BF94F40815181B5
:102C90004217530761F4880F991F880F991FFC0191
:102CA000E55CF94F60817181828193810895408153
:102CB0005181452B89F431832083880F991F880F18
:102CC000991FFC01E55CF94F108211821282138278
:102CD00060E070E0CB01089501968530910589F69A
:102CE000F7CF880F991F880F991FFC01ED5DF94FF1
:102CF00080819181A281B3810196A11DB11D808344
:102D00009183A283B383089585E090E00C947116BB
:102D100084E090E00C94711683E090E00C947116BE
:102D200082E090E00C94711681E090E00C947116B2
:102D300090E080E00C947116CF93DF93EC01E88172
:102D4000F9810484F585E02D199529893A892F5F49
:102D50003F4F3A8B298BDF91CF910895CF93DF932B
:102D6000EC018E8581110DC081E090E049895A897E
:102D70002C853D854217530708F080E0DF91CF9105
:102D80000895E881F9810484F585E02DCE01199537
:102D90008F3F910549F780E090E0F0CFFC018485FA
:102DA00095856817790708F4CB01928B818B08957C
:102DB000CF93DF93FC012685222351F0EC01019093
:102DC000F081E02D0190F081E02D6FEF19951E86C6
:102DD000DF91CF910895FC0187859089089581E066
:102DE000089590E080E00895DC011296ED91FC9149
:102DF000309761F00280F381E02D309739F0862F13
:102E00008295807F60856F70682B60870895DC01F4
:102E10001296ED91FC91309751F00280F381E02DF4
:102E2000309729F0808582958F7090E0089590E02A
:102E300080E00895CF93DF93CDB7DEB760970FB6EC
:102E4000F894DEBF0FBECDBF19821A821B821C828E
:102E50001D821E821F8218868A81807F81608A83FC
:102E60006FEF3E819F81888529817A815B814C81CA
:102E70004C873E87888B372F452F5C857E85892F31
:102E8000988960960FB6F894DEBF0FBECDBFDF9174
:102E9000CF9108950F931F93CF93DF9300D000D06D
:102EA0001F921F92CDB7DEB781E028960FB6F89437
:102EB000DEBF0FBECDBFDF91CF911F910F9108955F
:102EC000CF93DF93EC01888D883020F40E94959792
:102ED00088E0888FDF91CF9108950F931F93CF9350
:102EE000DF93EC018B01888D883010F40E94959758
:102EF000B80182E00E948D9B888F883050F41D8736
:102F00000C871A8E198E81E0DF91CF911F910F915E
:102F1000089580E0F9CF0F931F93CF93DF938C0137
:102F2000EA01FC018485883048F40E940598892BC9
:102F300039F481E090E0F80193838283D0E0C0E02F
:102F4000CE01DF91CF911F910F910895EF92FF92E3
:102F50000F931F93CF93DF937C0180917908D4E086
:102F6000833309F0D8E009E618E0C0E0F8012191C8
:102F700031918F01F701848195812817390729F054
:102F8000CF5FDC13F3CF80E006C08C2F0E947E9BC6
:102F90008431B1F781E0DF91CF911F910F91FF90C4
:102FA000EF900895CF93DF93EC018C858830D0F4B7
:102FB0000E947E9B843189F0882379F0883169F002
:102FC00021E08C3159F4E881F9810084F185E02D0C
:102FD000CE01199521E0892B09F420E0822FDF91A1
:102FE000CF91089580E0FBCFFC018485883010F4F8
:102FF0000C94B89490E080E00895CF93DF93EC01B7
:103000008C85883060F40E947E9B873111F08C3172
:1030100031F48C850E94E8978115984088F3DF9100
:10302000CF910895FC018485883010F40C94E897C2
:1030300090E080E00895CF93DF931F92CDB7DEB785
:1030400041E050E0BE016F5F7F4FFC0184850E942C
:1030500067981816190634F4898190E00F90DF9173
:10306000CF9108958FEF9FEFF9CFFC0184858830D1
:1030700010F40C94679890E080E00895CF93DF936C
:10308000FC012485283028F08FEF9FEFDF91CF914E
:103090000895EC010190F081E02D0084F185E02D90
:1030A0001995892B89F38C850E94819490E0EECF4D
:1030B000CF92DF92EF92FF920F931F93CF93DF9304
:1030C000CDB7DEB7AF970FB6F894DEBF0FBECDBF5A
:1030D0008C016B017A0188EE93E09A8389831B82CD
:1030E0001C821D821E821C861B8648EE53E060E017
:1030F00070E04D875E876F87788B2EEB33E03A87E1
:103100002987988F8F8B198E1A8E1B8E1C8E28E024
:1031100029A39BA78AA71CA61DA61EA61FA6D80189
:103120001C968C91883060F40E947E9B882321F04D
:10313000F80184850E94879788E0D8011C968C93BB
:103140008091210990912209A0912309B09124092D
:103150008EA39FA3A8A7B9A78B839C83AD83BE83AF
:1031600018861F82AE01465D5F4FB601CE01019603
:103170000E944EB60097C1F0D801ED91FC910684F3
:10318000F785E02D88EE93E09DA38CA38CA59DA5EB
:10319000AEA5BFA58EA39FA3A8A7B9A7A701BE01EF
:1031A0006C5D7F4FC8011995AF960FB6F894DEBFDE
:1031B0000FBECDBFDF91CF911F910F91FF90EF9088
:1031C000DF90CF900895CF93C62F0E94611361EED8
:1031D00085E299E00E94EC136C2F85E299E00E9451
:1031E000EC13CF910C94FDAF0E94611381E00E941B
:1031F0000DAF91E0811190E0892F0895ECEBF0E0A4
:1032000080818A7B808360E084E10E9461AE60E01F
:1032100085E10C9461AECF93DF93EC0160EA7BE132
:1032200085E69AE00E94138E6C817D8185E69AE0A6
:103230000E94ECA66AE97BE185E69AE00E94138E83
:1032400085E69AE00E94F58B60E08C810E948FAE4B
:10325000E881F9810484F585E02D60E0CE011995BF
:1032600081E090E0DF91CF91089560E278E18111F3
:1032700002C062E278E184EB99E00C94138E6FE572
:1032800074E184EB99E00E94138EF0E0E0E0199580
:1032900084EF91E0089580917D088823B1F0E0915A
:1032A0008208F0918308309731F08681978190935E
:1032B00081088093800864EB71E184EB99E00E94BF
:1032C000138E84EB99E00C94F58B089563E37AE018
:1032D000811102C06EE27AE085E69AE00C94138ECA
:1032E000DC0155962C915597273781F4ED91FC918F
:1032F000008CF18DE02D199565EC76E085E69AE07D
:103300000E94138E85E69AE00C94F58B0895EF9257
:10331000FF920F931F93CF937C018C01C0E0C330C9
:10332000E1F0F801428150E070E060E02AE030E036
:1033300084EB99E00E94E68C6BE77CE184EB99E0FA
:103340000E94138ECF5F0F5F1F4FC43041F7CF91A4
:103350001F910F91FF90EF900895F701458150E084
:1033600070E060E02AE030E084EB99E00E94E68CB7
:1033700069E77CE1E3CFEF92FF920F931F93CF9326
:10338000DF93EC018B018091840890918508009770
:10339000A9F0FC0120852F70263081F40E9446A2FE
:1033A000FC0190859F70943049F481859285DF916E
:1033B000CF911F910F91FF90EF900895EE88FF88B5
:1033C000C70101970D97D0F46AEE73E0C8010E941F
:1033D00052DA892B99F48FE2888F85E08E9DB001B7
:1033E0008F9D700D11246D5C734E46E050E0CE0150
:1033F00049960E945ECECE014896D9CF90E080E0FB
:10340000D6CF4F925F926F927F92AF92BF92DF9230
:10341000EF92FF920F931F93CF93DF9300D000D0D2
:10342000CDB7DEB77C01D62E80918908882309F4B8
:10343000BEC0D70114969C9180910002891708F4B0
:10344000B6C08091200790912107BAE06B13F0C0BD
:103450008053994FFC011082D70118960D911C9151
:103460000115110509F49FC0F80161857285611588
:10347000710591F4458056806780708480911B09A6
:1034800090911C09A0911D09B0911E09481659067A
:103490006A067B0609F487C0D8011B964D915C91A2
:1034A0001C974115510509F47EC0F70124815396FC
:1034B0008C91539790E0322F377002C09595879585
:1034C0003A95E2F780FF6FC0A22EB12CC501887F2C
:1034D0009370892B39F451968D919C91887F9370CC
:1034E000A82AB92AD8018D919C91DC01ED91FC911B
:1034F0006115710509F486C00688F789E02D1995D4
:10350000019709F050C06CE3F801808191810E941D
:10351000F98BA50170E060E02AE0D8018D919C91C3
:103520000E94A98BF8012281808191816DE27CE16A
:10353000222311F06BE27CE10E94138ED8011D96CC
:103540006D917C911E978D919C910E946C8D60E293
:10355000F801808191810E94F98BD8011F966D91AD
:103560007C9150978D919C910E946C8DF8012281E5
:103570008081918160E27CE1222311F06AE17CE1AB
:103580000E94138E60ED76E0D8018D919C910E948F
:103590006C8DF80180819181DC01ED91FC91008CB2
:1035A000F18DE02D19951092210710922007D70177
:1035B00015968D919C911697009771F014963C91F9
:1035C00020910102231740F0DC01ED91FC91019064
:1035D000F081E02D6D2D199581E090E026960FB6D3
:1035E000F894DEBF0FBECDBFDF91CF911F910F9139
:1035F000FF90EF90DF90BF90AF907F906F905F90C3
:103600004F9008950488F589E02D28EE33E03A8341
:103610002983D80115964D905D906D907C901897F8
:103620004B825C826D827E82BE016F5F7F4F67CF6F
:103630008F3491050CF0BBCFBDE06B1709F4B7CF09
:103640009C012F5F3F4F3093210720932007805329
:10365000994FFC016083ABCF0C948ACC0C948ACC3C
:10366000CF93C1E068EE73E080E090E00E9400B08C
:103670006C2F84EB99E00E94E5A6CF5FC43191F7EF
:1036800084EF91E0CF910895EF92FF920F931F93F3
:10369000CF93DF930097C1F0FC0120812223A1F09A
:1036A0008C018DE7E82E84E2F82EC1E0D0E0B7016E
:1036B000C8010E9427CE892B49F02196F5E0EF0E34
:1036C000F11CCE30D10599F7D0E0C0E0CE01DF91FA
:1036D000CF911F910F91FF90EF900895CF93DF93BB
:1036E00000D000D01F921F92CDB7DEB7EEE9F9E00F
:1036F000128A118A80E090E19587848784E890E0BF
:10370000948B838B81E0868780E090E2908B878723
:1037100087E7858B1C821B8289EA92E09A838983E2
:10372000FE83ED838FEF9FEF98878F8367E47BE1C4
:1037300084EB99E00E94138E60918F08709190083D
:10374000CE0101960E9416908EE999E00E947019B0
:1037500067E37BE184EB99E00E94138E84EB99E0B0
:103760000E94F58B0E946CB928960FB6F894DEBFC4
:103770000FBECDBFDF91CF910895892B71F0FB0172
:10378000828193810E9416A469E078E184EB99E03C
:103790000E94138E88EC90E0089590E080E0F2CFD4
:1037A0000F931F93CF93DF93EB0102970CF484C028
:1037B0000A811B8166E077E1C8010E9409CE892B4E
:1037C00051F481E00E94A4A688EC90E0DF91CF91B3
:1037D0001F910F9108956FE077E1C8010E9409CE13
:1037E000892B11F480E0EECF6DED76E184EB99E06A
:1037F0000E94138E0E9406A66295617081E0682780
:1038000070E084EB99E00E94ECA684EB99E00E94C2
:10381000F58B8091900990919109892BE9F10A81AA
:103820001B810E94A7A38823B9F1F8010190002011
:10383000E9F73197E01BF10BB09770F582E70E9432
:1038400092A38091900990919109DC01ED91FC91F6
:103850000088F189E02D60E270E01995B80180914F
:103860009009909191090E946C8D8091900990919E
:103870009109DC01ED91FC910190F081E02D60E077
:1038800019958091900990919109DC01ED91FC913D
:103890000488F589E02D19956A817B8184EB99E094
:1038A0000E946C8D66ED76E184EB99E00E94138EA8
:1038B00084EB99E00E94F58B80918C0790918D07A5
:1038C00002973CF080EF9FEF90938D0780938C07D9
:1038D0007BCF69EC76E18EEB99E00E94138E8EEB44
:1038E00099E00E94F58B84EF91E070CF892B71F005
:1038F000FB01828193810E9464A463EB76E184EBF7
:1039000099E00E94138E88EC90E0089590E080E0AA
:10391000F2CFEF92FF920F931F93CF93DF93CDB728
:10392000DEB72C970FB6F894DEBF0FBECDBF8C016B
:103930007B0188EE93E09A8389831B821C821D821F
:103940001E8298878F8319861A861B861C860530EF
:103950001105ECF0BE01695F7F4FF701808591850D
:103960000E943214892B99F0CE0107960E9407A578
:10397000BE01695F7F4FF701868197810E943214F3
:10398000892B61F0CE0107960E94B1A50EC0CE0131
:1039900001960E9407A50430110554F7CE01019647
:1039A0000E94B1A503301105A4F1BE01695F7F4FEC
:1039B000F701848195810E943214892B51F1CE0147
:1039C00007960E945CA5BE01695F7F4FF701828167
:1039D00093810E943214892B19F1CE0107960E941F
:1039E000B2A46CE976E184EB99E00E94138E80E04A
:1039F0000E949BA688EC90E02C960FB6F894DEBF50
:103A00000FBECDBFDF91CF911F910F91FF90EF902F
:103A10000895CE0101960E945CA5023011059CF626
:103A2000CE0101960E94B2A401301105D1F6CE015B
:103A300001960E94B2A463EA76E184EB99E00E94C9
:103A4000138ECFCF0F931F93CF93DF938C01EB0196
:103A50000297C4F08A819B810E94BBCD80930102B2
:103A600099270E94AEA60230110549F08C819D81F4
:103A70000E94BBCD8093000299270E94B8A6C8EC93
:103A8000D0E002C0C0E9D1E068E876E184EB99E0DB
:103A90000E94138E6091010284EB99E00E94E5A6DA
:103AA00063E776E184EB99E00E94138E6091000257
:103AB00084EB99E00E94E5A684EB99E00E94F58BE7
:103AC000CE01DF91CF911F910F910895CF93DF9396
:103AD000EB0102979CF166E077E18A819B810E946D
:103AE00009CE892B29F40E9406A67E7F0E944BA650
:103AF0006FE077E18A819B810E9409CE892B29F4AE
:103B00000E9406A671600E944BA662E676E184EBF5
:103B100099E00E94138E0E9406A6672F609561703F
:103B200070E084EB99E00E94ECA684EB99E00E949F
:103B3000F58B88EC90E0DF91CF9108950E946E1B89
:103B4000F8CF009789F0FC0120852F70253061F4B3
:103B50000E94BEA2009741F0FC0120852F70243006
:103B600019F481859285089590E080E0089565E0DC
:103B7000FC01828193810E94BEA2009749F0FC0162
:103B80008085982F907F21F082958F7090E0089526
:103B900090E080E008950F931F93CF93DF93FC0193
:103BA000C481D5812097C9F18B0188858F708530BC
:103BB00021F5CE010E9449A78017110671F16CF121
:103BC000602FCE010E94BEA2FC01892B31F18085BD
:103BD0008F70823039F461857285838594850E9467
:103BE00023D406C08330C9F46185728583859485AA
:103BF000DF91CF911F910F910895672B71F482305F
:103C000029F469857A858B859C85E9CF833029F4F1
:103C100069857A858B859C85EBCF60E070E0CB0170
:103C2000E7CFCF93C62F63E0FC01828193810E948E
:103C3000BEA2FC01892B91F09085892F8D7071F4C3
:103C4000907F9260908781859285A385B48588272F
:103C5000BB278C2B81879287A387B487CF91089548
:103C60008F929F92AF92BF92CF92DF92FF920F936B
:103C70001F93CF93DF93EC018A819B810E9449A718
:103C8000082F10E0043011059CF40E944C92FC01B6
:103C9000892B19F08085807F808780858F70808751
:103CA000BF018A819B810E94C4A60F5F1F4FEACF8C
:103CB00060E08A819B810E94BEA28C0101151105E2
:103CC00041F0F80180858F708430E1F128F4823072
:103CD00069F0FF24FA940BC0853089F18630C9F76A
:103CE0006EEE73E0C8010E9446A2E7CFF184FA8627
:103CF0000A811B8161E0C8010E94BEA29D838C8362
:103D000062E0C8010E94BEA29F838E8364E0C80166
:103D10000E94BEA299878887F0E1FF16D1F184E165
:103D2000F81609F485C0DF91CF911F910F91FF9094
:103D3000DF90CF90BF90AF909F908F9008950681B5
:103D40001781BCCFC184D284C114D10411F2F60111
:103D50008081882309F4BDCF84EB882E8AE0982ED9
:103D6000B12CA12CFA2CC4010E9437CEAC01B401B5
:103D7000C6010E9450CE892B09F468C0FFEFAF1A2C
:103D8000BF0A89E0880E911CE7E1AE16B10451F735
:103D9000A0CF8BE090E00E94EECB8C01FC01D3839E
:103DA000C28387E592E0918380831682CE010E94D0
:103DB00059A797FD2AC0F80195838483F80184816F
:103DC0009581009719F0863491052CF080E290E0FF
:103DD000F8019583848361E070E0CE010E94CB1DE1
:103DE00020E030E04AE754E40E9482D40E94F5D6F5
:103DF000611571058105910589F0F8016783708768
:103E0000818792871C870B878ECF91958195910929
:103E1000F8019583848381E08683D0CF88E893E19D
:103E2000A0E0B0E0F80187839087A187B287EACF4E
:103E300084E090E00E94EECBFC01D383C28325E3B3
:103E400032E0318320839C878B876DCFC6010E942F
:103E5000A48F8A2D90E0B0E0A0E0F80181879287DE
:103E6000A387B4878085807F8260808740CFCF9290
:103E7000DF92EF92FF920F931F93CF93DF93CDB713
:103E8000DEB760970FB6F894DEBF0FBECDBF7C01E2
:103E90006B01CA01B9012AE0AE014F5F5F4F0E947A
:103EA000CBCED701ED91FC910288F389E02D9801EA
:103EB000AE014F5F5F4FB601C701199560960FB60F
:103EC000F894DEBF0FBECDBFDF91CF911F910F9150
:103ED000FF90EF90DF90CF9008952F923F924F92F6
:103EE0005F926F927F928F929F92AF92BF92CF928A
:103EF000DF92EF92FF920F931F93CF93DF93CDB793
:103F0000DEB762970FB6F894DEBF0FBECDBF5C017F
:103F10004B0129013A01CA01B9010E94EED61B01E9
:103F20003F926F9380E494E09F938F93CE0101962C
:103F30007C019F938F930E94D7DA0F900F900F9080
:103F40000F900F900F9020E030E0A901C301B20163
:103F50000E9424D7181624F077FA709477F870949A
:103F6000F70101900020E9F731976F01CE18DF08C3
:103F70008EE28083A2E0B0E0AC0FBD1FAC0DBD1D92
:103F8000BA8BA98BB10137FE03C071956195710998
:103F9000072E000C880B990B0E9423D49B01AC01C7
:103FA000C301B2010E940FD620E030E040E251E4AC
:103FB0000E9482D40E94EED6605DE989FA8960830E
:103FC000FE01EC0DFD1D1382D501ED91FC910288DF
:103FD000F389E02D9801A701B401C50119956296F6
:103FE0000FB6F894DEBF0FBECDBFDF91CF911F910A
:103FF0000F91FF90EF90DF90CF90BF90AF909F9088
:104000008F907F906F905F904F903F902F9008958A
:104010001F93CF93DF93FC01162FC389D489818925
:1040200092899C012F5F3F4F328B218BC80FD91F84
:10403000CE010E9440D5181721F0612FCE010E94B9
:1040400048D581E090E0DF91CF911F910895FC0168
:1040500081899289248535858217930740F42389C5
:104060003489820F931F0E9440D590E008958FEF0E
:104070009FEF08959F92AF92BF92CF92DF92EF92FF
:10408000FF920F931F93CF93DF93EC017B018091FD
:104090007908811121C01B821A8288EE93E0A0E08A
:1040A000B0E08C839D83AE83BF8386E693E09983E3
:1040B000888388E08C8788EE93E09E878D87CE0189
:1040C000DF91CF911F910F91FF90EF90DF90CF90F4
:1040D000BF90AF909F90089534E0932E833311F0FA
:1040E00028E0922E89E6C82E88E0D82E10E098E0CD
:1040F000B92EA12CD6012D913D916D01F70184813E
:1041000095812817390791F4812F0E947E9B082FF3
:10411000873111F08C3139F5812F0E94B894892BA9
:1041200059F50C3119F4812F0E9487971F5F911266
:10413000E1CFA11008C0D701ED91FC910084F18579
:10414000E02DC70119951B821A8288EE93E0A0E04A
:10415000B0E08C839D83AE83BF8386E693E0998332
:104160008883BC86A8CF843149F08111DFCFF60166
:10417000329711821082DACFB12ED8CFAA24A3941D
:10418000D5CF8F929F92AF92BF92CF92DF92EF9254
:10419000FF920F931F93CF93DF93CDB7DEB72F9787
:1041A0000FB6F894DEBF0FBECDBF5C014B017A01A4
:1041B000809179088823C9F104E0833309F008E08D
:1041C000B501CE0101960E943A2089E6C82E88E00A
:1041D000D82E10E0F601219131916F01F501848113
:1041E00095812817390751F4812F0E947E9B8731D2
:1041F00029F4A701B401812F0E9405981F5F0113C4
:10420000E9CFC7012F960FB6F894DEBF0FBECDBF22
:10421000DF91CF911F910F91FF90EF90DF90CF90A2
:10422000BF90AF909F908F900895F12CE12CE9CF33
:10423000DA01E0918607F0E0FE2FEE27E60FF71F88
:1042400090E0982F8827A901BD018E0F9F1F0C9425
:10425000359344E050E0BC018FE090E00C94C093B3
:1042600044E050E0BC0185E090E00C94C09344E051
:1042700050E0BC0181E090E00C94C09308950F934E
:104280001F93CF938C01FC016481758181E20E94B0
:104290008D9BC82F8830F8F480E591E00E94D1AA68
:1042A0008C2F0E94E497833131F08C2FCF911F9196
:1042B0000F910C94879762E070E08C2F0E947797A3
:1042C000F80184819581EC2FF0E0EE0FFF1FE75994
:1042D000F74F91838083CF911F910F9108950F9392
:1042E0001F93CF93DF931F921F92CDB7DEB7FC01D0
:1042F00024852830E0F48C0180E591E00E94D1AA69
:1043000022E030E0AE014F5F5F4F60E170E0F80106
:1043100084850E94182189819A8198278927982766
:104320000F900F90DF91CF911F910F91089590E022
:1043300080E0F6CF0F931F93CF93DF931F921F92CE
:10434000CDB7DEB7FC0124852830E0F48C0180E590
:1043500091E00E94D1AA22E030E0AE014F5F5F4FB2
:1043600064E070E0F80184850E94182189819A81B7
:104370009827892798270F900F90DF91CF911F9151
:104380000F91089590E080E0F6CFCF93DF93EC019A
:1043900088EE93E0998388831A821B821C821D8297
:1043A00080E591E00E94D1AABE016E5F7F4F44E09C
:1043B00050E08FE090E00E943593CE01DF91CF91E5
:1043C0000895CF92DF92EF92FF920F931F93CF93B6
:1043D000DF9300D000D0CDB7DEB78091890881117E
:1043E0009AC080918C0790918D0702970CF493C02E
:1043F00080918F0890919008009709F48CC065EF28
:1044000073E00E9446A28C01009709F484C00E94C8
:1044100049A7E82EF12CE114F10409F47CC070E006
:1044200060E0C8010E94A11D6C01EA94EF2809F424
:1044300081C061E0C8010E94BEA2FC010185128515
:10444000CE0101960E94C521CE0101960E94D4AAF8
:104450006CE67DE084EB99E00E94138EB60184EB5C
:1044600099E00E946C8D6EE975E084EB99E00E9402
:104470006C8DB80184EB99E00E94ECA66EE975E0C2
:1044800084EB99E00E946C8D67EE78E084EB99E014
:104490000E946C8D84EB99E00E94F58B62E072E0E3
:1044A00083E89AE00E946D17D092790AC092780A48
:1044B00010937B0A00937A0A87EE98E0892BE9F53E
:1044C00083EF93E090937D0A80937C0A809180082B
:1044D00090918108009741F070E060E00E94A11D7A
:1044E00090937F0880937E0880917E0890917F084A
:1044F000009731F190937F0A80937E0A1092810A8F
:104500001092800A81E08093890863E57DE084EB66
:1045100099E00E94138E26960FB6F894DEBF0FBE68
:10452000CDBFDF91CF911F910F91FF90EF90DF9062
:10453000CF90089502E012E083CF87EE98E0C2CFDB
:1045400085E792E0D7CF0E945C96882331F0809176
:104550007908843329F0873381F090E080E0089572
:1045600080E591E00E94D1AA85E390E00E94319617
:1045700085FD0DC082E090E0089580E591E00E9405
:10458000D1AA8EE290E00E94319680FFF3CF81E0C5
:1045900090E008951092B70881E08093B6081092D9
:1045A000910861E084E10E9461AE61E085E10E94D2
:1045B00061AEE9EBF0E080818E7F808380818D7F2A
:1045C000808388E48093B80085E48093BC000895DC
:1045D000CF93DF9391E090932207882361F0C091FD
:1045E000B800D091BA000E94FE180E94CA22D0934F
:1045F000BA00C093B800DF91CF910895CF92DF92B7
:10460000EF92FF920F931F93CF93FC01C1810E9401
:10461000E8AE6B017C018091B708811164C081E034
:104620008093B7088093B6089FEF9093B5081092D7
:10463000B4081092B3088093920880919208CC0F2E
:10464000C82BC093920880919108813009F081C0F5
:10465000109291080E94E8AE6B017C018091920853
:104660008093BB008091B9089091BA08A091BB08D3
:10467000B091BC08892B8A2B8B2BA1F00E94E8AE4D
:104680000091B9081091BA082091BB083091BC087C
:104690006C197D098E099F09061717072807390726
:1046A00008F442C08091BC0083FDD8CF85EC809394
:1046B000BC000E94E8AE6B017C018091B70881309C
:1046C00009F449C08091B408811167C08091B40891
:1046D000E3E9F8E0A6E6B7E090E0981751F1219100
:1046E0002D939F5FFACF8091B9089091BA08A0915D
:1046F000BB08B091BC08892B8A2B8B2B09F48BCF7C
:104700000E94E8AE0091B9081091BA082091BB0848
:104710003091BC086C197D098E099F09061717078F
:104720002807390708F077CF8091B8080E94E8225F
:1047300080E01092E6088093E50885E299E00E9407
:10474000A513CF911F910F91FF90EF90DF90CF9025
:10475000089585EEACCF8091B9089091BA08A091E8
:10476000BB08B091BC08892B8A2B8B2B09F4A5CFF1
:104770000E94E8AE0091B9081091BA082091BB08D8
:104780003091BC086C197D098E099F09061717071F
:104790002807390708F091CFC7CF81E099CF8F92D2
:1047A0009F92AF92BF92EF92FF921F93CF93DF93AE
:1047B000EC010E9433B04B015C0110E08BE4E82E69
:1047C000F12C0E9433B0681979098A099B09683E67
:1047D00073408105910510F5ED85FE85309709F050
:1047E000199560EFCE010E94E318CE010E94FE22CF
:1047F000182F80FD0FC08A81813009F41A82812F21
:10480000DF91CF911F91FF90EF90BF90AF909F905D
:104810008F900895C7010197F1F7D3CF81E08A8384
:10482000EECF1F93CF93DF93EC01162F0E94CF237F
:10483000CE010E94611362ED85E299E00E94EC13C3
:10484000612F70E06095709584E0660F771F8A9500
:10485000E1F7612B85E299E00E94EC130E94FDAF25
:10486000CE010E94FE22811731F084E08A83DF911D
:10487000CF911F9108958A818430C9F71A82F7CFAA
:10488000CF93DF93EC0163EC0E94E318CE01DF913C
:10489000CF910C94FE220F931F93CF93DF93EC01E3
:1048A000162F042F0E94CF23002341F0CE010E9437
:1048B0004024682F6460CE010E941124CE010E9422
:1048C000611365EA85E299E00E94EC13612F85E2AD
:1048D00099E00E94EC13DF91CF911F910F910C94FE
:1048E000FDAFEF92FF920F931F93CF93DF938C0155
:1048F0007B0140E065E50E944B24E70188E0E80E7B
:10490000F11C699140E0C8010E944B24CE15DF05DF
:10491000C1F7DF91CF911F910F91FF90EF90089514
:10492000CF93DF93EC010E94611340E060EFCE0172
:104930000E944B24DF91CF910C94FDAF0F931F93F6
:10494000CF93DF93EC010E94CF2380FD36C0CE01D0
:104950000E94402460E0CE010E941124CE010E94FA
:10496000CF23CE010E94611364EB85E299E00E949F
:10497000EC130E94FDAFCE010E94CF23082F10E060
:1049800082FF16C082E08A838881882341F0CE01AD
:104990000E944024682F6160CE010E941124159569
:1049A0000795802F8170DF91CF911F910F9108950E
:1049B0008A81823049F71A82E7CF80E0F4CFCF9224
:1049C000DF92EF92FF920F931F93CF93DF938C01AF
:1049D000EB017A01FC01858196810E949E24882347
:1049E000C1F1BE01F801858196810E94712440E0E9
:1049F0006EEBF801858196810E944B24E7016701E7
:104A0000F9E0CF0ED11CF801E580F680C7010E94C5
:104A1000CF23C7010E94611366E985E299E00E94F5
:104A2000EC130E94FDAFC7010E94CF2361EEC701C6
:104A30000E94E318C7010E94FE228993CC16DD066E
:104A400011F7F801858196810E949E2491E08130C2
:104A500009F090E0892FDF91CF911F910F91FF9086
:104A6000EF90DF90CF900895CF93DF93EA010E94FB
:104A7000DF24882381F0DE0189E090E0815039F065
:104A8000ED91E927F0E0E85DF24E9491F7CF81E0F7
:104A90002885291380E0DF91CF910895CF93DF938C
:104AA00000D000D000D0CDB7DEB7AE014F5F5F4F72
:104AB0000E943425882331F08D818F33A9F020F4B2
:104AC0008F31A1F080E007C08F3521F08F37D1F70B
:104AD0008CE001C08BE029960FB6F894DEBF0FBEC4
:104AE000CDBFDF91CF9108958AE0F5CF89E0F3CF74
:104AF0006F927F928F929F92AF92BF92CF92DF92EE
:104B0000EF92FF920F931F93CF93DF93FC012485C5
:104B100021118CC0872E762EEC010E949E248823C2
:104B200009F486C0CE010E94CF2340E060EFCE01A1
:104B30000E944B2410E000E066246A94AA24A39407
:104B4000B12CE02EE694E694E694F12C802F877049
:104B5000650101C0CC0C8A95EAF78B85082E000C04
:104B6000990B0817190734F5FE01EE0DFF1D938010
:104B70009C20CE010E94CF23CE010E94611368E7E2
:104B800085E299E00E94EC13992011F080E8982EBC
:104B9000692D85E299E00E94EC130E94FDAFCE01E1
:104BA0000E94CF23982F907485FF0BC0992369F042
:104BB0008EEF2AC09924939408171907D1F2912CEB
:104BC000D8CF911102C087FF602EFE01EE0DFF1DB0
:104BD000938187FF28C0C92AC3820F5F1F4F00340B
:104BE000110509F0AECF6B86FFEF6F1202C081E0B6
:104BF0008C872396E72DF82DCF01089629912193D4
:104C0000E817F907D9F781E0DF91CF911F910F9154
:104C1000FF90EF90DF90CF90BF90AF909F908F90DC
:104C20007F906F900895C094C922D6CF80E0ECCFDA
:104C30008FEFEACF85ED8093BC008091B908909109
:104C4000BA08A091BB08B091BC080796A11DB11D80
:104C500023E0B695A795979587952A95D1F720914A
:104C6000BC0024FD03C01092B70808954091B90814
:104C70005091BA086091BB087091BC08452B462B37
:104C8000472B69F30097A105B10541F025E32A956B
:104C9000F1F700000197A109B109E1CF8091B808AF
:104CA0000C94E8221F920F920FB60F9211240BB6AC
:104CB0000F922F933F934F935F936F937F938F93B5
:104CC0009F93AF93BF93EF93FF938091B900887F39
:104CD000803609F44DC008F040C0883209F4A9C0FC
:104CE00028F5803109F49DC0C8F4882309F4FBC07D
:104CF000883009F496C0FF91EF91BF91AF919F91D9
:104D00008F917F916F915F914F913F912F910F9074
:104D10000BBE0F900FBE0F901F901895883109F4AD
:104D200088C0803241F78093B50814C0803409F4FC
:104D30009DC040F48033B9F38833E9F68093B50819
:104D400085ECB0C0803509F485C0883509F496C07B
:104D5000883489F60E941A26CECF883909F48CC08F
:104D600038F5883729F050F4883611F0803719F675
:104D700083E08093B7081092650757C0883809F41C
:104D80007BC0803919F0803809F0B5CF8091650774
:104D9000803208F071C0E091650781E08E0F80934A
:104DA00065078091BB00F0E0EB5BF84F80833DC06E
:104DB000803B39F0E0F4803A09F479C0883A09F090
:104DC0009ACF84E08093B70810924407109243076B
:104DD000E091E108F091E208199580914307811173
:104DE0000FC081E0809343071092230709C0803CE5
:104DF00009F4A6CF883C09F4A3CF883B09F07BCF08
:104E0000E091440781E08E0F80934407F0E0ED5D70
:104E1000F84F80818093BB009091440780914307B5
:104E200029C0809192088093BB0085EC8093BC00E0
:104E300062CF9091B4088091B308981758F5E0912B
:104E4000B40881E08E0F8093B408F0E0ED56F74F80
:104E50008081E9CFE091B40881E08E0F8093B4089F
:104E60008091BB00F0E0ED56F74F80839091B4083D
:104E70008091B3089817C8F285E8D8CFE091B408BC
:104E800081E08E0F8093B4088091BB00F0E0ED5676
:104E9000F74F80838091B60881115CCF81E08093C9
:104EA000910884EA8093BC001092B70824CF85EC67
:104EB0008093BC001092B70880916507803230F46F
:104EC000E0916507F0E0EB5BF84F108260916507B9
:104ED00070E0E091DF08F091E00885E497E0199533
:104EE0001092650708CF1092B50834CF4F925F92A9
:104EF0006F927F92AF92BF92CF92DF92EF92FF922A
:104F00000F931F93CF93DF9300D01F92CDB7DEB7DF
:104F10002B013C0129833A834B835C83A6019501D5
:104F2000C801B701640D751D861D971D211531053A
:104F30004105510511F00E9466D529813A814B81C6
:104F40005C816217730784079507D0F42415350533
:104F50004605570530F521E0822F0F900F900F90F6
:104F60000F90DF91CF911F910F91FF90EF90DF9005
:104F7000CF90BF90AF907F906F905F904F900895CB
:104F8000461657066806790650F421E089819A8111
:104F9000AB81BC8184159505A605B705E8F220E034
:104FA000DBCF21E04616570668067906A8F2F7CF50
:104FB0000F931F93CF93DF936EE17DE185E69AE037
:104FC0000E94378E81E00E940DAF0E94FE1861E0C2
:104FD00085E10E948FAE60E084E10E948FAEC4E163
:104FE000D0E010E001E0612F85E10E9461AE102762
:104FF0006AE070E080E090E00E9400B0219799F7AD
:1050000064E170E080E090E00E9400B00E9412AB8A
:105010008091890790918A07009729F10E94F418DE
:10502000882309F18091890790918A070E94902432
:1050300063E07DE185E69AE00E94378EE091890782
:10504000F0918A0700838091890790918A070E94D6
:105050009E246FEE7CE1811102C06AED7CE185E661
:105060009AE00E94378E81E0DF91CF911F910F91DE
:1050700008950F931F93182F0E9433B004C0969584
:105080008795779567951A95D2F78B019C0101500A
:105090001109210931090E3F1F4F2F4F3F4F20F0BB
:1050A00061E070E080E090E01F910F9108958F9291
:1050B0009F92AF92BF92CF92DF92EF92FF920F93A7
:1050C0001F93CF93DF937C014A015901C09184085B
:1050D000D0918508062F660F110B209709F45CC04C
:1050E00088858F70863009F055C06CEF73E0CE0173
:1050F0000E9446A26C0182E08816910449F061E0AA
:1051000074E0E3E08E16910429F0D0E0C0E006C020
:1051100065E074E0CE010E9446A2EC01C114D10406
:10512000D9F1F60180858F708430B1F56185728583
:10513000A801C7010E9480DAA8016AE074E0C701F3
:105140000E9462DA209779F188858F70843059F552
:1051500069857A85A801C7010E9462DAA8016AE020
:1051600074E0C7010E9462DAA114B10429F0A80119
:10517000B501C7010E9462DAC701DF91CF911F918B
:105180000F91FF90EF90DF90CF90BF90AF909F90E6
:105190008F900895D0E0C0E0A80166E87CE1C701E7
:1051A0000E945ECEC9CFF2E08F16910481F083E0B9
:1051B0008816910429F060917E0870917F08CACF0B
:1051C000A80160E87CE1C7010E9440CEC7CFA801DA
:1051D0006DE77CE1F8CFCF92DF92EF92FF920F93D1
:1051E0001F93CF93DF93CDB7DEB7C154D1090FB66C
:1051F000F894DEBF0FBECDBF6C01AB0130E020E004
:1052000060E4CE0101967C010E945728F7010190CD
:105210000020E9F731978F010E191F09A801B70186
:10522000C6010E9472DA892B11F010E000E0C8017B
:10523000CF5BDF4F0FB6F894DEBF0FBECDBFDF915F
:10524000CF911F910F91FF90EF90DF90CF90089535
:10525000CF92DF92EF92FF920F931F93CF93DF9342
:10526000CDB7DEB7C054D1090FB6F894DEBF0FBE7C
:10527000CDBF80918C0790918D07059709F449C0A7
:105280006115710509F445C069017A018B0140E49B
:1052900050E0CE0101960E9480DA6FE270E0CE010C
:1052A00001960E9447DA892B41F4980143E050E0CF
:1052B00060E4CE0101960E9457284FE350E0B6010A
:1052C000CE0101960E9462DA0E9464A2882309F14D
:1052D00080918C0790918D070697D9F48091F808FA
:1052E000811117C0B701CE0101960E9401B181E082
:1052F00090E0C05CDF4F0FB6F894DEBF0FBECDBFAD
:10530000DF91CF911F910F91FF90EF90DF90CF90A1
:10531000089590E080E0EDCFCF93DF931F921F922E
:10532000CDB7DEB780916E0B90916F0B009711F4A3
:105330008AE79BE0BE016F5F7F4F681B790B072EEA
:10534000000C880B990B0F900F90DF91CF9108956F
:105350004F925F926F927F928F929F92AF92BF9285
:10536000DF92EF92FF920F931F93CF93DF93CDB70E
:10537000DEB760970FB6F894DEBF0FBECDBFFC015D
:1053800019861A861B861C869A85907F96609A8756
:10539000A081B181109709F4F7C08C91882309F49A
:1053A000F3C000811181D8019C91992309F443C075
:1053B0009D3209F4EDC090539A3028F00F5F1F4FD3
:1053C00011830083EECFC801D12CDC017D01E81AE6
:1053D000F90A2D91022E000C330B205331092A308B
:1053E0003105A0F35F016EE270E0C8010E9447DA68
:1053F000FC01009709F448C0DC014D018E1A9F0A98
:1054000011968C911197082E000C990BC09711964C
:105410000A9798F38181282F082E000C330B205314
:1054200031092A30310518F480330CF06EC020E0C9
:1054300030E0A90108C0D12CF12CE12CD3CF29E018
:1054400030E040E050E0AAE0B0E00E94A7D52B0198
:105450003C012281822F022E000C990BC0978A30CA
:10546000910570F420330CF458C02A330CF059C065
:10547000092E000CAA0BBB0B480E591E6A1E7B1E80
:105480008114910409F052C0C8010E94D9CD2A8527
:10549000207F2A602A872B013C016CE270E0D50155
:1054A0008D919C910E9447DA009709F068C0F50140
:1054B000118210824D865E866F86788A88E0FE01B2
:1054C0003996DE01119601900D928A95E1F72981B6
:1054D0003A814B815C816D817E818F819885609658
:1054E0000FB6F894DEBF0FBECDBFDF91CF911F91F5
:1054F0000F91FF90EF90DF90BF90AF909F908F90B3
:105500007F906F905F904F9008958A330CF097CF03
:10551000032E000C440B550B96CF80E090E0DC018D
:10552000ABCF89E090E0A0E0B0E0A6CFC801B3E047
:105530008B169104DCF4E8E0EE16F104BCF40E9452
:10554000D9CD9B01AC01A4E6B0E00E94A7D5DD2037
:1055500041F07094609450944094411C511C611C23
:10556000711C460E571E681E791E97CF0E94B7CD3C
:105570002B013C018A85807F87608A878ECF0196C8
:10558000D5018D939C9396CF412C512C320192CF13
:10559000C8010196DD24D39418CFCF92DF92EF9209
:1055A000FF920F931F93CF93DF93EC01A881B981F2
:1055B000109781F18C91882369F108811981F80194
:1055C0009081992351F09D3241F090539A3028F008
:1055D0000F5F1F4F19830883F0CFC8010E94D9CDF8
:1055E0006B017C016CE270E0C8010E9447DA009711
:1055F00069F419821882C701B601DF91CF911F911A
:105600000F91FF90EF90DF90CF90089501969983CE
:105610008883F1CFC12CD12C7601EDCF0097B1F169
:10562000FC01DB01AC01405F5F4F80E090812FE91E
:10563000290F263098F497559295907F9C9321815D
:105640003FE9320F3630B0F42755922B9D933296B6
:10565000E417F50759F791E0892708952FEB290FF3
:10566000263010F49753E8CF90539A3028F381E016
:1056700090E0E2CF3FEB320F363010F42753E5CF06
:1056800020532A3010F381E020E0DFCF80E008953E
:105690000097D1F0DC011696ED91FC913097A1F0C6
:1056A00080858F70843021F481859285009771F414
:1056B0000680F781E02D309739F080858F70843037
:1056C00019F481859285089590E080E00895CF9245
:1056D000DF92EF92FF920F931F93CF93DF93CDB79B
:1056E000DEB769970FB6F894DEBF0FBECDBFE0916D
:1056F0008907F0918A07309709F483C080917B086D
:1057000090917C08892B09F47CC08FEF83871486E5
:1057100013821482158216821782108611861286D1
:1057200060E874E184EB99E00E94138E84EB99E0C9
:105730000E94F58B8E010F5E1F4FBE016E5E7F4F84
:105740008091890790918A070E94782518160CF09D
:1057500058C0A895DE0111969E012E5E3F4F7D0137
:10576000F90141919F01842F90E054E09595879530
:105770005A95E1F782589D4FFC0180818C93E42F6C
:10578000EF70F0E0E258FD4F808111968C931197F5
:105790001296A017B10721F7198AB70180917B08EB
:1057A00090917C080E9446A26C016BE774E184EB47
:1057B00099E00E94138EB70184EB99E00E946C8DF2
:1057C000C114D104B9F0C6010E94482B7C01892B79
:1057D00009F4B3CF66E774E184EB99E00E94138E7D
:1057E000B70184EB99E00E946C8D84EB99E00E94F4
:1057F000F58BA3CF61E774E184EB99E00E94138EEF
:10580000F4CF88EC90E069960FB6F894DEBF0FBE37
:10581000CDBFDF91CF911F910F91FF90EF90DF905F
:10582000CF900895EF92FF921F93CF93DF93192F9C
:105830007B01C82FD92FD7FF03C0D195C195D109BE
:1058400061E08C2F0E948FAE82E0E816F10499F49B
:1058500060E08C2F0E9461AE6FE27BE185E69AE00A
:105860000E94138E85E69AE0DF91CF911F91FF9001
:10587000EF900C94F58B612FEF2851F46095661F23
:105880006627661F8C2F0E9461AE6BE27BE1E6CF3C
:10589000661F6627661F8C2F0E9461AE66E27BE161
:1058A000DDCF64E07BE184EB99E00E94138E61EF31
:1058B0007AE184EB99E00E94138E63EE7AE184EB47
:1058C00099E00E94138E6BED7AE184EB99E00E94DF
:1058D000138E84EB99E00E94F58B6BEC7AE184EBFC
:1058E00099E00E94138E6FEB7AE184EB99E00E94BD
:1058F000138E62EB7AE184EB99E00E94138E6DE9DE
:105900007AE184EB99E00E94138E6EE87AE184EBF1
:1059100099E00E94138E66E87AE184EB99E00E9498
:10592000138E6BE77AE184EB99E00E94138E6EE6AA
:105930007AE184EB99E00E94138E64E67AE184EBCD
:1059400099E00E94138E65E57AE184EB99E00E946C
:10595000138E6DE47AE184EB99E00E94138E61E48A
:105960007AE184EB99E00E94138E67E27AE184EB9E
:1059700099E00E94138E68E07AE184EB99E00E943E
:10598000138E63EF79E184EB99E00E94138E66EE4B
:1059900079E184EB99E00E94138E68ED79E184EB64
:1059A00099E00E94138E6CEC79E184EB99E00E94FF
:1059B000138E64EC79E184EB99E00E94138E69EB1D
:1059C00079E184EB99E00E94138E6CEA79E184EB33
:1059D00099E00E94138E64EA79E184EB99E00E94D9
:1059E000138E69E979E184EB99E00E94138E6AE8ED
:1059F00079E184EB99E00E94138E61E879E184EB10
:105A000099E00E94138E63E779E184EB99E00E94AC
:105A1000138E65E679E184EB99E00E94138E69E5C7
:105A200079E184EB99E00E94138E61E579E184EBE2
:105A300099E00E94138E84EB99E00C94F58B0F9300
:105A40001F93CF93DF9300D000D0CDB7DEB70E9475
:105A5000512C6BEC71E184EB99E00E94138ECE0126
:105A600001960E94C521CE0101960E94871908EE79
:105A700013E01A8309838091210990912209A09152
:105A80002309B09124098B839C83AD83BE83CE010F
:105A900001960E9487191A8309831B821C821D822A
:105AA0001E8280E591E00E94D1AA44E050E0BE0150
:105AB0006D5F7F4F81E090E00E943593CE010196AB
:105AC0000E9487191A8309831B821C821D821E82F1
:105AD00080E591E00E94D1AA44E050E0BE016D5FF4
:105AE0007F4F85E090E00E943593CE0101960E94A1
:105AF000871961EF71E184EB99E00E94138E88ECC5
:105B000090E026960FB6F894DEBF0FBECDBFDF91B2
:105B1000CF911F910F9108950F931F93CF936EE430
:105B20007DE084EB99E00E94138E08E919E0C0E063
:105B3000F80181918F01803130F46CE074E084EBE6
:105B400099E00E946C8DC530C9F0F8013197408111
:105B500050E070E060E020E130E084EB99E00E94EA
:105B6000E68C6CE47DE084EB99E00E94138ECF5FBD
:105B7000C630F1F6CF911F910F91089540919D0984
:105B800050E070E060E020E130E084EB99E00E94BA
:105B9000E68C84EB99E00E94F58BE9CFEF92FF92BF
:105BA0000F931F93CF93DF9300D000D01F92CDB7F8
:105BB000DEB77B01CE0107969F938F9301979F934A
:105BC0008F9301979F938F9301979F938F93019743
:105BD0009F938F9301979F938F938E010F5F1F4F1A
:105BE0001F930F938EE094E09F938F93DB011396A6
:105BF0008C9113978F9312968C918F930E9407DB51
:105C00000FB6F894DEBF0FBECDBF0697ECF46EED75
:105C100077E18EEB99E00E94138ED70112966D9179
:105C20007C918EEB99E00E946C8D80E991E0279643
:105C30000FB6F894DEBF0FBECDBFDF91CF911F919D
:105C40000F91FF90EF9008958091900990919109A4
:105C5000892BA9F10E94A7A3882389F182E70E94DA
:105C600092A38091900990919109DC01ED91FC91B2
:105C70000088F189E02D64E070E019958091900929
:105C800090919109DC01ED91FC910280F381E02D6E
:105C900046E050E0B801199586E0F801A8E9B9E0BE
:105CA00001900D928A95E1F7809190099091910968
:105CB000DC01ED91FC910488F589E02D19950E9495
:105CC0008C2D60EF77E184EB99E00E94138E88ECD5
:105CD00090E0ADCF2F923F924F925F926F927F9262
:105CE0008F929F92AF92BF92CF92DF92EF92FF92EC
:105CF0000F93CF93DF9300D01F92CDB7DEB77C0117
:105D00007A8369835C834B83DB011C92FC01608195
:105D1000662309F44BC030FF49C0F9E06F9FB00122
:105D200011246F5D7C4DCD010E945ECED70111968E
:105D30008C918F7041F04B815C816DE574E08981BD
:105D40009A810E9462DAE981FA8101900020E9F7E4
:105D5000319729813A81E21BF30B19012E0E3F1E68
:105D60004B815C814E1B5F0B415051095C834B831F
:105D7000D7011196EC911197EF7009F4F5C0E1503D
:105D8000EC3008F0F1C0F0E08827E653F14D8F4F7A
:105D90000C94F1D5D92E7C2FE92F48306330272F72
:105DA000F92FF92FF92F152FFD2E7F3029803A80FA
:105DB000DFCFF7018481282F30E050E040E000235E
:105DC00059F030E0A4E6B0E00E94BAD52FEF30E001
:105DD00040E050E00E9488D55F934F933F932F930C
:105DE00082E294E09F938F93FC81FF932B812F930A
:105DF0003F922F920E949ADAB2C017968C91179711
:105E00008F9316968C9116978F9315968C91159764
:105E10008F9314968C918F9385E294E09F938F9348
:105E2000BC81BF93EB81EF93E3CF17968C911797CB
:105E30008F9316968C9116978F9315968C91159734
:105E40008F9314968C918F9389E294E0E7CF149608
:105E5000CD90DD90ED90FC901797F7FE34C084E66E
:105E6000882E912CA12CB12CC701B601A50194015B
:105E70000E9488D59B01AC0188279927DC01821BF1
:105E8000930BA40BB50BBF93AF939F938F93662790
:105E90007727CB016C197D098E099F09A501940113
:105EA0000E9488D55F934F933F932F938DE294E0A8
:105EB0009F938F933C813F934B814F933F922F92BF
:105EC0000E949ADA4CC0C701B60124E630E040E0F7
:105ED00050E00E9488D59F938F937F936F935F9339
:105EE0004F933F932F938EE294E09F938F939C81E7
:105EF0009F93AB81AF93E2CFC7010E94CA15BC014B
:105F0000D7011696CC9016971796DC901797D0FA73
:105F1000DD24D0F814969C9114971596FC90EB8094
:105F2000BC80292F30E050E040E077FD35C0011102
:105F300035C07F936F931F921F921F929F931F9262
:105F4000FF92DF92CF9287E394E09F938F93FC813F
:105F5000FF932B812F933F922F920E949ADA0FB6D4
:105F6000F894DEBF0FBECDBF89819A810F900F904C
:105F70000F900F90DF91CF910F91FF90EF90DF90F6
:105F8000CF90BF90AF909F908F907F906F905F90D9
:105F90004F903F902F900895002361F0292F30E01B
:105FA000A4E6B0E00E94BAD52FEF30E040E050E028
:105FB0000E9488D55F934F933F932F931F92FF9238
:105FC000DF92CF928AE394E09F938F93BF92EF92F8
:105FD00075CF15968C9115971F928F9316969C915D
:105FE000169717968C9181708F939F938DE394E011
:105FF00015CF14968D909D90AD90BC90179720E092
:1060000030E0A901C501B4010E941CD4240135016E
:1060100087FF04C077FA709477F87094C301B201D7
:106020000E94EED66B01072E000C880B990B0E9484
:1060300023D49B01AC01C301B2010E940FD620E022
:1060400030E04AE754E40E9482D40E9479D70E944B
:10605000EED6062F772E20E030E0A901C501B4016D
:106060000E941CD487FF07C07F920F93DF92CF92CC
:1060700083E494E0D3CE7F920F93DF92CF9284E4B7
:1060800094E09F938F933C813F934B814F93B0CE8D
:1060900014968C9114971F928F9315968C91159747
:1060A0001F928F9316968C911F928F938AE394E0A0
:1060B0009F938F93BC81BF93EB81EF933F922F927D
:1060C0000E949ADA4CCF17968C9117971F928F9354
:1060D00014968C9114971F928F9315968C91159707
:1060E0001F928F9316968C911F928F9387E394E063
:1060F0009F938F93BC81BF93EB81EF93DFCE149678
:106100006D917C914B815C81C1010E9480DA2CCF22
:10611000EF92FF920F93CF93DF93CDB7DEB7A097A7
:106120000FB6F894DEBF0FBECDBF7C0100E020E0CB
:1061300033E040E250E0BE016F5F7F4F0E946A2E65
:10614000BE016F5F7F4F85E69AE00E946C8D6EE224
:106150007CE085E69AE00E94138EF70161816F7002
:1061600085E69AE00E94E5A667E27CE085E69AE093
:106170000E94138EF701628185E69AE00E94E5A6EF
:1061800085E69AE00E94F58BA0960FB6F894DEBFE4
:106190000FBECDBFDF91CF910F91FF90EF9008958B
:1061A000CF93DF9300D000D01F921F92CDB7DEB700
:1061B000FC01628398E0DE01119601900D929A95A0
:1061C000E1F729813A814B815C816D817E818F81EC
:1061D000988528960FB6F894DEBF0FBECDBFDF912D
:1061E000CF910895CF93DF9300D000D01F921F92DC
:1061F000CDB7DEB7FC01608398E0DE011196019017
:106200000D929A95E1F729813A814B815C816D81EC
:106210007E818F81988528960FB6F894DEBF0FBED9
:10622000CDBFDF91CF910895DC011196EC911197CC
:10623000EF70E150EB3008F039C0F0E08827EC5DFA
:10624000FE4C8F4F0C94F1D54731473156312F31E9
:106250002F3138314F314F314F312F312F3114968B
:106260006D917D918D919C9117970E9423D40895F3
:1062700014966D917D918D919C91179724E630E055
:1062800040E050E00E9488D5CA01B901EECF1496D3
:106290006C9170E090E080E00E9421D40895149603
:1062A0006D917D918D919C911797089560E070E0BC
:1062B000CB010895DC011196EC911197EF70E1503C
:1062C000EB3008F037C0F0E08827E659FE4C8F4FDE
:1062D0000C94F1D57C317C319A31753175318B312B
:1062E0008231823182317531753114966D917D9193
:1062F0008D919C911797089514966C9170E090E0A1
:1063000080E0089514966D917D918D919C911797E1
:106310000E94EED6089514966D917D918D919C9179
:10632000179724E630E040E050E00E9488D5CA018B
:10633000B901089560E070E0CB0108958F929F92BB
:10634000AF92BF92CF92DF92EF920F931F93CF93B2
:10635000DF9300D000D01F921F92CDB7DEB7098324
:106360001A832B833C834D835E836F837887FC0184
:106370002281338121153105A1F490E080E0289637
:106380000FB6F894DEBF0FBECDBFDF91CF911F9146
:106390000F91EF90DF90CF90BF90AF909F908F9034
:1063A00008958C01C9010E9449A7C82ED12CF6E09E
:1063B000CF16D104ACF40E944C92FC01892B19F049
:1063C0008085807F808780858F708087BF01F801FE
:1063D000828193810E94C4A6FFEFCF1ADF0AE7CF24
:1063E00065E0F801828193810E94BEA28C01892B15
:1063F00021F28981803108F6CE0101960E945A313E
:10640000161617061806190644F4F8018085982F09
:106410009D70A1F08F70873089F0F80180858F70B2
:10642000808768EA77E085E69AE00E94138E85E629
:106430009AE00E94F58B81E090E0A1CF0E9433B0FA
:106440004B015C01CE0101960E945A31860E971EC7
:10645000A81EB91EF80181869286A386B48682E0C2
:10646000E11087E099819295907F892BF8018087D0
:106470006DE977E085E69AE00E94138ECE010196E1
:106480000E945A31AB01BC012AE030E085E69AE077
:106490000E94E68C67E977E085E69AE00E94138E19
:1064A000F80141855285638574852AE030E085E6F0
:1064B0009AE00E94E68CBBCFCF93DF93EC0161158D
:1064C000710539F48F8181708F8381E0DF91CF91E5
:1064D00008958981982F9F7029F180E09430B0F75A
:1064E0009B01770F440B550B29593109410951097B
:1064F000A4E6B0E00E94A7D52BE531E040E050E0F3
:106500000E9488D537FF02C030E020E025363105F3
:1065100014F024E630E02F5F220F8F818170282B4A
:106520002F83D3CF807F82608983DACF2F923F92EF
:106530004F925F926F927F928F929F92AF92BF9293
:10654000CF92DF92EF92FF920F931F93CF93DF933F
:10655000CDB7DEB766970FB6F894DEBF0FBECDBFDE
:106560006C0109871A872B873C874D875E876F8769
:10657000788B22E1E216F10480F5F701ED51FD4F31
:106580008081898BCE0109960E94CA1597FD04C0AF
:10659000BC01C6010E945C328B85D60112968C9399
:1065A000129789858C931196EC911197EF70EC30CE
:1065B00008F06CC0F0E08827EF51FD4C8F4F0C9431
:1065C000F1D533340A330A337834EF32FC344634AD
:1065D00081348134813446344634198AD3CF10E073
:1065E0009A859F709D3008F002C4E92FF0E088275B
:1065F000E350FD4C8F4F0C94F1D546333335533572
:106600003335FE34FE3433353335F736F73633352C
:1066100033350E349A859F709D3008F00FC1E92FF5
:10662000F0E08827E95EFC4C8F4F0C94F1D546339F
:10663000EC33DF333C3327332433C333EE331E34A0
:106640001E34AD33AD330E348889F60187838F85D0
:10665000D60116968C9316978E8515968C93159762
:106660008D8514968C93149711968C911197807F39
:10667000892B11968C930AC08F859889F6018683A1
:10668000878190FB80F987838E858583F989FF2335
:1066900009F460C0D60111968C918F702F2F30E0D5
:1066A0008217130609F456C068E87BE085E69AE095
:1066B0000E94138EF60161816F7085E69AE00E9458
:1066C000E5A665E87BE085E69AE00E94138E69897D
:1066D00085E69AE00E94E5A663E87BE085E69AE01D
:1066E0000E94138ED6010C9119821A821B821C8281
:1066F0001D821E821F82188689898F709A81907FE1
:10670000892B8A830983EE24EA94FE2C11961C912E
:10671000119712962C91129713963C9113971496F9
:106720004C91149715965C91159716966C91169747
:1067300017967C91CE0101960E949632F601208335
:106740003183428353836483758386839783C60131
:106750000E94883088E0F6015FC18D859E85AF85F7
:10676000B889B7FD0EC08F3F9105A105B10529F08D
:1067700024F08FEF90E0A0E0B0E0D60114968C9367
:1067800085CF80E0FACF6D857E858F85988920E062
:106790006D39BFEF7B078B079B076CF02FEF6115FF
:1067A000E4E67E078105910534F424E630E040E01C
:1067B00050E00E9488D5D60114962C9367CF8F8520
:1067C0009889F6018683878190FB80F987838E857F
:1067D00085838D8584835ACF8D85CFCF8D849E848C
:1067E000AF84B88820E030E0A901C501B4010E945F
:1067F0001CD460E087FD0FC020E030E04FE753E499
:10680000C501B4010E9424D76FEF181624F0C5010A
:10681000B4010E94F5D6F601648338CFD6011196F3
:106820008C911197807F8C6011968C9311978D8538
:106830009E8515969C938E93149728CF65E17CE0F6
:1068400085E69AE00E94138E6A856F7085E69AE06D
:106850000E94E5A662E17CE085E69AE00E94138E44
:10686000F6016181BFC09A859F7011968C91119736
:10687000807F892B11968C938D859E85AF85B889F5
:10688000F60184839583A683B78300CF9A859F7092
:10689000933081F09C3011F24D855E856F8578894B
:1068A000F60144835583668377838181807F892BBA
:1068B0008183ECCEC6010E94CDA2D60114968C93A2
:1068C00014978F85988916968C93169717968C91A6
:1068D000179790FB80F917968C9317978E851596CE
:1068E0008C93159711968C911197807F8260C1CE01
:1068F000CE0109960E94CDA2D60114968C931497CE
:10690000F1CF9A859F709D3008F057C0E92FF0E0D5
:106910008827E257FB4C8F4F0C94F1D54633A834AF
:10692000D5345A34D534D5349B34C734C734C734FE
:10693000B634C2340E348D859E85AF85B889F60194
:1069400084839583A683B7838181807F8660B0CF5F
:106950006D8570E090E080E00E9421D4D60114960D
:106960006D937D938D939C93179790CE6D857E85C7
:106970008F8598890E9423D4F6016483758386836A
:10698000978384CE6D857E858F859889E5CFF601C6
:106990008181807F982B91838D859E85AF85B88975
:1069A00084839583A683B78371CE11968C911197BA
:1069B000807F982B11969C935FCF60E07CE085E60A
:1069C0009AE00E94138E6A856F7085E69AE00E94B5
:1069D000E5A66DEF7BE085E69AE00E94138ED60176
:1069E00011966C916F7085E69AE00E94E5A685E6A7
:1069F0009AE00E94F58B4ACE11E0F2CD4D855E857E
:106A00006F857889F6014483558366837783818116
:106A1000807F982B918388E0DE01119601900D9282
:106A20008A95E1F729813A814B815C816D817E8174
:106A30008F81988566960FB6F894DEBF0FBECDBFE6
:106A4000DF91CF911F910F91FF90EF90DF90CF904A
:106A5000BF90AF909F908F907F906F905F904F907E
:106A60003F902F900895963009F4BFC048F46D858B
:106A7000913071F06FEF70E0933051F060E008C03A
:106A8000973009F4BEC09A506D857E859230B0F77C
:106A900084E68F8788898E7F888B1E868A85807F93
:106AA00082608A876D872E8530E0AFEFB0E00E946C
:106AB000BAD5812C912C54018A946115F4E67F0794
:106AC0008105910544F424E630E040E050E00E9466
:106AD00088D549015A01112309F473C02D852A8BE9
:106AE000022F10E028882694822D8150990B1C01DA
:106AF0009FEF2916390609F0A4C0A0E88A16910470
:106B00000CF086C08FE790E088199909809FD0012A
:106B1000819FB00D909FB00D11242FEF30E00E94A7
:106B200008D621E83EE740E050E00E9488D5F60113
:106B30002783ABE9B0E0A50194010E94A7D52FE718
:106B4000422E512C612C712CA30192010E9488D5F8
:106B50002C593F4F4F4F5F4F7901AEEFB1E0A50188
:106B600094010E94A7D5A30192010E9488D5D80163
:106B70000E94A7D52FEF30E040E050E00E9488D57A
:106B800089012F3F310519F014F00FEF10E060EF8D
:106B90007BE085E69AE00E94138EB70185E69AE0D5
:106BA0000E94ECA662EE7BE085E69AE00E94138EDE
:106BB000B80185E69AE00E94ECA685E69AE00E947C
:106BC000F58B60EB7BE085E69AE00E94138E85E60C
:106BD0009AE00E94F58B69EA7BE085E69AE00E94E4
:106BE000138EC6010E94883051CD6D857E858F85BC
:106BF000988924E630E040E050E00E9488D5B90151
:106C000047CF6D857E858F8598890E94EED640CFCF
:106C1000A50194012058310941095109ABE9B0E0BF
:106C20000E94A7D52FE730E040E050E00E9488D5D1
:106C30002C593F4F4F4F5F4F7901D60117961C9249
:106C4000A6CF9101AAEBBFEF0E9400D624E630E068
:106C500040E050E00E9488D529013A01B4E64B0E8D
:106C6000511C611C711C26E430E0D1010E9408D641
:106C700024E630E040E050E00E9488D5DA01C90106
:106C80004E96A11DB11D8B8B9C8BAD8BBE8B90E85E
:106C9000891691040CF090C08FE790E0881999094B
:106CA000809FD001819FB00D909FB00D11242B8942
:106CB0003C894D895E890E94B2D59B01AC01AFEF42
:106CC000B0E00E94A7D524E63AE640E050E00E94FA
:106CD00088D5D60117962C93A5019401240D351D56
:106CE000461D571DAEEFB1E00E94A7D523EE30E060
:106CF00040E050E00E9488D579018A011901AFEF88
:106D0000B0E0A50194010E94A7D52FE730E040E054
:106D100050E00E9488D55901EA89AE2FB0E0A80161
:106D200097010E94A7D52FEF30E040E050E00E948D
:106D300088D589012F3F310519F014F00FEF10E0CD
:106D40006CED7BE085E69AE00E94138E2AE030E04D
:106D5000B301A20185E69AE00E94E68C66ED7BE035
:106D600085E69AE00E94138E2AE030E04B895C8928
:106D70006D897E8985E69AE00E94E68C6EEC7BE068
:106D800085E69AE00E94138EB50185E69AE00E949E
:106D9000ECA666EC7BE085E69AE00E94138EB801D3
:106DA00085E69AE00E94ECA66DEB7BE085E69AE032
:106DB0000E94138EB101FDCEA50194012058310926
:106DC00041095109ABE9B0E00E94A7D52FE730E0B7
:106DD00040E050E00E9488D52C593F4F4F4F5F4F05
:106DE0005901D60117961C92312C212CA9CF67E9A5
:106DF0007BE085E69AE00E94138E6A856F7085E6D7
:106E00009AE00E94E5A664E97BE026CDFC01918131
:106E1000892F8F7021F0823029F080E00895907FD3
:106E2000926091839B0177FF02C030E020E02E3614
:106E300081E0380714F02DE631E02683878130FBAE
:106E400080F9878381E008950F931F93CF93DF9399
:106E50008C01FC01C081D1816FE270E0CE010E9403
:106E60008FDA0097D9F0FC011192CF010E94441BE8
:106E7000EC016CE677E085E69AE00E94138EBE0195
:106E800085E69AE00E94ECA685E69AE00E94F58BE2
:106E9000CE01DF91CF911F910F910895CE010E94F5
:106EA000441BEC01892BA1F3F80111821082F0CF71
:106EB000DC011296ED91FC91309729F090859F703E
:106EC00081E0953009F080E00895CF92DF92EF9253
:106ED000FF920F931F93CF93DF93EC016A017B0125
:106EE00088859985892BF1F48A819B810E9449A725
:106EF000082F10E005301105ACF40E944C92FC0103
:106F0000892B19F08085807F808780858F708087AE
:106F1000F987E887BF018A819B810E94C4A60F5F21
:106F20001F4FE8CFE885F985309781F08085982F4D
:106F30009F7051F4807F82608087E885F985C186E3
:106F4000D286E386F48602C09230B9F3DF91CF9106
:106F50001F910F91FF90EF90DF90CF900895FC016B
:106F600080859185009799F0FC0120852F70223053
:106F700029F461857285838594850895253039F4D7
:106F800060E00E94BEA2009711F0FC01F2CF60E029
:106F900070E0CB010895CF92EF92FF920F931F9371
:106FA000CF93DF9300D000D01F921F92CDB7DEB7F2
:106FB0007C0109831A832B833C834D835E836F831B
:106FC00078876EE77BE185E69AE00E94138ECE011A
:106FD00001960E9488308981811128C00B8101307F
:106FE00069F128F010E00230D1F5CC20E1F0CE01BB
:106FF00001960E94CDA2F70102811381892B69F0CD
:10700000C8010E94AF37672B682B692B61F480E0C1
:107010000E943928AB01BC0103C040E050E0BA0136
:10702000C8010E94653781E090E02AC08031B0F548
:107030008E30B8F58130A9F18230B9F161E77BE19A
:1070400085E69AE00E94138E698185E69AE00E94A7
:10705000E5A685E69AE00E94F58B01E010E061E686
:107060007BE185E69AE00E94138EB80185E69AE0FE
:107070000E94ECA685E69AE00E94F58B90E080E005
:1070800028960FB6F894DEBF0FBECDBFDF91CF912B
:107090001F910F91FF90EF90CF900895835183300F
:1070A00068F6F70102811381ABCF40E050E0BA01EE
:1070B000F70182819381B5CFCF92DF92EF92FF9259
:1070C0006A017B0163E0FC01828193810E94BEA280
:1070D000FC01892BA9F080858D7091F4C094D09427
:1070E000E094F094CC24CA9481859285A385B485DC
:1070F0008C219D21AE21BF2181879287A387B487F0
:10710000FF90EF90DF90CF900895CF92DF92EF92B3
:10711000FF926A017B0163E0FC01828193810E94FE
:10712000BEA2FC01892BA9F09085892F8D7089F46E
:10713000907F92609087CC24FF244185528563859F
:1071400074854C295D296E297F2941875287638781
:107150007487FF90EF90DF90CF900895CF92DF92E9
:10716000FF920F931F93CF93DF93F12C611571055D
:1071700009F492C06A01EB018C01CB010E945837DF
:10718000F82E882309F488C0D2FE0AC0D8018C9159
:107190008B3009F44DC008F03EC08A3009F44DC070
:1071A000D0FE09C0F801608186EF860F843018F0A8
:1071B000CE010E94111ED1FE6FC0D80114964D91D0
:1071C0005D916D917C91179711968C918F7087309E
:1071D00038F0893008F440C08A50823008F465C025
:1071E000CE010E94EB15EE81FF81309709F454C067
:1071F00080858F709EEF980F923010F081114CC0F7
:10720000D80111968C91982F9295907F80858F70E0
:10721000892B808741C08C30B9F040E050E062E0BB
:1072200070E08D3009F0BCCFCE010E948538B8CF18
:1072300040E050E061E070E0F7CF40E050E061E016
:1072400070E0CE010E945C3840E050E062E070E007
:10725000CE010E945C38A4CFEE81FF813097E1F02F
:1072600080858F709EEF980F923010F0811114C0BE
:107270004187528763877487EE81FF818085807F95
:1072800083608087EE81FF818085982F907F8F704B
:107290008067903609F4BDCF8F2DDF91CF911F917C
:1072A0000F91FF90DF90CF900895CE010E94EB15D3
:1072B000F3CFCF92DF92EF92FF926A017B0163E0FE
:1072C000FC01828193810E94BEA2009791F0FC0193
:1072D00020852F70223069F46185728583859485BD
:1072E0006C217D218E219F21FF90EF90DF90CF9028
:1072F000089560E070E0CB01F7CFAF92BF92CF92DC
:10730000EF920F931F93CF93DF93CDB7DEB7C8569D
:10731000D1090FB6F894DEBF0FBECDBF5C01A296B7
:107320000FAFA297A3961FAFA397A4962FAFA497D2
:10733000A5963FAFA597A6964FAFA697A7965FAF26
:10734000A797A8966FAFA897A9967FAFA9979E2DEC
:1073500028E0FE01EF59FF4FDE01A75ABF4F019011
:107360000D922A95E1F7A296EFADA297E150ED308C
:1073700008F0F0C0EC2CF0E08827EE53F64C8F4F6D
:107380000C94F1D5373A403A9E3AA83A943ACF391C
:107390002E3AAA3AAA3A493A5B3A813A6E3A992386
:1073A00031F0C5010E94B71D009709F447C067E09E
:1073B000CE01875A9F4F0E94F23063E877E085E65E
:1073C0009AE00E94138E6A966FAD6A9785E69AE0FE
:1073D0000E94E5A668E777E085E69AE00E94138EB2
:1073E000CE01875A9F4F0E945A31AB01BC012AE05F
:1073F00030E085E69AE00E94E68C85E69AE00E94FD
:10740000F58B6A960FAD6A976B961FAD6B976C966E
:107410002FAD6C976D963FAD6D976E964FAD6E9795
:107420006F965FAD6F97A0966FADA097A1967FAD59
:10743000A197C5010E949E3181E090E0C859DF4FBD
:107440000FB6F894DEBF0FBECDBFDF91CF911F9175
:107450000F91EF90CF90BF90AF900895911105C01C
:10746000C5010E94B71D009749F366E0A1CF99239B
:1074700029F0C5010E94B71D009701F362E098CF83
:10748000911105C0C5010E94B71D0097B9F261E0D6
:107490008FCF40E050E061E070E0C5010E945939B3
:1074A000672B682B692B29F4C5010E94B71D009733
:1074B00029F26BE07DCF40E050E061E070E0C50173
:1074C0000E945939672B682B692B31F0C5010E9446
:1074D000B71D009709F4B2CF6AE06ACF40E050E0F0
:1074E00062E070E0C5010E945939672B682B692B57
:1074F00031F0C5010E94B71D009709F49FCF6CE0E1
:1075000057CF40E050E062E070E0C5010E94593979
:10751000672B682B692B31F4C5010E94B71D0097BA
:1075200009F48CCF6DE044CF911106C0C5010E94D3
:10753000B71D009709F482CF63E03ACF992331F069
:10754000C5010E94B71D009709F478CF65E030CFE0
:1075500064E02ECF90E080E071CF63E0FC01828197
:1075600093810E94BEA2009719F0FC0181850895C5
:107570008FEF0895FF920F931F93CF93DF93CDB7B3
:10758000DEB764970FB6F894DEBF0FBECDBF8C0197
:10759000F62E8FE290E09A838983FE01339688E08D
:1075A000DF011D928A95E9F7F8016681FF2011F04D
:1075B00081E06827D80114968C910E9461AEF80191
:1075C00087819085A185B285883E9340A105B1054C
:1075D00008F48BC066EE7BE185E69AE00E94138E8C
:1075E000D80114966D917C9185E69AE00E94ECA6F4
:1075F00061EE7BE185E69AE00E94138E6F2D70E0CC
:1076000085E69AE00E94ECA685E69AE00E94F58B5A
:1076100068E07CE1CE0101960E941CCEF8018281D7
:1076200093810E94AD3AFF2009F46BC069ED7BE1C4
:10763000843151F062ED7BE1853131F066EC7BE124
:107640008F3011F46EEC7BE1CE010B960E9430CEB0
:1076500061EB7BE185E69AE00E94138ED8011296D9
:10766000ED91FC9113970280F381E02D608171818F
:10767000ED91FC910288F389E02D9E012F5F3F4F31
:10768000AE01455F5F4FC8011995BC0185E69AE0E0
:107690000E94ECA66FEA7BE185E69AE00E94138ED9
:1076A000D8011296ED91FC910280F381E02D60816A
:1076B000718185E69AE00E946C8DBE016F5F7F4FFD
:1076C00085E69AE00E946C8D6CEA7BE185E69AE0A3
:1076D0000E94138EBE01655F7F4F85E69AE00E948F
:1076E0006C8D85E69AE00E94F58B64960FB6F8944F
:1076F000DEBF0FBECDBFDF91CF911F910F91FF90E5
:10770000089562EC7BE1823009F49ECF6DEB7BE162
:107710009BCFAF92BF92CF92EF92FF920F931F93A6
:10772000CF93DF9300D000D01F921F92CDB7DEB76A
:107730005C0109831A832B833C834D835E836F83B3
:1077400078876FE07CE185E69AE00E94138ECE0197
:1077500001960E948830E114F10439F068E07CE180
:10776000C7010E9427CE009719F1F501028113810C
:1077700001151105D9F08981811158C08B818130A3
:1077800009F45CC038F1823019F1082F10E06BEE7B
:107790007BE185E69AE00E94138EB80185E69AE0C7
:1077A0000E94ECA685E69AE00E94F58B90E080E0CE
:1077B00028960FB6F894DEBF0FBECDBFDF91CF91F4
:1077C0001F910F91FF90EF90CF90BF90AF900895D1
:1077D000CC20B9F0CE0101960E94CDA2892B09F4EC
:1077E00044C0C8010E94AF37672B682B692BD9F4BE
:1077F00080E00E943928AB01BC01C8010E946537B6
:1078000012C0C8010E94AD3A8E3019F048F48130A0
:1078100051F4CE0101960E94CDA2892B21F0E1CF37
:1078200083518330B0F381E090E0C2CF8031C0F467
:107830008E30B8F68130A9F28230B9F06BEF7BE17F
:1078400085E69AE00E94138E698185E69AE00E949F
:10785000E5A685E69AE00E94F58B01E010E097CF5F
:107860008351833008F4BDCFE9CF40E050E0BA0146
:10787000C8010E94653760E0C5010E94BA3AD3CFC3
:10788000DC01ED91FC910484F585E02D62E0199511
:1078900081E090E00895CF92DF92EF92FF920F93F4
:1078A0001F93CF93DF936115710509F454C06A01EA
:1078B0007B01EC01CB010E945837082F882351F13E
:1078C000D70116968D919C910097C9F1FC01108506
:1078D000212F2F703EEF320F323010F0211124C0D3
:1078E00012951F70D0FE04C0C7010E94AD3A888374
:1078F000112339F18981807F182B1983D7011696BE
:10790000ED91FC9181859285A385B4858C839D83BF
:10791000AE83BF83802FDF91CF911F910F91FF9096
:10792000EF90DF90CF900895253049F460E00E94F9
:10793000BEA2009721F0DC0118961C91D1CF10E077
:10794000D1CFD7011696ED91FC9180858F70823052
:1079500021F0833079F000E0DDCF418552856385E9
:1079600074858981807F8A6089834C835D836E837F
:107970007F83D0CF41855285638574858981807FDF
:10798000876089834C835D836E837F83C3CFCF926F
:10799000DF92EF92FF920F931F93CF93DF9300D06C
:1079A00000D01F921F92CDB7DEB76C017B0160FF44
:1079B00003C0E894E0F8F4F8F4FC0DC00E948C29B0
:1079C000663971058105910530F080918C079091A1
:1079D0008D07059709F5A70144275770052E000C60
:1079E000660B770BC6010E94853863EA7AE085E66C
:1079F0009AE00E94138E8FEF9FEF28960FB6F894AF
:107A0000DEBF0FBECDBFDF91CF911F910F91FF90D1
:107A1000EF90DF90CF90089519821A821B821C820A
:107A20001D821E821F8218868A81807F8A8340E0A1
:107A300053E0B601CE0101960E944B3C40E057E076
:107A400060E070E0C6010E945939E62AF72A0981F0
:107A50001A812B813C814D815E816F817885C601C1
:107A60000E941CB1CACF4F925F926F927F928F9209
:107A70009F92AF92BF92CF92DF92EF92FF920F93BD
:107A80001F93CF93DF93CDB7DEB72C970FB6F89443
:107A9000DEBF0FBECDBF6D7F6130710509F4BAC086
:107AA000DC011296ED90FC90E114F10409F4B2C0EF
:107AB0004C01C7010E94AF372B013C0161E070E02F
:107AC000C7010E94CB1D411451046104710409F4E3
:107AD000A1C020E030E04AE754E40E9482D40E9432
:107AE000F5D669877A878B879C87672B682B692BEC
:107AF00009F490C00E9433B09B01AC01A12CB12CC1
:107B00006501E984FA840B851C85C301B2010E94DA
:107B10007627882309F47EC0F4016280738070E0C8
:107B200060E0C3010E94CB1D20E030E048EC52E44D
:107B30000E9482D40E94F5D66B017C0180E00E94F5
:107B40003928AB01BC01C3010E94653719821A8232
:107B50001B821C821D821E821F8218868A81807F62
:107B60008A83D40112966D917C9140E053E0CE015E
:107B700001960E944B3CCE0101960E947F152B017D
:107B80003C016CE474E085E69AE00E946C8DB301E0
:107B9000A20185E69AE00E94E2A66BE574E085E624
:107BA0009AE00E946C8DB701A60185E69AE00E94DA
:107BB000E2A685E69AE00E94F58BC40CD51CE61C73
:107BC000F71C8A81807F86608A83CD82DE82EF8285
:107BD000F886F4016281738140E052E0CE010196A3
:107BE0000E94AE386FE574E085E69AE00E946C8DE5
:107BF000B701A60185E69AE00E94E2A685E69AE032
:107C00000E94F58B60E072E0D40112968D919C91F8
:107C10000E94C73C90E080E02C960FB6F894DEBF3F
:107C20000FBECDBFDF91CF911F910F91FF90EF90CD
:107C3000DF90CF90BF90AF909F908F907F906F908C
:107C40005F904F9008950F931F93CF93DF9300D0D1
:107C500000D01F921F92CDB7DEB719821A821B8205
:107C60001C821D821E821F8218862A81207F2A8301
:107C7000FC0102811381C8010E94AD3A813041F0BC
:107C800020F0823011F0853081F490E080E002C075
:107C900081E090E028960FB6F894DEBF0FBECDBF0E
:107CA000DF91CF911F910F91089540E052E0B8010C
:107CB000CE0101960E944B3CCE0101960E94CDA2BE
:107CC000E9CF8F929F92AF92BF92CF92DF92EF92C5
:107CD000FF920F931F93CF93DF93CDB7DEB76797D4
:107CE0000FB6F894DEBF0FBECDBF8C017B016A01D9
:107CF0004C018DE0880E911C9F8A8E8AF801518379
:107D00004083148613861586168E158E672B09F40C
:107D10005EC0452B09F45BC06FE270E0C7010E94B2
:107D200047DA5C01892B09F44AC0F701DE0111969C
:107D300090E080E0BD012191222341F02F3231F00B
:107D40008431910519F02D930196F5CF860F971F79
:107D5000FC011082C6010E9446A2F801938382832F
:107D6000B5016F5F7F4F4FE050E0C4010E9480DAA1
:107D7000CE0146960E942437F801968F858F8E8912
:107D80009F89892B09F41586C8010E9458378823DA
:107D900019F0C8010E94301E67960FB6F894DEBF36
:107DA0000FBECDBFDF91CF911F910F91FF90EF904C
:107DB000DF90CF90BF90AF909F908F900895B701C4
:107DC000C6010E9446A2F80193838283DDCFF801A9
:107DD00013821282D9CFDC011B968D919C91009762
:107DE00039F0DC01ED91FC910280F381E02D1994D2
:107DF00008958F929F92AF92BF92CF92DF92EF92AF
:107E0000FF920F931F93CF93DF93CDB7DEB7CF557C
:107E1000D1090FB6F894DEBF0FBECDBF8C016B0148
:107E20006115710519F041155105D1F46AE47DE041
:107E300085E69AE00E94138E61E47DE085E69AE093
:107E40000E94138EB80185E69AE00E946C8D6FE364
:107E50007DE085E69AE00E94138E85E69AE030C0C8
:107E6000460F571FDA011C920E948C294B0169E3CF
:107E70007DE085E69AE00E94138EB40185E69AE0E3
:107E80000E94ECA666E37DE085E69AE00E94138EF0
:107E9000B80185E69AE00E946C8D63E37DE085E69B
:107EA0009AE00E94138EBAE38B16B1E09B06F4F4BD
:107EB00066E27DE08EEB99E00E94138E8EEB99E0F6
:107EC0000E94F58BC15ADF4F0FB6F894DEBF0FBE8C
:107ED000CDBFDF91CF911F910F91FF90EF90DF9079
:107EE000CF90BF90AF909F908F90089564E27DE017
:107EF00085E69AE00E94138EB60185E69AE00E941C
:107F00006C8D62E27DE085E69AE00E94138E85E644
:107F10009AE00E94F58B1A821982FE0133968EE355
:107F2000DF011D928A95E9F780918C0790918D076A
:107F3000059791F563E070E0C8010E94EB287C0191
:107F4000892BE9F5E0913709F0913809808180FFAC
:107F5000B9CF61E070E0C8010E94EB28892B09F4D9
:107F6000B1CF64E270E0C8010E948FDA892B09F07A
:107F7000A9CF64E07DE085E69AE00E94138EB80107
:107F800085E69AE00E946C8D85E69AE00E94F58B6A
:107F9000C8010E94CBAC96CF61E070E0C8010E949E
:107FA000EB287C01892B21F562E070E0C8010E947A
:107FB000EB287C0169EF7CE0892B09F44ACFE00EC5
:107FC000F11E60EF7CE0C7010E9427CE892BC1F42F
:107FD000F60101900020E9F73197EC19FD0932977D
:107FE00078F0C8010E94CBACC6010E94ED8E6ACF2A
:107FF0004FE350E0B801CE0101960E9480DADFCF56
:1080000064E270E0C8010E948FDA892B09F05ACF30
:1080100040918C0850918D08B701CE018F5B9F4F26
:108020000E94613ECE018F5B9F4F0E94583788238C
:1080300039F1B601CE018F5B9F4F0E9409A8181637
:108040001906F4F489818823D9F080918C079091E6
:108050008D070597A9F062ED7CE085E69AE00E9425
:10806000138EBE016F5F7F4F85E69AE00E946C8D94
:1080700085E69AE00E94F58BCE0101960E94CBAC7A
:10808000CE018F5B9F4F0E94EB3E1CCFCF93DF93BF
:10809000EC01598348837B836A831C861B861D867B
:1080A0001E8E1D8E0E945837882329F0CE01DF9145
:1080B000CF910C94301EDF91CF9108952F923F9273
:1080C0004F925F926F927F928F929F92AF92CF92D8
:1080D000DF92EF92FF920F931F93CF93DF93CDB771
:1080E000DEB7A1970FB6F894DEBF0FBECDBFFC017F
:1080F0006115710509F4BDC0DB0118969C919F7054
:10810000953009F0B6C0D02E19014A01F9A3E8A3B1
:10811000FB016680778080918E088F5F80938E0848
:108120006114710409F4A0C0D30118968C911897BA
:108130008F70843009F094C019966D917C91E8A1FC
:10814000F9A1808191810E9446A22C01009709F437
:1081500087C0DC0118968C918F70853009F080C043
:1081600040918C0850918D08B201CE0101960E9479
:10817000464081149104B1F0CE0101960E94583717
:10818000882381F0AD2CC12C7101F4010081118193
:10819000228133814481558166817781CE010196A8
:1081A0000E948A4360E0C2010E94BEA2009709F4C7
:1081B00044C0DC0118962C9118972F702230E9F5F5
:1081C00019968D919D910D90BC91A02D0797A105B9
:1081D000B10599F561E0C2010E94BEA20D2D910189
:1081E000A401BC0188A199A10E945E408114910460
:1081F00099F5882389F180918E08815080938E08AB
:10820000CE0101960E94EB3E81E0A1960FB6F89454
:10821000DEBF0FBECDBFDF91CF911F910F91FF90B9
:10822000EF90DF90CF90AF909F908F907F906F9066
:108230005F904F903F902F9008958114910461F4C6
:10824000CE0101960E945837882331F0CE01019665
:108250000E943B41892B79F6CE0101960E94EB3EAC
:10826000F301628073805CCF80918E08815080938F
:108270008E0880E0CACFDF92EF92FF920F931F9398
:10828000CF93DF9300D000D01F921F92CDB7DEB7FF
:108290007C0119821A821B821C821D821E821F820F
:1082A00018868A81807F8A83D7011296ED91FC918E
:1082B0006081718185E69AE00E946C8D6BE57AE0C1
:1082C00085E69AE00E94138EC7010E9458378111FB
:1082D0001BC062E57AE085E69AE00E94138E85E68F
:1082E0009AE00E94F58B0FEF1FEFC80128960FB69A
:1082F000F894DEBF0FBECDBFDF91CF911F910F91DC
:10830000FF90EF90DF900895C7010E94AD3AD82EFC
:10831000F70183859485009791F0DC01ED91FC9144
:108320000688F789E02D19958C0197FD08C081E03A
:108330000115110509F480E00E946619D6CFF701F6
:108340008285873009F42EC0EFEFED0DE43150F552
:10835000F0E08827E155FE4B8F4F0C94F1D5C341D7
:10836000CC41D241D241CC41C341D241D241D24190
:10837000D241D241D241D241C341D241D241D24174
:10838000D241C341C34163E37AE085E69AE00E94AB
:10839000138E01E010E0A9CF80E00E94661910E082
:1083A00000E0A3CF40E052E0B701CE0101960E9469
:1083B0004B3CD7011A968C911A97873071F160F473
:1083C000833009F455C0843061F063E47AE085E6D7
:1083D0009AE00E94138EE3CF883009F449C08930B7
:1083E000A1F7CE0101960E94CDA28C0168E37AE04C
:1083F00085E69AE00E94138EB80185E69AE00E9415
:10840000ECA685E69AE00E94F58B91E080E0012BD6
:1084100009F490E0092F182F68CF1496ED91FC9184
:1084200080858F7010E000E0853001F760E57AE02C
:1084300085E69AE00E94138EF7016481758100E061
:1084400030E020E050E040E0C7010E945E40F82E9E
:10845000082F10E06DE47AE085E69AE00E94138E22
:108460008F2D0E94661985E69AE00E94F58B3DCF1C
:10847000CE0101960E945A318B01B8CF2F923F92C4
:108480004F925F926F927F928F929F92AF92BF9224
:10849000CF92DF92EF92FF920F931F93CF93DF93D0
:1084A000CDB7DEB760970FB6F894DEBF0FBECDBF75
:1084B0006130710509F494C0DC0112966D917C91D4
:1084C0006115710509F48CC04C0119821A821B8256
:1084D0001C821D821E821F8218868A81807F8A8369
:1084E00040E052E0CE0101960E944B3CCE01019645
:1084F0000E94CDA21C01F401828193810E94AF37BA
:108500002B013C01D40117962D913D914D915C9129
:108510001A97D1010E94B2D52FEF30E040E050E031
:108520000E9466D529873A874B875C870E9433B0C3
:108530009B01AC0189859A85AB85BC850097A10517
:10854000B10509F468C0A12CB12C65017C018D0135
:10855000C301B2010E947627898741145104610446
:108560007104F1F1D40117968D919D910D90BC91FC
:10857000A02D8D879E87AF87B88B0E9433B09B015B
:10858000AC018D859E85AF85B8890097A105B105A1
:1085900061F0A12CB12C65017C018D01C301B201F8
:1085A0000E947627882309F451C0D40112966D9059
:1085B0007C9080E00E943928AB01BC01C3010E947D
:1085C0006537232869F0F40184810E941B14D401CB
:1085D00016969C91891304C061E0C4010E94BA3AC6
:1085E00090E080E060960FB6F894DEBF0FBECDBF7E
:1085F000DF91CF911F910F91FF90EF90DF90CF907F
:10860000BF90AF909F908F907F906F905F904F90B2
:108610003F902F90089591E099879FCFB985BB2314
:10862000F1F060E0C4010E94BA3AF40182819381C2
:108630000E943B41892BA1F640E050E0BA01D401F1
:1086400012968D919C910E946537CACFF401848166
:108650000E941B14D40116969C918913DFCF232806
:1086600009F4BECFF40184810E941B14D401169634
:108670009C918913B5CFB985B111B2CFADCFCF934E
:10868000DF93EC016EE87BE185E69AE00E94138EB1
:108690006C817D8185E69AE00E94ECA668E87BE12A
:1086A00085E69AE00E94138E85E69AE00E94F58B9B
:1086B00061E08C810E948FAE6E818C810E9461AEE0
:1086C0008A819B81009729F040E050E0BA010E9426
:1086D0006537E881F9810484F585E02D62E0CE01FB
:1086E00019958A819B81009781F00E943B41181661
:1086F00019065CF40A80DB81C02D80E00E943928D5
:10870000AB01BC01CE010E94653781E090E0DF91B2
:10871000CF9108952F923F924F925F926F927F92E6
:108720008F929F92AF92BF92CF92DF92EF92FF9281
:108730000F931F93CF93DF93CDB7DEB7CB5CD109F7
:108740000FB6F894DEBF0FBECDBF3C01CF54DF4F54
:108750000883C15BD040CE54DF4F1883C25BD0404A
:10876000CD54DF4F2883C35BD040CC54DF4F3883D8
:10877000C45BD040CB54DF4F4883C55BD040CA5464
:10878000DF4F5883C65BD040C954DF4F6883C75B57
:10879000D040C854DF4F7883C85BD040C754DF4F08
:1087A000F982E882C95BD040C354DF4FC882CD5BF9
:1087B000D040CB53DF4FA882C55CD0400E948C29AB
:1087C0006B01C554DF4F79836883CB5BD040683C35
:1087D0007105A4F46AE17AE08EEB99E00E94138EB1
:1087E000B6018EEB99E00E94ECA68EEB99E00E9418
:1087F000F58BAA24AA94BA2C0C944C4D0E9433B049
:10880000C853DF4F688379838A839B83C85CD040D9
:10881000CD54DF4F8881C35BD040282E312C20916E
:108820008C0730918D07CA53DF4F39832883C65C8C
:10883000D040C754DF4FE881F981C95BD040309701
:1088400021F0808181110C944C51D3011D968C91A3
:10885000882341F0C3010D96C754DF4F9983888365
:10886000C95BD0402114310411F00C949551C754C8
:10887000DF4FE881F981C95BD040309711F00C944B
:108880005051F301258C368C2114310411F40C94D1
:108890009551CD54DF4F8881C35BD04081110C943A
:1088A0009551622DCE018F549F4F0E94D030C756F4
:1088B000DF4F2883C959D040C656DF4F3883CA5985
:1088C000D040C556DF4F4883CB59D040C456DF4F08
:1088D0005883CC59D040C356DF4F6883CD59D04020
:1088E000C256DF4F7883CE59D040C156DF4F8883C0
:1088F000CF59D040C056DF4F9883C05AD0400C9417
:108900009551D30112962D913C91232B09F471CFEF
:10891000B4E02B16310499F5CB53DF4FE880C55CEA
:10892000D040CF54DF4F0881C15BD040CE54DF4FE1
:108930001881C25BD040CD54DF4F2881C35BD0404B
:10894000CC54DF4F3881C45BD040CB54DF4F4881DB
:10895000C55BD040CA54DF4F5881C65BD040C95474
:10896000DF4F6881C75BD040C854DF4F7881C85B58
:10897000D040C3010E949E315C010C944C4D28E014
:10898000FE01EF54FF4FDE01A755BF4F01900D923E
:108990002A95E1F7CF54DF4F1881C15BD0401430E6
:1089A00009F4DEC248F4112309F467C0912C812C2C
:1089B000AA24AA94BA2C4BC388EF810F8230B0F757
:1089C00088E0FE01EF54FF4FDE01119601900D92F9
:1089D0008A95E1F7CE54DF4F8881C25BD0408F701B
:1089E00009F440C3CE018F549F4F0E947F156B0145
:1089F0007C01C114D104E104F10409F433C319303A
:108A000041F4F094E094D094C094C11CD11CE11CBA
:108A1000F11CB301CE018F549F4F0E947BA760E0F1
:108A2000CE018F549F4F0E94F2306A962FAF6A9703
:108A30006B963FAF6B976C964FAF6C976D965FAF31
:108A40006D976E966FAF6E976F967FAF6F97A0968C
:108A50008FAFA097A1969FAFA19722E02216310475
:108A600009F456C30CF004C3442443942114310484
:108A700009F44FC3912C812C22C519821A821B82C2
:108A80001C821D821E821F8218862A81207F2A83D3
:108A9000CE54DF4F2881C25BD0402F7009F486CFBF
:108AA000EAE02E16310409F417C25CF421143104F3
:108AB00059F102E02016310409F4D4C0912C812C24
:108AC00006C21BE02116310409F4B3C12CE02216C2
:108AD0003104A1F7B301CE0101960E947BA7CE011C
:108AE0008F549F4F0E94CA15BC01CE0101960E946F
:108AF0005C3288E0FE013196DE01AF54BF4F019039
:108B00000D928A95E1F7E0C1892B59F067ED79E084
:108B100085E69AE00E94138E85E69AE00E94F58B26
:108B2000CDCFC3010E943B418C0161E070E018167B
:108B3000190614F070E060E085E69AE00E94ECA669
:108B40006DE574E085E69AE00E946C8DCE018F544D
:108B50009F4F0E945A31AB01BC012AE030E085E60C
:108B60009AE00E94E68C85E69AE00E94F58BCE01A1
:108B70008F549F4F1016110614F00C9440510E9410
:108B80005A31912C812C672B682B692B89F562E077
:108B9000CE018F549F4F0E94F230CF56DF4F288373
:108BA000C159D040CE56DF4F3883C259D040CD5640
:108BB000DF4F4883C359D040CC56DF4F5883C45948
:108BC000D040CB56DF4F6883C559D040CA56DF4FDF
:108BD0007883C659D040C956DF4F8883C759D040E3
:108BE000C856DF4F9883C859D04088248394982C66
:108BF00044244394DD24D3943AC061E0CE018F54E1
:108C00009F4F0E94F230C757DF4F2883C958D0408A
:108C1000C657DF4F3883CA58D040C557DF4F488307
:108C2000CB58D040C457DF4F5883CC58D040C3579F
:108C3000DF4F6883CD58D040C257DF4F7883CE587E
:108C4000D040C157DF4F8883CF58D040C057DF4F47
:108C50009883C059D04088248394982C442443940A
:108C6000D12C05C0912C812C412CDD24DA94B30148
:108C7000CE0101960E947BA78A819CE0980F9F708D
:108C8000923058F4CE54DF4F9881C25BD0409F7031
:108C9000923019F4807F82608A83D3011A969C9166
:108CA000973069F4CE54DF4F8881C25BD0408F701B
:108CB0008250843020F48A81807F82608A83F3012D
:108CC000A385B485892F90E0109741F0ED91FC9138
:108CD0001197048CF58DE02DCD0119957C01CF54B1
:108CE000DF4F0881C15BD040CE54DF4F1881C25B9B
:108CF000D040CD54DF4F2881C35BD040CC54DF4FF0
:108D00003881C45BD040CB54DF4F4881C55BD04035
:108D1000CA54DF4F5881C65BD040C954DF4F6881C9
:108D2000C75BD040C854DF4F7881C85BD040CE01CC
:108D300001960E949632CF57DF4F2883C158D0400A
:108D4000CE57DF4F3883C258D040CD57DF4F4883CE
:108D5000C358D040CC57DF4F5883C458D040CB576E
:108D6000DF4F6883C558D040CA57DF4F7883C65855
:108D7000D040C957DF4F8883C758D040C857DF4F0E
:108D80009883C858D040CE0101960E948830442074
:108D900041F1CE54DF4F8881C25BD0408F709FE09D
:108DA000980F9F70923020F08A5F8F708230C8F4E5
:108DB0008A818F7081508230A0F42D8130E0AFEF36
:108DC000B0E00E94BAD52FEF6115F4E67F07810568
:108DD000910534F424E630E040E050E00E9488D56C
:108DE0002D8388E0FE013196DE01AF54BF4F019024
:108DF0000D928A95E1F702E1902A512CAA24AA94B7
:108E0000BA2CD3011A968C911A97873009F075C540
:108E1000C554DF4FE881F981CB5BD040EE35F1409E
:108E20000CF076C363E979E08EEB99E00E94138E33
:108E3000DCCCB301CE0101960E947BA7CA54DF4F60
:108E40008881C65BD0409A819F7039F0923049F09A
:108E5000912C812C552453943BC09A81907F926031
:108E60009A8390E08536910514F084E690E08E8335
:108E700088E0FE013196DE01AF54BF4F01900D92A4
:108E80008A95E1F762E0CE018F549F4F0E94D03067
:108E9000EA962FAFEA97EB963FAFEB97EC964FAF82
:108EA000EC97ED965FAFED97EE966FAFEE97EF967E
:108EB0007FAFEF97C158DF4F8883CF57D040C0585E
:108EC000DF4F9883C058D040812CE2E19E2E512C78
:108ED000412CDD24DA9492CFB301CE0101960E9499
:108EE0007BA7C954DF4F6881C75BD040C854DF4FB0
:108EF0007881C85BD0407170CE0101960E94063720
:108F0000482E912C812C55245394882311F388E00A
:108F1000FE013196DE01AF54BF4F01900D928A954C
:108F2000E1F762E0CE018F549F4F0E94D030E2966D
:108F30002FAFE297E3963FAFE397E4964FAFE49706
:108F4000E5965FAFE597E6966FAFE697E7967FAF5A
:108F5000E797E8968FAFE897E9969FAFE997B4CF88
:108F600019E02116310409F459C0C3010E943B41A4
:108F70001816190654F562E0CE018F549F4F0E94D7
:108F8000F230AA962FAFAA97AB963FAFAB97AC96AD
:108F90004FAFAC97AD965FAFAD97AE966FAFAE9754
:108FA000AF967FAFAF97E0968FAFE097E1969FAF18
:108FB000E19788248394982CAA24AA94BA2C512C43
:108FC00044244394DD24D3941CCF61E0CE018F541C
:108FD0009F4F0E94F230A2962FAFA297A3963FAF69
:108FE000A397A4964FAFA497A5965FAFA597A69613
:108FF0006FAFA697A7967FAFA797A8968FAFA897B2
:10900000A9969FAFA99788248394982CAA24AA9400
:10901000BA2C512C44244394D12CF3CE40E050E0A0
:1090200061E070E0C3010E945939672B682B692BFE
:1090300089F040E050E061E070E0C3010E945C38DC
:109040008824839494E0992EAA24A394B12C512CC3
:10905000412CCCC040E050E061E070E0C3010E94D0
:109060008538EECF85E0C82ED12CE12CF12CC7CC71
:109070008AE02816310409F4C6C19BE029163104A0
:1090800009F0F8CCCE54DF4F8881C25BD0408F709E
:10909000823009F030C2C701B60124E630E040E07A
:1090A00050E00E9488D5CA54DF4F8881C65BD0400B
:1090B00090E0280F391F37FF02C030E020E025364E
:1090C000310514F024E630E0CA54DF4F2883C65B34
:1090D000D04062E0CE018F549F4F0E94D0302A963C
:1090E0002FAF2A972B963FAF2B972C964FAF2C97ED
:1090F0002D965FAF2D972E966FAF2E972F967FAF41
:109100002F9760968FAF609761969FAF6197D4C19C
:10911000412CD3011B968D919C911C97009781F552
:109120001A968C9190E010E5812E912CA12CB12CF7
:109130008530910549F0812C912C5401449721F000
:10914000812C912C54018A94CE54DF4FE881C25B6C
:10915000D040EF70E150EB3008F046C1F0E08827D6
:10916000EB54F74B8F4F0C94F1D5C848C848F449DD
:10917000F449F449C1497F497F497F49F948F94891
:10918000DC01ED91FC91048CF58DE02D1995CBCF90
:10919000CB54DF4F1881C55BD040C701B60124E630
:1091A00030E040E050E00E9488D5DA01C901810F2B
:1091B000911DA11DB11DB7FF03C080E090E0DC014F
:1091C0008F3F9105A105B10529F024F08FEF90E0C4
:1091D000A0E0B0E0CB54DF4F8883C55BD040812C4A
:1091E000B2E19B2E512CAA24AA94BA2CDD24DA9445
:1091F00008CECB54DF4F088119812A813B81C55BA2
:10920000D040CF53DF4F088319832A833B83C15C4F
:10921000D04014E6C116D104E104F1040CF041C0C1
:10922000A4E6B0E0CF53DF4F288139814A815B81CA
:10923000C15CD0400E94A7D5C60ED71EE81EF91EFD
:1092400081149104A104B104B9F0A50194010E9414
:10925000A7D5362F272FB701A60177FF03C040E01F
:1092600050E0BA01C32ED22E7C014C155D056E056F
:109270007F0514F46A017B01CB54DF4FC882D98289
:10928000EA82FB82C55BD040CE54DF4F8881C25B4F
:10929000D040807F8660CE54DF4F8883C25BD04051
:1092A0009ECFC701B60124E630E040E050E00E94C6
:1092B00088D5CF53DF4F88819981AA81BB81C15C5A
:1092C000D040280F391F4A1F5B1F81149104A1044D
:1092D000B10461F057FF03C020E030E0A90182161D
:1092E0009306A406B50614F4A5019401CB54DF4FF0
:1092F000288339834A835B83C55BD04070CFCB54CE
:10930000DF4F688179818A819B81C55BD0400E9453
:10931000EED6CF53DF4F688379838A839B83C15C0A
:10932000D040C701B60124E630E040E050E00E94A2
:1093300088D5CF53DF4F688179818A819B81C15C59
:10934000D040620F731F841F951F81149104A104E4
:10935000B10461F097FF03C060E070E0CB018616B6
:109360009706A806B90614F4C501B4010E9423D4D7
:10937000CB54DF4F688379838A839B83C55BD0405E
:109380002ECFCB54DF4F88819981AA81BB81C55BE9
:10939000D040C80ED91EEA1EFB1E81149104A10400
:1093A000B104C9F0A4E6B0E0A50194010E94A7D5DC
:1093B000362F272FB701A60177FF03C040E050E00A
:1093C000BA01C32ED22E7C014C155D056E057F05BA
:1093D00014F46A017B01CB54DF4FC882D982EA8240
:1093E000FB82C55BD040FBCE88E0FE013196DE01FA
:1093F000AF54BF4F01900D928A95E1F7912C812CCB
:1094000055245394F0CECE54DF4F8881C25BD040B8
:109410008F70823009F055C0C701B60124E630E0F4
:1094200040E050E00E9488D5C954DF4F8881C75B77
:10943000D040C854DF4F6881C85BD040962F9170F0
:10944000280F391F2E3691E039072CF437FF05C05D
:109450002DE631E002C030E020E0C954DF4F288320
:10946000C75BD040C854DF4F8881C85BD04030FB19
:1094700080F9C854DF4F8883C85BD04062E0CE01DA
:109480008F549F4F0E94D03062962FAF62976396A1
:109490003FAF639764964FAF649765965FAF6597EC
:1094A00066966FAF669767967FAF679768968FAF40
:1094B000689769969FAF6997812CA2E19A2E512CEB
:1094C00018C088E0FE013196DE01AF54BF4F019015
:1094D0000D928A95E1F76BEC79E08EEB99E00E94B2
:1094E000138E8EEB99E00E94F58B912C812C5524E4
:1094F0005394412C78CE88E0FE013196DE01AF54C2
:10950000BF4F01900D928A95E1F76FEB79E0E5CFBF
:10951000C354DF4F1881CD5BD040112309F46DC0D7
:109520001496ED91FC9180858F70853009F076C09E
:10953000CA53DF4FE881F981C65CD040359709F402
:109540006DC0C3010E943B4121E0181619060CF0C2
:1095500020E0D22EC754DF4F28813981C95BD0402B
:10956000D30114966D917C91CB53DF4F0881C55C7C
:10957000D040AE014F545F4FC3010E945E40B1E046
:109580002B16310409F04AC0CE54DF4F8881C25BEC
:10959000D0408F7009F442C0CB53DF4FC880C55C08
:1095A000D040ED2CC755DF4F0881C95AD040C65571
:1095B000DF4F1881CA5AD040C555DF4F2881CB5A9A
:1095C000D040C455DF4F3881CC5AD040C355DF4F0F
:1095D0004881CD5AD040C255DF4F5881CE5AD04035
:1095E000C155DF4F6881CF5AD040C055DF4F7881D9
:1095F000C05BD040C3010E947D39CF54DF4F8881CA
:10960000C15BD040853009F447C170F48330C9F1A3
:10961000C554DF4F1882CB5BD040B8C0C354DF4F76
:109620001882CD5BD040E9CF863009F47CC087300A
:1096300079F7C3010E94AD3A182F863009F062C055
:1096400067E679E085E69AE00E94138E66E070E0B6
:1096500085E69AE00E94ECA685E69AE00E94F58BEA
:1096600062E0CE018F549F4F0E94F23029AF3AAF93
:109670004BAF5CAF6DAF7EAF8FAF21969FAF2197A1
:109680003DC0C3010E94AD3A853021F093E0A92E80
:10969000B12C02C26EE779E085E69AE00E94138E53
:1096A00065E070E085E69AE00E94ECA685E69AE027
:1096B0000E94F58BB301CE018F549F4F0E947BA770
:1096C00061E0CE018F549F4F0E94F23022962FAF5F
:1096D000229723963FAF239724964FAF2497259642
:1096E0005FAF259726966FAF269727967FAF279770
:1096F00028968FAF289729969FAF2997689480F86E
:1097000090F886CF69E479E085E69AE00E94138EAE
:10971000612F70E085E69AE00E94ECA685E69AE06B
:109720000E94F58BB3CF40E050E061E070E0C301F0
:109730000E945939672B682B692B09F0AAC0EFEFFB
:10974000DE129DC0C3010E943B41181619060CF49D
:1097500099C0B301CE018F549F4F0E947BA761E057
:10976000CE018F549F4F0E94F23029AB3AAB4BABE6
:109770005CAB6DAB7EAB8FAB98AF689480F890F824
:10978000F6E0C554DF4FF883CB5BD0408401016025
:10979000CD54DF4F8881C35BD040823050F4CF542A
:1097A000DF4F8881C15BD040882319F084010160BC
:1097B0001160CE54DF4F8881C25BD0408F7009F4B6
:1097C00091C01260C354DF4F2881CD5BD04021117E
:1097D0001D7FA801B301CE018F549F4F0E94AE3868
:1097E0004801AA24A394B12C5110EFC5D3011B96B4
:1097F0008D919C91009709F070C340E050E062E0C9
:1098000070E0C3010E945939672B682B692B09F45A
:1098100096C36BEE77E08EEB99E00E94138E8EEB91
:1098200099E00E94F58B92FC16C569EB77E085E61E
:109830009AE00E94138EB50185E69AE00E94ECA69C
:1098400062EB77E085E69AE00E94138E0E9433B0C7
:10985000AB01BC01C853DF4F088119812A813B81CC
:10986000C85CD040401B510B620B730B85E69AE03D
:109870000E94E2A685E69AE00E94F58B0DC1DD20EC
:1098800009F467CF6FE279E085E69AE00E94138ED3
:10989000FDCE6AE179E0F8CF0FEFD01209C0C30125
:1098A0000E943B41181619062CF06DEF78E0ECCFC2
:1098B000DD20D9F362E0CE018F549F4F0E94F23039
:1098C00029A73AA74BA75CA76DA77EA78FA798AB40
:1098D000689480F890F815E0C554DF4F1883CB5B8F
:1098E000D04054CF40E052E0B301CE018F549F4F9F
:1098F0000E944B3C811165CF65CF3FEFD312E7C08B
:10990000C3010E943B41DD24D394181619060CF4C0
:10991000E1C0D12C6FEE78E085E69AE00E94138ECC
:109920000D2D0D2C000C110BCF53DF4F1983088325
:10993000C15CD040B80185E69AE00E94ECA668EED2
:1099400078E085E69AE00E94138E642D70E085E64B
:109950009AE00E94ECA685E69AE00E94F58BC75437
:10996000DF4FE880F980C95BD040E114F10409F4CD
:10997000BAC063EF74E2C7010E9427CE01E010E095
:10998000892B09F44BC06CEF74E2C7010E9427CE0B
:1099900002E010E0892B09F441C067E175E2C701DC
:1099A0000E9427CE05E010E0892BC1F160E275E24C
:1099B000C7010E9427CE06E010E0892B79F165E906
:1099C00075E2C7010E9427CE03E110E0892B31F137
:1099D0006EE975E2C7010E9427CE04E110E0892BF1
:1099E000E9F068E675E2C7010E9427CE0EE010E0BC
:1099F000892BA1F061E775E2C7010E9427CE0FE035
:109A000010E0892B59F067EA75E2C7010E9427CE62
:109A100010E000E0892B11F405E110E0C3010E9481
:109A2000AD3A282F30E0C554DF4F39832883CB5B14
:109A3000D040232B61F4CF53DF4F88819981C15CE3
:109A4000D040C554DF4F99838883CB5BD04001154C
:109A5000110509F491C0C554DF4FA881B981CB5BD2
:109A6000D040A017B107C9F16CEC78E085E69AE028
:109A70000E94138EC554DF4F68817981CB5BD04043
:109A800085E69AE00E94ECA685E69AE00E94F58BB6
:109A90006DEFA62EBB24BA94C501C553DF4F0FB698
:109AA000F894DEBF0FBECDBFDF91CF911F910F9114
:109AB000FF90EF90DF90CF90BF90AF909F908F90EE
:109AC0007F906F905F904F903F902F900895DD2092
:109AD00009F420CF442443941DCFC754DF4F19828B
:109AE0001882C95BD040B1E02B163104A9F4C354ED
:109AF000DF4FE881CD5BD040EE2399F0CE54DF4FAD
:109B00008881C25BD0408F70F1E0C354DF4FF8838F
:109B1000CD5BD040811105C0C354DF4F1882CD5BAF
:109B2000D040CF54DF4F0881C15BD040C554DF4FD8
:109B30000883CB5BD040063108F0B9C1E02FF0E0DC
:109B40008827EA55F24B8F4F0C94F1D5F94D184FF9
:109B5000094F3C4EF94DEC4EB24E834EF94DF94D46
:109B6000544F544F644F644F324F324F574F574FFB
:109B7000574F324F324F324FF30183859485009710
:109B800009F4B1CFDC01ED91FC910488F589E02D59
:109B9000CB53DF4FA880C55CD040C42CCF54DF4FDF
:109BA0000881C15BD040CE54DF4F1881C25BD040EA
:109BB000CD54DF4F2881C35BD040CC54DF4F388178
:109BC000C45BD040CB54DF4F4881C55BD040CA5402
:109BD000DF4F5881C65BD040C954DF4F6881C75BF7
:109BE000D040C854DF4F7881C85BD04019950C94A1
:109BF000BC44C554DF4F1882CB5BD040C354DF4F09
:109C00002881CD5BD040222309F4EECD3D2D31706B
:109C1000E32ECB53DF4FC880C55CD040C755DF4F24
:109C20000881C95AD040C655DF4F1881CA5AD04062
:109C3000C555DF4F2881CB5AD040C455DF4F3881FE
:109C4000CC5AD040C355DF4F4881CD5AD040C25581
:109C5000DF4F5881CE5AD040C155DF4F6881CF5A6F
:109C6000D040C055DF4F7881C05BD040C3010E9417
:109C70007D39E89491F8B8CDC3010E94AD3A8530A2
:109C800009F004CD67EB78E085E69AE00E94138E38
:109C900065E070E085E69AE00E94ECA685E69AE031
:109CA0000E94F58BB301CE018F549F4F0E947BA77A
:109CB000D3011A968C918530B9F46EE0CE018F54A1
:109CC0009F4F0E94F23029A33AA34BA35CA36DA33C
:109CD0007EA38FA398A7689480F890F8C554DF4FAF
:109CE0001882CB5BD0406FC061E0CE018F549F4F94
:109CF0000E94F230298F3A8F4B8F5C8F6D8F7E8F51
:109D00008F8F98A3E8CFC3010E94AD3A182F8630F9
:109D100031F560EA78E085E69AE00E94138E66E00D
:109D200070E085E69AE00E94ECA685E69AE00E9443
:109D3000F58B62E0CE018F549F4F0E94F230298B49
:109D40003A8B4B8B5C8B6D8B7E8B8F8B988F40E02F
:109D500050E068E070E0C3010E945C38BCCF62E86C
:109D600078E0D2CC40E050E061E070E0C3010E94B6
:109D70005939672B682B692B61F5D11027C0B301C6
:109D8000CE018F549F4F0E947BA761E0CE018F547C
:109D90009F4F0E94F23029873A874B875C876D87F7
:109DA0007E878F87988B40E050E068E070E0C301C9
:109DB0000E948538689480F890F8B6E0C554DF4F6B
:109DC000B883CB5BD0404424439418CF68E678E056
:109DD0005BCD63E578E058CDDD20C1F062E0CE01D7
:109DE0008F549F4F0E94F23029833A834B835C83C8
:109DF0006D837E838F839887689480F890F8E5E080
:109E0000C554DF4FE883CB5BD040DDCF66E378E01D
:109E10003BCDCD54DF4F8881C35BD040823008F00A
:109E20005DCFC3010E94AD3A853009F054CF2ECCEE
:109E3000CD54DF4F8881C35BD040823008F04ECFD5
:109E4000DD2081F06DE178E085E69AE00E94138ED6
:109E500061E0C3010E94111E60E071E1C3010E9434
:109E6000C73C14CCCD54DF4F8881C35BD0408230D7
:109E700008F034CFC554DF4FF881CB5BD040FF23CF
:109E800009F4A1CFCE54DF4F8881C25BD0408F70E0
:109E900031F4B301CE018F549F4F0E947BA7689489
:109EA00080F803E0902A1ACF689492F817CFCE5426
:109EB000DF4F8881C25BD0408F7019F4689490F8AE
:109EC0000DCF13E0912A0ACFC554DF4F1882CB5B28
:109ED000D040812C54E0952E76CFDC01ED91FC91A1
:109EE000008CF18DE02DCF54DF4F0881C15BD04055
:109EF000CE54DF4F1881C25BD040CD54DF4F288154
:109F0000C35BD040CC54DF4F3881C45BD040CB54CE
:109F1000DF4F4881C55BD040CA54DF4F5881C65BD4
:109F2000D040C954DF4F6881C75BD040C854DF4F71
:109F30007881C85BD040199581115FCC6ACCF30160
:109F400083859485892B09F473C08114910439F0B9
:109F5000A401B301CE018F549F4F0E94AE38D301AC
:109F60001B968D919C91C754DF4FE880F980C95BA7
:109F7000D040DC01ED91FC910488F589E02DCB53B4
:109F8000DF4FA880C55CD040C42CCF54DF4F088180
:109F9000C15BD040CE54DF4F1881C25BD040CD545E
:109FA000DF4F2881C35BD040CC54DF4F3881C45B86
:109FB000D040CB54DF4F4881C55BD040CA54DF4FFF
:109FC0005881C65BD040C954DF4F6881C75BD04021
:109FD000C854DF4F7881C85BD04019955C01F3010C
:109FE00083859485DC01ED91FC91048CF58DE02D49
:109FF0001995059711F4689480F892FC24C1C55412
:10A00000DF4FB881CB5BD040BB2321F06B2FC30166
:10A010000E94111ECA53DF4FE881F981C65CD0400F
:10A02000B401359709F401CCC3010E94C73CFDCBB4
:10A030008285853009F474C0863009F7CF54DF4F2C
:10A04000D880C15BD040DD2009F46AC0C3010E9402
:10A0500059A78C018114910439F0A401B301CE01F8
:10A060008F549F4F0E94AE380115110541F2F12C1B
:10A07000E12C17FF06C0119501951109EE24E39418
:10A08000F12CC80101978634910508F0B8CFC02E95
:10A0900061E0802F0E948FAEEFEFED0DE53110F5FE
:10A0A000F0E08827E95AFF4A8F4F0C94F1D56C50A5
:10A0B0006E50725072506E506C506E5072507250A2
:10A0C00072507250725072506C506C50725072508C
:10A0D000725072506C506C50F1E0EF266E2D8C2D4A
:10A0E0000E9461AE66EE77E085E69AE00E94138EEC
:10A0F000B80185E69AE00E94ECA664EE77E085E67A
:10A100009AE00E94138EB70185E69AE00E94ECA6C1
:10A1100085E69AE00E94F58B689480F890F893C0E9
:10A120008114910439F0A401B301CE018F549F4FE3
:10A130000E94AE3802E02016310409F488C013E012
:10A140002116310429F02A94232809F058CFE4CFAE
:10A15000C3010E94AF37892BF1F464ED77E084EB03
:10A1600099E00E94138ED3011296ED91FC916081CB
:10A17000718184EB99E00E946C8D84EB99E00E94E0
:10A18000F58BD3011296ED91FC916081718184E78A
:10A1900094E00E9409B4CE018F549F4F0E94143165
:10A1A00020E030E048EC52E40E9482D40E94EED6D7
:10A1B000C354DF4F688379838A839B83CD5BD04010
:10A1C000C354DF4FC880D980CD5BD04088E00E9467
:10A1D00039281B012C016DEC77E085E69AE00E949E
:10A1E000138ED3011296ED91FC916081718185E609
:10A1F0009AE00E946C8D69EC77E085E69AE00E9417
:10A20000138EC354DF4F68817981CD5BD04085E6E2
:10A210009AE00E94ECA664EC77E085E69AE00E9462
:10A22000138EB201A101662777272AE085E69AE01E
:10A230000E94A98B85E69AE00E94F58BB101A601E8
:10A24000C3010E946537AA24A394B12CD8CE689488
:10A2500080F891F8F8CFCA53DF4F08811981C65CA6
:10A26000D0400530110509F4E0CA40E054E0B301E4
:10A27000CE018F549F4F0E94AE3860E074E0D4CE80
:10A280000E945A31672B682B692B11F00C94FD4505
:10A29000912C812C0C942E462114310409F045C0D8
:10A2A0008081882311F40C944144CE0187549F4F40
:10A2B0000E9424371C01CD54DF4F8881C35BD040FE
:10A2C00081112EC0622DCE018F549F4F0E94D0303D
:10A2D000CF55DF4F2883C15AD040CE55DF4F38834A
:10A2E000C25AD040CD55DF4F4883C35AD040CC55D9
:10A2F000DF4F5883C45AD040CB55DF4F6883C55ACF
:10A30000D040CA55DF4F7883C65AD040C955DF4F79
:10A310008883C75AD040C855DF4F9883C85AD04069
:10A320002114310411F40C9441446FE07AE085E685
:10A330009AE00E94138EB60185E69AE00E94ECA690
:10A3400068E07AE085E69AE00E94138ED3011296C7
:10A35000ED91FC916081718185E69AE00E946C8D9F
:10A3600062E07AE085E69AE00E94138EC754DF4FE0
:10A3700068817981C95BD04085E69AE00E946C8D46
:10A3800060E07AE085E69AE00E94138ECE018F5459
:10A390009F4F0E948830C754DF4F88819981C95BE5
:10A3A000D040009711F40C948144FC0120812432A8
:10A3B00011F00C9481446CEE79E085E69AE00E94FD
:10A3C000138E85E69AE00E94F58B8CEFA82EBB24B5
:10A3D000BA9462CB2F923F924F925F926F927F928C
:10A3E0008F929F92AF92BF92CF92DF92EF92FF92A5
:10A3F0000F931F93CF93DF93CDB7DEB7CB57D10920
:10A400000FB6F894DEBF0FBECDBF3C01362EE296EC
:10A41000EFAEE297E396FFAEE397E4960FAFE497D3
:10A42000E5961FAFE597E6962FAFE697E7963FAF25
:10A43000E797E8964FAFE897E9965FAFE997EA9616
:10A44000CFAEEA97EB96DFAEEB97EC96AFAEEC971C
:10A450002B2C2401009709F47AC1FC0180858F70B0
:10A46000843009F45FC128F4882309F464C180E0D2
:10A470002FC0853009F446C08630C9F763E874E020
:10A48000C3010E9446A22C01009709F476C0912CCA
:10A49000812CB12CA12CD12CC12CE296EFACE297EF
:10A4A000E396FFACE397E4960FADE497E5961FAD16
:10A4B000E597E6962FADE697E7963FADE797E896E6
:10A4C0004FADE897E9965FADE997632D0E94EA5199
:10A4D000C558DF4F0FB6F894DEBF0FBECDBFDF917A
:10A4E000CF911F910F91FF90EF90DF90CF90BF9091
:10A4F000AF909F908F907F906F905F904F903F9024
:10A500002F90089580918E088F5F80938E086680CB
:10A5100077806114710459F14201EC96AFACEC976D
:10A52000B22CEA96CFACEA97EB96DFACEB97E296CB
:10A53000EFACE297E396FFACE397E4960FADE497B8
:10A54000E5961FADE597E6962FADE697E7963FAD0A
:10A55000E797E8964FADE897E9965FADE997632DE9
:10A56000C3010E94EA51F30162807380D2CF8091CF
:10A570008E08815080938E087ACF67E874E0C3011B
:10A580000E9446A27C016CE874E0C3010E9446A2CE
:10A590006C0161E974E0C3010E9446A2332039F0E6
:10A5A000F1E03F1609F49FC010E000E00CC065E93F
:10A5B00074E0C3010E9446A22C016AE974E0C30161
:10A5C0000E9446A28C014114510409F42301011593
:10A5D000110509F48301E114F10431F4EA96EFACBA
:10A5E000EA97EB96FFACEB97C114D10421F4EC96FB
:10A5F000CFACEC97D22C4114510409F4A5C0F20160
:10A6000080858F70843009F09FC061847284011549
:10A61000110509F4A8C0F80180858F70843009F015
:10A62000A2C04184528410E000E0E114F10409F476
:10A6300000C16114710409F4BDC063ED7CE185E6DD
:10A640009AE00E94138EF7016185728585E69AE093
:10A650000E946C8D6EEC7CE185E69AE00E94138E80
:10A66000B30185E69AE00E946C8D85E69AE00E942F
:10A67000F58BCE018F589F4F0E948830C114D104B2
:10A6800009F092C1F70180858F70843009F08AC18A
:10A6900040918C0850918D0861857285CE0101969C
:10A6A0000E94613ECE0101960E9458378823B1F086
:10A6B0000E948C296B01683C71050CF08FC06DE81D
:10A6C0007CE18EEB99E00E94138EB6018EEB99E04F
:10A6D0000E94ECA68EEB99E00E94F58BCE010196CC
:10A6E0000E94EB3E5FC16FE974E0C3010E9446A285
:10A6F0002C0164EA74E0C3010E9446A28C0141145B
:10A70000510409F056C165E974E0C3010E9446A2F4
:10A710002C010115110509F450CF892B09F05BCFED
:10A72000230159CF10E000E0512C412CD12CC12C39
:10A73000F12CE12C48CF10E000E0512C412CD12C21
:10A74000C12CF12CE12C47CF712C612C60CFEA9603
:10A75000EFACEA97EB96FFACEB97EC96CFACEC97AF
:10A76000DB2C712C612C00E020E033E040E150E074
:10A77000BE016F597F4FCE018F589F4F0E946A2EA6
:10A780002C01E4960FADE49710E00115110509F0D6
:10A790004CCFE2968FADE297811109C0E3968FAD61
:10A7A000E3978F7009F441CF02E010E03ECF01E063
:10A7B00010E03BCF64EC7CE185E69AE00E94138ECA
:10A7C000F7016185728585E69AE00E946C8D6FEBDA
:10A7D0007CE185E69AE00E94138E4BCF61147104F0
:10A7E00031F0B301CE0101960E9409A877CFA12CC8
:10A7F000CC24C394F12CE12CE2960FADE297E396C2
:10A800001FADE397E4962FADE497E5963FADE5974E
:10A81000E6964FADE697E7965FADE797E8966FADA2
:10A82000E897E9967FADE997CE0101960E948A43A9
:10A8300055CFC114D10409F4B5C04114510409F431
:10A84000B1C0F60180858F70843009F0A7C0818582
:10A85000928525961FAE1EAE259748EE53E060E028
:10A8600070E029964CAF5DAF6EAF7FAF29972FEBAD
:10A8700032E023963FAF2EAF23972F969FAF8EAF38
:10A880002F9761961FAE1EAE619763961FAE1EAEE8
:10A89000639765961FAE1EAE659767961FAE1EAE98
:10A8A000679769961FAF0EAF69976A961FAE6A9752
:10A8B00040E450E0BE016F5F7F4FCE018F5B9F4F42
:10A8C0000E94ECA321E030E02C0F3D1F820F931F6C
:10A8D000FC01108267EB7CE185E69AE00E94138E12
:10A8E000F6016185728585E69AE00E946C8D69EAC1
:10A8F00074E085E69AE00E946C8DBE016F5F7F4F29
:10A9000085E69AE00E946C8D62EB7CE185E69AE038
:10A910000E94138EB20185E69AE00E946C8D85E656
:10A920009AE00E94F58B0E9464A28823B9F180917D
:10A93000F808811133C06FE270E0CE0101960E94E9
:10A9400047DA892B51F4F6012185328543E050E046
:10A9500060E4CE0101960E9457286BEA7CE185E60F
:10A960009AE00E94138EBE016F5F7F4F85E69AE0EA
:10A970000E946C8D66EA7CE185E69AE00E94138E67
:10A98000B20185E69AE00E946C8D85E69AE00E940D
:10A99000F58BB201CE0101960E9401B1E114F104E0
:10A9A00009F070CE81E094CD4114510409F049CFF3
:10A9B00069CE892B09F00FCE00CE2F923F924F9295
:10A9C0005F926F927F928F929F92AF92BF92CF923F
:10A9D000DF92EF92FF920F931F93CF93DF93CDB748
:10A9E000DEB7A0970FB6F894DEBF0FBECDBF8C01C7
:10A9F000662E6A01DC018D919C911197892B09F4D7
:10AA000064C01596ED91FC91309709F45EC0808189
:10AA10008071BFEF6B135BC0D1F481E0A0960FB6DD
:10AA2000F894DEBF0FBECDBFDF91CF911F910F9184
:10AA3000FF90EF90DF90CF90BF90AF909F908F905E
:10AA40007F906F905F904F903F902F90089543308C
:10AA5000510519F3618062942FE0622265E377E08B
:10AA600085E69AE00E94138ED80113966C9185E6D4
:10AA70009AE00E94E5A663E377E085E69AE00E940B
:10AA8000138ED8011596ED91FC9161816F7085E66A
:10AA90009AE00E94E5A660E377E085E69AE00E94EE
:10AAA000138E662D85E69AE00E94E5A685E69AE07B
:10AAB0000E94F58BD8011596ED91FC9181818F70E4
:10AAC000681207C080818F7E808380E0A7CF8111CC
:10AAD000FCCF198E1A8E1B8E1C8E1D8E1E8E1F8E05
:10AAE00018A28A8D807F8A8FD8011596ED91FC91EE
:10AAF00081818F70861579F1B3E0CB16D10459F1BD
:10AB00006EE277E085E69AE00E94138EF801638199
:10AB100085E69AE00E94E5A66CE277E085E69AE099
:10AB20000E94138ED8011596ED91FC9161816F7092
:10AB300085E69AE00E94E5A669E277E085E69AE07C
:10AB40000E94138E662D85E69AE00E94E5A685E6B2
:10AB50009AE00E94F58BF80120813181FCE0F61526
:10AB600008F41DC1E62DF0E08827E654FA4A8F4F1D
:10AB70000C94F1D5C75504568C56A356AF568C5637
:10AB800065568C56B256BD567956C056CC56D8012D
:10AB90001596ED90FC90F70181818F70853009F456
:10ABA000FEC050F48230C1F06AEB74E0C9010E942B
:10ABB00046A22C01712C4BC08730D1F08A30A1F70E
:10ABC00063EB74E0C9010E9446A22C01D7017C907E
:10ABD00072FA772470F83BC06DEA74E0C9010E94F4
:10ABE00046A22C01D7017C9070FA772470F82FC010
:10ABF0006CEA74E0C9010E9446A22C01F701708042
:10AC000071FA772470F823C06FEB74E0C9010E94D9
:10AC100046A22C01D8011596ED91FC91808180FB14
:10AC2000772470F8982F9E7F80FF91609083411465
:10AC3000510469F461E0CE0149960E94F230298BFB
:10AC40003A8B4B8B5C8B6D8B7E8B8F8B988FF80147
:10AC5000E080F18067E874E0C7010E9446A21C0111
:10AC60006CE874E0C7010E9446A25C0161E974E0EF
:10AC7000C7010E9446A24C01A114B10481F4211421
:10AC8000310469F460E0CE0149960E94F2302983D4
:10AC90003A834B835C836D837E838F839887D8014F
:10ACA0001596ED91FC914114510409F07CC0898DF9
:10ACB000811179C0B62DBF706B2E8181807F682A8B
:10ACC000618280818F7E8083A8CE64EC74E0C901AC
:10ACD0000E9446A22C01D8011596ED91FC9180812D
:10ACE00081FB772470F8982F9D7F81FF926090837D
:10ACF000AECF6AEC74E0C9010E9446A22C01D801D3
:10AD00001596ED91FC91808182FB772470F8982F45
:10AD10009B7F82FF9460EBCF6AEB74E0C9010E94D5
:10AD200046A22C01892B09F045CF62E0CE0149965D
:10AD30000E94F23029873A874B875C876D877E8730
:10AD40008F87988B37CF60ED74E0C9010E9446A2CF
:10AD50002C01D8011596ED91FC91708045CF65EDE1
:10AD600074E0F3CF6BED74E0C9010E9446A22C01A0
:10AD7000D8011596ED91FC9142CF61EE74E0F4CFCD
:10AD800068EE74E0C9010E9446A22C01D801159614
:10AD9000ED91FC9170801CCF6EEE74E0F3CF712CBE
:10ADA000512C412C54CF83E0C816D104C1F0962D0C
:10ADB0009F70692E8181807F682A618280818F7E69
:10ADC00080836101E98CFA8C0B8D1C8D2D8D3E8D5D
:10ADD0004F8D58A1672DC2010E94EA511ECE81817C
:10ADE0008F70861509F419CE629490EF6922682A53
:10ADF00061828081806167CF7F928F929F92AF92B4
:10AE0000BF92CF92DF92EF92FF920F931F93CF9357
:10AE1000DF93EC014B01809159068F5F80935906B7
:10AE2000AB016FEFCE010E94DD548A8181FB0027C8
:10AE300000F91B819AEC910F903110F08730E1F509
:10AE400065EF74E0888199810E9446A27C01009799
:10AE500099F1FC0180858F70853071F58091A40A8D
:10AE600018131DC08091A50A8034C9F48091A60AE8
:10AE70009091A70A5C01990FCC08DD0860E0C7013A
:10AE80000E94BEA2FC0181859285A385B485A81687
:10AE9000B906CA06DB060CF05CC0712C37C01093F3
:10AEA000A40A80E48093A50A812F0E94CBAE9093E0
:10AEB000A70A8093A60ADECF212F30E0F901E55DD5
:10AEC000FE4D8491F901EB51FF4D1491F901E156CA
:10AED000FF4DF490FF2009F439C081110E94FAADB2
:10AEE000EF2DF0E0EE0FFF1FE15CF84FA591B4915C
:10AEF000EC911E2331E020E009F430E0832F922F03
:10AF0000772473940817190609F0C7CFF3E08F165A
:10AF1000910409F47EC0ED81FE81E181EF70E15082
:10AF2000EC3008F076C0F0E08827E656F84A8F4FFC
:10AF30000C94F1D5BA571559EC571D58155934587A
:10AF4000155964588C58A358DF58FE5890E080E09B
:10AF5000D7CF61E0C7010E94BEA277247394FC01A1
:10AF600081859285A385B4858A159B05AC05BD05B1
:10AF70006CF693CF0E9433B09B01AC014427552758
:10AF8000ED81FE816281738190E080E0AA24AA9421
:10AF9000BA2CC12CD12C18EEE12E13E0F12E00E0DA
:10AFA00010E00E9476278823A1F10881198160EDC5
:10AFB00074E0C8010E9446A2892B41F465ED74E05B
:10AFC000C8010E9446A2892B09F4F6C0A40163E0DF
:10AFD000CE010E94DD541DC00E9433B09B01AC0124
:10AFE00044275527ED81FE816281738190E080E0E6
:10AFF000AA24AA94BA2CC12CD12C1CE2E12EFF2445
:10B00000F39400E010E00E947627A40164E081112F
:10B0100079C0ED81FE81808183FB992790F9971596
:10B0200009F4BDC1982F907E09F41EC1982F907E1F
:10B0300090528F71892B808339C10E9433B09B015C
:10B04000AC0144275527ED81FE816281738190E038
:10B0500080E0AA24AA94BA2CC12CD12C16E9E12EA6
:10B06000F12C00E010E0CFCF0E9433B09B01AC0187
:10B0700044275527ED81FE816281738190E080E055
:10B08000AA24AA94BA2CC12CD12C18EEE12E13E0DC
:10B09000F12E00E010E00E947627882309F4B9CF52
:10B0A000088119816BED74E0C8010E9446A2892BCA
:10B0B00041F461EE74E0C8010E9446A2892B09F4B4
:10B0C0007BC0A40168E084CF0E9433B09B01AC0137
:10B0D00044275527ED81FE816281738190E080E0F5
:10B0E000AA24AA94BA2CC12CD12C1CE2E12EFF2454
:10B0F000F39400E010E00E947627A40169E0882321
:10B1000009F487CFCE010E94DD540E9433B0ED8157
:10B11000FE81738362837DCF0E9433B09B01AC01BB
:10B1200044275527ED81FE816281738190E080E0A4
:10B13000AA24AA94BA2CC12CD12C16E9E12EF12C08
:10B1400000E010E0D8CF0E9433B09B01AC0144274F
:10B150005527ED81FE816281738190E080E0AA2411
:10B16000AA94BA2CC12CD12C18EEE12E13E0F12EAA
:10B1700000E010E00E947627882309F44ACF088176
:10B18000198168EE74E0C8010E9446A2892B39F447
:10B190006EEE74E0C8010E9446A2892B19F0A4014A
:10B1A0006BE016CF6AEC74E0C8010E9446A2A401CD
:10B1B00066E0892B09F40CCFA4016DE009CF0E9451
:10B1C00033B09B01AC0144275527ED81FE8162819C
:10B1D000738190E080E0AA24AA94BA2CC12CD12CCF
:10B1E0001CE2E12EFF24F39400E010E00E94762799
:10B1F000882309F40ECFA4016CE084CF0E9433B001
:10B200009B01AC0144275527ED81FE81628173814A
:10B2100090E080E0AA24AA94BA2CC12CD12C16E983
:10B22000E12EF12C00E010E0E1CF0E9433B09B0151
:10B23000AC0144275527ED81FE816281738190E046
:10B2400080E0AA24AA94BA2CC12CD12C18E5E12EB6
:10B2500012E0F12E00E010E00E947627882309F426
:10B26000D8CEA40160E0B4CE0E9433B0ED81FE815F
:10B2700073836283E181EF70772009F44EC0E2307E
:10B2800041F148F4EE2309F445C0ED81FE8180814F
:10B2900070FA83F9D0CEE530E1F0A4016AE0E7303E
:10B2A000A1F7CE010E94DD548111EFCF80915906A4
:10B2B000815080935906DF91CF911F910F91FF909C
:10B2C000EF90DF90CF90BF90AF909F908F907F9046
:10B2D00008950881198164EC74E0C8010E9446A2B7
:10B2E000892BA9F46BED74E0C8010E9446A2892B5A
:10B2F00071F461EE74E0C8010E9446A2892B39F412
:10B300006CEA74E0C8010E9446A2892B19F0A401DE
:10B3100066E0C7CFA40161E0C4CFE150ED3008F092
:10B32000B4CFF0E08827E856F64A8F4F0C94F1D559
:10B33000A5594559A859A8594559AB594559CC590A
:10B34000CC59CC59CC59CC59A859A40162E0A9CF09
:10B35000A40165E0A6CF0881198164EC74E0C801FE
:10B360000E9446A2892BA9F46BED74E0C8010E94EB
:10B3700046A2892B71F461EE74E0C8010E9446A2D6
:10B38000892B39F46CEA74E0C8010E9446A2892B2B
:10B3900019F0A40167E085CFA40160E082CF8F712E
:10B3A000806449CE2F923F924F925F926F927F922C
:10B3B0008F929F92AF92BF92CF92DF92EF92FF92C5
:10B3C0000F931F93CF93DF93CDB7DEB763970FB67D
:10B3D000F894DEBF0FBECDBF4C013B0140E058E00A
:10B3E00060E070E00E945939672B682B692B09F4E3
:10B3F0005DC019821A821B821C821D821E821F82DE
:10B4000018868A81807F8A8340E053E0B401CE01B0
:10B4100001960E944B3CD4011B968D919C91892BE7
:10B4200009F444C040E058E060E070E0C4010E94CC
:10B430005C386DE67AE085E69AE00E94138EF401AE
:10B4400083859485DC01ED91FC910488F589E02DDC
:10B45000A12CCC24C394F12CE12C09811A812B81DD
:10B460003C814D815E816F81788519958F3F98076A
:10B47000E9F0D4011296ED91FC9160817181892BE4
:10B4800009F0B8C085E69AE00E946C8D6BE67AE020
:10B4900085E69AE00E94138E63E67AE085E69AE0FC
:10B4A0000E94138E85E69AE00E94F58B65E0F40118
:10B4B000828193810E94BEA26C01009709F4D0C0E2
:10B4C000DC011896BC91B98BBB2EB2942FE0B2224E
:10B4D000FC0121843284438454840E9433B0BB2015
:10B4E00009F4BEC0261A370A480A590A19861A866C
:10B4F0001B861C86B9861A85107F1A601A872D86CE
:10B500003E864F86588AF4E06F16710439F5E12CB7
:10B5100090E2F92E0B2D2B853C854D855E856F8540
:10B520007889C4010E941CB1C201B10128EE33E048
:10B5300040E050E00E9488D5BA01A9012AE030E03D
:10B5400085E69AE00E94E68C64E97AE085E69AE076
:10B550000E94138E85E69AE00E94F58B57FE80C00C
:10B5600022E022163104410420E852060CF478C08F
:10B570000E948C291B017B8B6A8BE12C80E2F82EC8
:10B5800009851A852B853C854D855E856F85788973
:10B59000C4010E941CB18A899B89883C9105BCF535
:10B5A0006BE77AE08EEB99E00E94138EB1018EEB8F
:10B5B00099E00E94ECA68EEB99E00E94F58B8FEF4C
:10B5C0009FEF63960FB6F894DEBF0FBECDBFDF913D
:10B5D000CF911F910F91FF90EF90DF90CF90BF9090
:10B5E000AF909F908F907F906F905F904F903F9023
:10B5F0002F90089585E69AE00E946C8D61E67AE0CE
:10B6000085E69AE00E94138E6DE57AE047CFD60179
:10B6100018968C9118978F7018968C9319821A82AD
:10B620001B821C821D821E821F8218868A81807F57
:10B630008A83B98289898F70AA24A394873009F0FC
:10B64000A12CCC24C394F12CE12C09811A812B81EB
:10B650003C814D815E816F817885C4010E948A435F
:10B66000B1E06B167104E9F440E053E060E070E093
:10B67000C4010E945939611571058105910589F050
:10B6800020918C0730918D072630310551F4C4018B
:10B690000E94C73C40E053E060E070E0C4010E94BB
:10B6A0005C38F40183859485009719F490E080E07C
:10B6B00088CFDC01ED91FC910284F385E02D199592
:10B6C000892BA1F3F40183859485DC01ED91FC9134
:10B6D0000480F581E02DB301199573CF2F923F922D
:10B6E0004F925F926F927F928F929F92AF92BF9292
:10B6F000CF92DF92EF92FF920F931F93CF93DF933E
:10B70000CDB7DEB7CB56D1090FB6F894DEBF0FBE6A
:10B71000CDBF3C0165EF74E0DC018D919C910E94EE
:10B7200046A28C01F30183819091A40A8913FCC085
:10B730009091A50A903409F0F7C08091A60A9091E3
:10B74000A70A2C010115110509F415C1D801189695
:10B750002C912F70253009F00EC1C8010E9449A715
:10B76000A2968FAFA297843008F4EAC063E0C801C4
:10B770000E94BEA2FC01818592854AE0E42EE89EEB
:10B780001001E99E300C112462E0C8010E94BEA2A3
:10B79000DC0119968D919C91E89E6001E99ED00C88
:10B7A0001124AC96DFAECEAEAC974601DD0CAA08F4
:10B7B000BB0861E0C8010E94BEA27C0160E0C80134
:10B7C0000E94BEA2DC0119962D913D914D915C9194
:10B7D0001C97A6962CAF3DAF4EAF5FAFA6979201D8
:10B7E000052C000C440B550BA6968CAD9DADAEAD53
:10B7F000BFADA697281B390B4A0B5B0BB101032C7D
:10B80000000C880B990B681979098A099B090E9419
:10B8100056D5D70119962D913D914D915C911C976C
:10B82000A696CCACDDACEEACFFACA6972C193D09CE
:10B830004E095F09A6962CAF3DAF4EAF5FAFA697FE
:10B840000E9488D5820E931EA41EB51EA2962FAD0F
:10B85000A297253009F486C081E090E0A101032C75
:10B86000000C660B770B481559056A057B0534F407
:10B870004A015B0144244A9423E0522EAC96CEAC9C
:10B88000DFACAC97A601DD0C660B770B8416950632
:10B89000A606B70624F44A015B01512C412CA2965E
:10B8A0002FADA297223009F079C06201550CEE0845
:10B8B000FF0860E0C8010E94BEA2FC01818592855C
:10B8C000A385B485812C912C5401C816D906EA06AB
:10B8D000FB060CF455C261E0C8010E94BEA2FC0147
:10B8E00081859285A385B4858C159D05AE05BF0520
:10B8F0000CF442C2C559DF4F0FB6F894DEBF0FBE3D
:10B90000CDBFDF91CF911F910F91FF90EF90DF900E
:10B91000CF90BF90AF909F908F907F906F905F90EF
:10B920004F903F902F9008958093A40A90E49093B5
:10B93000A50A0E94CBAE9093A70A8093A60A01CFD6
:10B940008AE0849D4001859D900C1124092C000CF7
:10B95000AA08BB08AC961FAE1EAEAC97212C38E2ED
:10B96000332E7ACF64E0C8010E94BEA2DC01199692
:10B970008D919C9173CF2AE0289F4001299F900CC4
:10B980001124092C000CAA08BB08AC961FAE1EAEF1
:10B99000AC97212C98E2392E81E090E0D3011596E6
:10B9A000ED91FC9122813381A201421B530B57FF81
:10B9B00003C0519541955109841795070CF4C4C0F3
:10B9C0008081982F929596959770963008F0BFC019
:10B9D0009F5F9295990F907E8F71892BB7C0F70169
:10B9E00061857285DB018C9181115EC2A114B10465
:10B9F00009F45BC0D50118968C9118978F7084302C
:10BA000009F053C040918C0850918D0819966D91A2
:10BA10007C91CE0101960E94613ECE0101960E946A
:10BA200058378823F1F18114910409F460C0E114BE
:10BA3000F10431F0F70180858F70843009F44CC037
:10BA400025961CAE1DAE1EAE1FAE259729961CAEC8
:10BA50001DAE1EAE1FAE299723961FAD2397107FF4
:10BA600023961FAF239781E022968FAF2297A12CB8
:10BA7000CC24C394F12CE12C01E024962FAD249723
:10BA800025963FAD259740E027965FAD27972896EE
:10BA90006FAD289729967FAD2997CE0101960E9418
:10BAA0008A43CE0101960E94EB3ED3011596ED919B
:10BAB000FC91938282821ECF0115110529F0F801B5
:10BAC00080858F70843019F06CEF74E0EDC1618572
:10BAD0007285FB01808188CF61857285FB01808141
:10BAE0008823F9F2CE0101960E9409A8DACF011548
:10BAF000110531F0D80118968C918F708430F1F0D7
:10BB000025961CAE1DAE1EAE1FAE259729961CAE07
:10BB10001DAE1EAE1FAE299723961FAD2397107F33
:10BB200023961FAF239782E022968FAF2297A12CF6
:10BB3000CC24C394F12CE12C02E09FCFF801618565
:10BB40007285DB018C91CCCF80818F718083808165
:10BB5000803AB8F0AC96EEADFFADAC976F01FF0F39
:10BB6000EE08FF08C814D904EA04FB0451F0C1012F
:10BB7000330CAA0BBB0B88159905AA05BB0509F068
:10BB8000B9CE2415350509F4B5CE6D961CAE1DAEA3
:10BB90001EAE1FAE6D976B968FAD6B97807F8660E4
:10BBA0006B968FAF6B976D968CAD9DADAEADBFAD07
:10BBB0006D9765968CAF9DAFAEAFBFAF6597AAE0AE
:10BBC000B0E0A50194010E94A7D569966CAF7DAF46
:10BBD0008EAF9FAF69976BE577E085E69AE00E94AC
:10BBE000138ED30113966C9185E69AE00E94E5A628
:10BBF00069E577E085E69AE00E94138ECE018F5AC0
:10BC00009F4F0E94883063E874E0F3018081918146
:10BC10000E9446A2912C812CB12CA12CD12CC12C9C
:10BC20006296EFAC62976396FFAC639764960FAD34
:10BC3000649765961FAD659766962FAD6697679674
:10BC40003FAD679768964FAD689769965FAD699706
:10BC50006FEF0E94EA51D3010D911C9167E874E0E7
:10BC6000C8010E9446A27C016CE874E0C8010E94F1
:10BC700046A28C010097E1F1FC0180858F70843031
:10BC8000B9F56185728540E450E0CE0101960E94CD
:10BC900080DA6FE270E0CE0101960E9447DA892BCC
:10BCA00059F4D80119962D913C9143E050E060E49D
:10BCB000CE0101960E94572800E020E032E040E1EA
:10BCC00050E0BE016F5B7F4FCE018F5A9F4F0E94A5
:10BCD0006A2E0E9464A2882359F08091F80881118D
:10BCE00007C0BE016F5B7F4FCE0101960E9401B17C
:10BCF000E114F104D1F1F70180858F708430A9F54A
:10BD000040918C0850918D0861857285CE01019615
:10BD10000E94613ECE0101960E945837882309F1A6
:10BD2000A12CCC24C394F12CE12C62960FAD629728
:10BD300063961FAD639764962FAD649765963FAD8C
:10BD4000659766964FAD669767965FAD67976896FD
:10BD50006FAD689769967FAD6997CE0101960E9495
:10BD60008A43CE0101960E94EB3ED3011596ED91D8
:10BD7000FC9153824282BECD812C912C540183943C
:10BD8000D3011596ED91FC9182819381092E000CCF
:10BD9000AA0BBB0B88159905AA05BB0509F4AACD0A
:10BDA000D3010D911C9167E874E0C8010E9446A27E
:10BDB0005C016CE874E0C8010E9446A26C0161E974
:10BDC00074E0C8010E9446A2A114B10431F4C11468
:10BDD000D10419F4892B09F468CE6FEB74E0C80123
:10BDE0000E9446A27C016AEB74E0C8010E9446A250
:10BDF0008C0161E677E085E69AE00E94138EF301FC
:10BE0000638185E69AE00E94E5A66FE577E085E626
:10BE10009AE00E94138EB40185E69AE00E94ECA697
:10BE200085E69AE00E94F58BC114D10409F4DECDB9
:10BE3000D60118968C9118978F70843009F0D6CD62
:10BE400019966D917C9140E450E0CE0101960E94DC
:10BE500080DA0E9464A2882309F4C8CD8091F80892
:10BE60008111C4CD6FE270E0CE0101960E9447DAE5
:10BE7000892B51F4F6012185328543E050E060E4DE
:10BE8000CE0101960E9457288114910409F414CE22
:10BE9000E114F10439F0D70118968C918F70843039
:10BEA00009F49DCD69EF74E0CE0101960E9401B1C5
:10BEB0009DCD4F925F926F927F928F929F92AF92A1
:10BEC000BF92CF92DF92EF92FF920F931F93CF9387
:10BED000DF93CDB7DEB7CA54D1090FB6F894DEBFF1
:10BEE0000FBECDBFDC0115962D913C911697232BEB
:10BEF00009F470C14C01FC0182816230710544F08B
:10BF0000643071050CF44AC06430710509F462C0F4
:10BF1000883009F46DC0803109F052C00E9433B0FE
:10BF20002B013C01C4010E943C16A12CB12C6501DF
:10BF300010E3E12E15E7F12E00E010E0A3019201DD
:10BF40000E9476278823E1F16CE874E0D4018D919A
:10BF50009C910E9446A28C01009709F430C1FC011B
:10BF600080858F70843009F02AC10E9433B02AE0A6
:10BF7000AE014F5F5F4F0E94CBCE0E9464A2882328
:10BF800009F41DC18091F808811119C1BE016F5FCC
:10BF90007F4FD80119968D919C910FC1803499F0F3
:10BFA00040F4843068F4873059F0C4010E94FC5694
:10BFB00007C0823441F020F090E8980F943098F355
:10BFC00090E080E009C163307105D1F3C4010E94A3
:10BFD0006E5BF6CF8730A1F7CD010E946E5BD40176
:10BFE00015968D919C91892B59F364E070E0DDCF1B
:10BFF0000E9433B02B013C01C4010E943C16A12CCD
:10C00000B12C650118E9E12E1AE3F12E00E010E0F1
:10C01000A30192010E947627882391F2D4011596FC
:10C02000ED91FC911697818113961C91811153C05B
:10C030001630F0F58CE0EEE1F2E0DE0111960190B1
:10C040000D928A95E1F7E12FF0E0EE0FFF1F21E05E
:10C0500030E02C0F3D1FE20FF31F60E080810E9453
:10C060008FAE6CE876E183E01330C9F070F464E9D8
:10C0700076E181E0113099F060E976E182E01230FA
:10C0800071F068E976E180E00AC068E876E184E072
:10C09000143029F064E876E185E0153091F70E94CC
:10C0A000F4A6D4011596ED91FC9181E0818388CFAF
:10C0B00064E277E085E69AE00E94138EF4016381E2
:10C0C00085E69AE00E94E5A667EF76E085E69AE0CD
:10C0D0000E94138E75CF24E0129FF0011124ED5DB4
:10C0E000F94FC080D180E280F38063EF76E085E68F
:10C0F0009AE00E94138ED40113966C9185E69AE023
:10C100000E94E5A66FED76E085E69AE00E94138E28
:10C110002AE030E0B701A60185E69AE00E94E68CAD
:10C120006CE874E0F401808191810E9446A28C0148
:10C13000009709F44CC0DC0118968C9118978F7009
:10C14000843009F044C019966D917C9140E450E030
:10C15000CE0101960E9480DA6FE270E0CE01019676
:10C160000E9447DA892B51F4F8012185328543E09A
:10C1700050E060E4CE0101960E945728FF92EF92B2
:10C18000DF92CF9289E294E09F938F938E010F5BB1
:10C190001F4F1F930F930E94D7DA0E9464A20FB61D
:10C1A000F894DEBF0FBECDBF882349F08091F80818
:10C1B000811105C0B801CE0101960E9409B40E9408
:10C1C00033B0AB01BC01C4010E941516F9CE60ED7D
:10C1D00076E07CCF8FEF9FEFC65BDF4F0FB6F89412
:10C1E000DEBF0FBECDBFDF91CF911F910F91FF90AA
:10C1F000EF90DF90CF90BF90AF909F908F907F9007
:10C200006F905F904F900895EF92FF920F931F935E
:10C21000CF93DF93EC018B011E821D821A821B8259
:10C220001C82E880F980E114F10409F476C0809161
:10C230008F0890919008892B09F46FC0672B09F43F
:10C240008701F80180858F708630D9F460E075E051
:10C25000C8010E9446A2009719F0FC0181858A83DB
:10C2600066E875E0C8010E9446A2FC01892B09F42A
:10C2700076C080858F70823009F46EC0853009F4F5
:10C2800053C062E075E0C7010E9446A2009709F022
:10C2900041C06BEC76E085E69AE00E94138E6B81DC
:10C2A00085E69AE00E94E5A669EC76E085E69AE0EC
:10C2B0000E94138E6A8185E69AE00E94E5A685E6D3
:10C2C0009AE00E94F58BE880F9800E944C928C01E4
:10C2D000892BC1F082E0F8018087118612861386CF
:10C2E000148680819181009711F00E94A48F82E0D2
:10C2F00095E00E94D38FF80191838083B801C70134
:10C300000E94C4A662E075E0888199810E9446A2DD
:10C31000009719F009969E838D83DF91CF911F912D
:10C320000F91FF90EF9008950680F781E02D3097F0
:10C3300009F4A7CF80858F70823009F0A2CF818564
:10C340008B830680F781E02D309709F49ACF8085A2
:10C350008F70823009F095CF81858B8392CFF80161
:10C36000808191810E94BBCDF8CF8F929F92AF9236
:10C37000BF92CF92DF92EF92FF920F931F93CF93D2
:10C38000DF93CDB7DEB72E970FB6F894DEBF0FBEA2
:10C39000CDBF2091860830918708232B09F4BAC0BD
:10C3A00020918B072111B6C04C0180918B078F5FC4
:10C3B00080938B0780918E088F5F80938E080E94F8
:10C3C00033B09B01AC016091CC067091CD06809199
:10C3D000CE069091CF06A12CB12C65011BE0E12E79
:10C3E000F12C00E010E00E947627882309F488C031
:10C3F000F12C83E088169104A1F00E9433B09B01D8
:10C40000AC016091C8067091C9068091CA069091EE
:10C41000CB0614E6E12EF12C00E010E00E94762716
:10C42000F82EE0918608F0918708068117810115A2
:10C43000110509F447C0F80180858F708630F1F549
:10C440001987088770E060E0CE0108960E940461B9
:10C45000B401CE0108960E94595FFF2031F064E0DC
:10C4600070E0CE0108960E94595F63E874E0C8014D
:10C470000E9446A2009711F1FC0120852F70253003
:10C48000E9F4C680D780C114D104C1F0DA82C98230
:10C49000B801CE0101960E940461B401CE0101965B
:10C4A0000E94595FFF2031F064E070E0CE010196F8
:10C4B0000E94595FF601C280D380E5CFF801028166
:10C4C0001381B5CFF3E08F16910451F00E9433B081
:10C4D0006093CC067093CD068093CE069093CF06E2
:10C4E000FF2051F00E9433B06093C8067093C906D4
:10C4F0008093CA069093CB061092A40A1092A50AC4
:10C5000080918E08815080938E0880918B07815096
:10C5100080938B072E960FB6F894DEBF0FBECDBF6B
:10C52000DF91CF911F910F91FF90EF90DF90CF900F
:10C53000BF90AF909F908F9008958091F8088F5F83
:10C540008093F808A89583E090E00E94B5610E946E
:10C550005E8F8091F80881508093F8080895CF92FB
:10C56000DF92EF92FF92CF93DF93EC018C858830BE
:10C5700068F40E9487970E9433B06B017C018C8520
:10C580000E947E9B811109C088E08C87DF91CF914A
:10C59000FF90EF90DF90CF9008950E949D6261E040
:10C5A00070E080E090E00E9400B00E9433B0AB01E8
:10C5B000BC014C195D096E097F098D859E85B0E02F
:10C5C000A0E0481759076A077B07C8F28C850E94CC
:10C5D0009597DACFCF92DF92EF92FF921F93CF938E
:10C5E000DF93EC017B016A018C85883048F40E945E
:10C5F0007E9B882319F08C850E94879788E08C8722
:10C60000F70182819381A481B5810097A105B105CD
:10C6100051F490E080E0DF91CF911F91FF90EF9077
:10C62000DF90CF9008958F3F9F4FAF4FBF4F89F35B
:10C6300070E060E081E20E948D9B182F8C8788302B
:10C6400040F780E591E00E94D1AAA7014E5F5F4FBD
:10C6500024E030E06CE070E0812F0E94DF94B601AE
:10C66000812F0E94AF9564E070E0812F0E94779740
:10C670000E9433B06B017C018C850E947E9B8731C8
:10C6800021F18C3111F1882321F20E9433B0AB01EA
:10C69000BC014C195D096E097F098D859E85B0E04E
:10C6A000A0E084179507A607B70748F00E949D628F
:10C6B00061E070E080E090E00E9400B0DDCF8C850A
:10C6C0000E94959788E08C87A4CF81E090E0A3CF6B
:10C6D000A89582E090E00C94B5618F929F92BF92F2
:10C6E000CF92DF92EF92FF920F931F93CF93DF933E
:10C6F000CDB7DEB7AE970FB6F894DEBF0FBECDBF95
:10C7000080918F0890919008892B09F4B7C480918B
:10C710008E088111B3C480918E088F5F80938E083C
:10C720006CEE75E184EB99E00E94138E84EB99E046
:10C730000E94F58B00918F081091900865E075E0DC
:10C74000C8010E9446A290938D0880938C086BE0EC
:10C7500075E0C8010E9446A29093850880938408E2
:10C7600060E375E0C8010E9446A290938708809319
:10C77000860862E175E0C8010E9446A29093830892
:10C7800080938208009739F1DC011696ED91FC91B7
:10C79000309709F120852F702530E9F468ED75E1B7
:10C7A00084EB99E00E94138E809182089091830817
:10C7B0000E9449A780937D08682F84EB99E00E942E
:10C7C000E5A684EB99E00E94F58BE0918208F09158
:10C7D00083088681978190938108809380080E94C6
:10C7E000E12167E175E080918F08909190080E94A7
:10C7F00046A290937C0880937B08892BA1F08091BE
:10C800008E07811110C08091890790918A07892B2A
:10C8100009F47DC081E080938E0768EC75E184EBBC
:10C8200099E00E94138E10928B0810928A08E09172
:10C830008C08F0918D08309709F4F4C2E680F780F7
:10C8400000918C0810918D080115110509F4E3C2BF
:10C85000E114F10409F4DFC2F70180858F7085309F
:10C8600099F7C7010E9449A7823070F3A801B70168
:10C87000CE0101960E944640CE0101960E94583793
:10C880008823E1F18C859D85009709F43DC2DC0188
:10C89000ED91FC910284F385E02D1995892B49F0E7
:10C8A0008C859D85DC01ED91FC910084F185E02D66
:10C8B00019958C859D85DC01ED91FC910680F781B1
:10C8C000E02D1995892BD1F0CE0101960E94AD3A49
:10C8D000882341F040E051E060E070E0CE01019635
:10C8E0000E9485388F819885892B41F040E052E085
:10C8F00060E070E0CE0101960E948538D701129663
:10C90000ED90FC90CE0101960E94EB3E99CF6AE833
:10C9100075E185E69AE00E94138E85E69AE00E9412
:10C92000F58B8FE090E00E94EECB8C0188E1F8015E
:10C93000818312821082168615860E9412AB109394
:10C940008A0700938907012B69F46BE775E18EEB89
:10C9500099E00E94138E8EEB99E00E94F58B109265
:10C960008E0761CF0E9412AB8091890790918A0750
:10C970000E94F418882309F493C06CE575E184EBF8
:10C9800099E00E94378E8091890790918A070E94D2
:10C990009024E0918907F0918A0781E0808380915B
:10C9A000890790918A070E949E2468E475E18111AD
:10C9B00002C063E375E185E69AE00E94378E8091BC
:10C9C0007B0890917C08892B51F280918707909188
:10C9D0008807892B09F0EAC083E190E00E94EECB42
:10C9E0008C018091890790918A072CE331E8D80166
:10C9F00052963C932E93519716969C938E9315972F
:10CA000014961C9214971C9289E011968C9311979E
:10CA100081E012968C93129713968C93109388074B
:10CA2000009387070E9433B06B017C01B0E1CB0E0D
:10CA3000B7E2DB1EE11CF11CD8011596ED91FC91CB
:10CA400016978FEF838714861382148215821682BD
:10CA5000178210861186128614961C92BB24B394FA
:10CA6000BE01605E7F4FF801858196810E94782526
:10CA700018160CF096C00E9433B06C157D058E051B
:10CA80009F0508F08EC0DE01909698E080E09150FE
:10CA900019F1ED91E827F0E0E85DF24E8491F7CFCF
:10CAA0000E94D8278091890790918A070E94F418E4
:10CAB000882359F066E175E184EB99E00E94138EBA
:10CAC00084EB99E00E94F58B7ACF6AEF74E18EEBEC
:10CAD00099E00E94378E43CF9FA19813C1CFD80110
:10CAE0008C91811138C015968D919C910E949E2445
:10CAF000BE01605E7F4FF801858196810E9471249E
:10CB000040E064EBD80115968D919C910E944B24D6
:10CB1000F80185809680C4010E94CF23C4010E9441
:10CB2000611367E885E299E00E94EC1360E885E212
:10CB300099E00E94EC130E94FDAFC4010E94CF2334
:10CB4000982ED80115968D919C910E949E2495FC5B
:10CB500002C0F801B082AE014F5F5F4FBE01605E60
:10CB60007F4FC8010E94DF24D80111969C9088A1B4
:10CB7000803109F495C2BE01605E7F4FC8010E94FA
:10CB80004E25891508F0B4C0F8018181D8011196AD
:10CB90008C93119714968C9114978F5F14968C93A5
:10CBA0005FCFE0918707F09188071282E0917B08C0
:10CBB000F0917C08E680F7809FE7D92E80917B0872
:10CBC00090917C08892B09F425CEE114F10409F435
:10CBD00021CEBE01605E7F4FF701808191810E946E
:10CBE0000E2B882309F416CE63EE74E185E69AE0F5
:10CBF0000E94138ED7016D917C9185E69AE00E9488
:10CC00006C8D85E69AE00E94F58B00918707109164
:10CC10008807AE014F5F5F4FBE01605E7F4FC80166
:10CC20000E943425882309F45EC088A1803109F46C
:10CC30005AC0DD82F801858196810E949E24BE0142
:10CC4000605E7F4FD80115968D919C910E94712452
:10CC500040E06EE4F801858196810E944B2440E01B
:10CC60006B81D80115968D919C910E944B2440E0D8
:10CC70006C81F801858196810E944B2488A18031C6
:10CC800041F040E06D81D80115968D919C910E94F4
:10CC90004B24F801858196810E949E24BE01605E2E
:10CCA0007F4FD80115968D919C910E947124F801B7
:10CCB000408168E4858196810E944B2464E170E0A4
:10CCC00080E090E00E9400B0D8018C91882331F080
:10CCD0006AE070E080E090E00E9400B0F801858199
:10CCE00096810E949E24D7011296ED90FC9066CF0B
:10CCF00088A1803111F48CE049CFBE01605E7F4F86
:10CD0000C8010E944E2542CFCE0101960E9459A72C
:10CD10008C01912C812C97FF06C01195019511096A
:10CD200088248394912CCE0101960E94AD3AC82E9E
:10CD3000D12C8B85853091F0863009F0DFCDB02E77
:10CD400061E0802F0E948FAE61E0892809F441C024
:10CD5000CA94CD2809F041C060E03FC0CD2829F435
:10CD600062E0CE0101960E94111E40E051E060E0B9
:10CD700070E0CE0101960E9485388F819885892BBD
:10CD800041F040E052E060E070E0CE0101960E9488
:10CD9000853861E0802F0E948FAE60E0802F0E9476
:10CDA00061AE60EC75E185E69AE00E94138EB801F1
:10CDB00085E69AE00E94ECA66BEB75E185E69AE0C9
:10CDC0000E94138E69EB75E185E69AE00E94138E4E
:10CDD00095CDCA94CD2809F0BFCFC62ED12C8B2D6E
:10CDE0000E9461AE64EB75E185E69AE00E94138EC5
:10CDF000B80185E69AE00E94ECA662EB75E185E653
:10CE00009AE00E94138EB60185E69AE00E94ECA695
:10CE100060EB75E1D9CFF8018681978190938B08FB
:10CE200080938A0885E69AE00E94F58B6FEC74E1A6
:10CE300084EB99E00E94138E84EB99E00E94F58BBD
:10CE4000E0918608F0918708309709F48DC08091B1
:10CE50008E088F5F80938E0806811781011511055A
:10CE600009F47DC0D80118968C918F70863009F036
:10CE70006CC019A708A770E060E0CE0188960E94F8
:10CE800004618DA59EA5892B09F45FC080918F0850
:10CE900090919008892B09F458C0E8A4F9A4E114F2
:10CEA000F104C1F1F70180858F70863099F5F9A200
:10CEB000E8A270E060E0CE0180960E940461EDA1DE
:10CEC000FEA1108211821282138263E874E0C7010E
:10CED0000E9446A20097F1F0DC0118962C91189759
:10CEE0002F702530B9F41696CD90DC90C114D10482
:10CEF00089F0DA82C982B701CE0101960E940461ED
:10CF0000EE81FF811082118212821382F601C280AB
:10CF1000D380ECCFEDA5FEA5108211821282138280
:10CF20008AA5843068F462E0823008F060E08BA566
:10CF30000E948FAEEDA5FEA58181807F818305C013
:10CF4000803441F060E0823431F0D80112960D91C6
:10CF50001C9184CF62E08BA50E948FAEF6CF8091AA
:10CF60008E08815080938E0862EC74E184EB99E026
:10CF70000E94138E6AEB74E184EB99E00E94138E99
:10CF800081E020918C0830918D08232B09F480E0FA
:10CF90000E94351961EB74E184EB99E00E94138ED5
:10CFA00081E02091860830918708232B09F480E0E6
:10CFB0000E9435196AEA74E184EB99E00E94138EAD
:10CFC00081E02091800830918108232B09F480E0D2
:10CFD0000E94351961EA74E184EB99E00E94138E96
:10CFE00081E020917B0830917C08232B09F480E0BC
:10CFF0000E94351968E974E184EB99E00E94138E70
:10D00000809189080E94351984EB99E00E94F58B84
:10D0100063E974E184EB99E00E94138E0E948C29ED
:10D02000AB01BC0184EB99E00E94E2A684EB99E09D
:10D030000E94F58B81E08093880881E899E00E9446
:10D04000D217882351F081E899E00E94AF6284E012
:10D0500090E090938D0780938C0780918C0790913E
:10D060008D07079731F484E090E090938D078093CB
:10D070008C0780918E08815080938E08AE960FB6F3
:10D08000F894DEBF0FBECDBFDF91CF911F910F91FE
:10D09000FF90EF90DF90CF90BF909F908F9008957A
:10D0A000BCE0B91508F470CD26CEAF92BF92DF92E6
:10D0B000EF92FF920F931F93CF93DF9300D000D096
:10D0C000CDB7DEB78C017B01D42EFB018481958125
:10D0D000892BF9F0A080B1806FE370E0C5010E9458
:10D0E00047DA0097B1F09C012A193B0937FD11C0BE
:10D0F00050E040E0B701CE0101960E94A689BE0132
:10D100006F5F7F4FC7010E94F487CE0101960E9496
:10D1100056896AE175E0C7010E94AF87882321F133
:10D12000F801128A118A80E090E19587848784E86B
:10D1300090E0948B838B81E0868780E090E2908BF7
:10D140008787D58A81E090E026960FB6F894DEBFF7
:10D150000FBECDBFDF91CF911F910F91FF90EF9048
:10D16000DF90BF90AF90089567E275E0C7010E941D
:10D17000AF87882369F0F801128A118A148A138A0A
:10D1800084E890E095878487168680E090E3D7CF87
:10D1900090E080E0D9CFEF92FF920F931F93CF934F
:10D1A000DF9300D01F92CDB7DEB78C017B01FB016E
:10D1B00084858830A8F088EE93E0F801918380831D
:10D1C0001282138214821582C8010F900F900F9063
:10D1D0000F90DF91CF911F910F91FF90EF900895E5
:10D1E00080E591E00E94D1AA24E030E0AE014F5FDB
:10D1F0005F4F6CE070E0F70184850E941821BE014A
:10D200006F5F7F4FC8010E94538EDECFEF92FF9277
:10D210000F931F93CF93DF9300D000D0CDB7DEB72D
:10D220008091900990919109892B09F46CC087E74E
:10D230000E9492A38091900990919109DC01ED9157
:10D24000FC910088F189E02D70E060E0199510E014
:10D2500000E08091900990919109DC01ED91FC91A1
:10D2600011971C962D913C910217130740F40190E1
:10D27000F081E02D60E019950F5F1F4FEACF008825
:10D28000F189E02D70E060E0199505EF12E089EF7B
:10D29000E82E82E0F82E8091900990919109F80192
:10D2A00061918F01DC01ED91FC910190F081E02D05
:10D2B0001995E016F10679F78091900990919109FE
:10D2C000DC01ED91FC910488F589E02D19956AE85F
:10D2D00075E0CE0101960E949589CE0101960E94CB
:10D2E000FDB8CE0101960E94568987E090E00E9429
:10D2F000AEA687E090E00E94B8A669EF77E184EBE4
:10D3000099E00E94138E1092B0091092AF0980E04C
:10D3100090E19093AB098093AA0984E890E0909300
:10D32000B2098093B10981E08093AC0980E090E27A
:10D330009093AE098093AD0982E78093B3098EE99B
:10D3400099E00E94D8168EE999E00E94701988EC45
:10D3500090E026960FB6F894DEBF0FBECDBFDF91EA
:10D36000CF911F910F91FF90EF900895CF93DF938E
:10D37000CDB7DEB72E970FB6F894DEBF0FBECDBF88
:10D3800080918E08811119C180918E088F5F8093E2
:10D390008E0867E476E184EB99E00E94138E84EBBB
:10D3A00099E00E94F58B1092B0091092AF0980E0CD
:10D3B00090E19093AB098093AA0984E890E0909360
:10D3C000B2098093B10981E08093AC0980E090E2DA
:10D3D0009093AE098093AD0982E78093B3098EE9FB
:10D3E00099E00E9427208B37910509F0BDC069E3C1
:10D3F00076E185E69AE00E94138E85E69AE00E9427
:10D40000F58B1C821B8289EA92E09A8389838EE9DC
:10D4100099E09E838D838FEF9FEF98878F830E9483
:10D42000E3B9CE0101960E9429AB909390088093B6
:10D430008F088EE999E00E94701980918F08909171
:10D440009008892B01F56DE276E18EEB99E00E9460
:10D45000138E8EEB99E00E94F58B6AE875E0CE01A1
:10D4600009960E949589CE0109960E94FDB8CE01C9
:10D4700009960E94568980918E08815080938E086B
:10D4800090E080E019C06AE176E184EB99E00E94C7
:10D49000138E84EB99E00E94F58B80918E08815069
:10D4A00080938E080E946D638091900990919109FC
:10D4B000892B59F481E090E02E960FB6F894DEBFE8
:10D4C0000FBECDBFDF91CF9108950E94A7A38823FF
:10D4D00089F382E70E9492A380919009909191092B
:10D4E000DC01ED91FC910088F189E02D60E670E0AF
:10D4F0001995609190097091910940E0CE010996CB
:10D500000E94728BBE01675F7F4F82E999E00E94A3
:10D51000F487CE0109960E945689809190099091D6
:10D520009109DC01ED91FC910488F589E02D1995B4
:10D530006CEF75E185E69AE00E94138E62E979E06E
:10D54000CE0109960E948C89BE01675F7F4F85E6F8
:10D550009AE00E94058E85E69AE00E94F58BCE0146
:10D5600009960E945689A6CF8EE999E00E94AE16D0
:10D57000892BA1F08EE999E00E94D8166AE875E03F
:10D58000CE0101960E949589CE0101960E94FDB8B8
:10D59000CE0101960E9456890E946CB98EE999E0ED
:10D5A0000E94701969E076E184EB99E00E94138E85
:10D5B00084EB99E00E94F58B5ECF8FEF9FEF7CCFDD
:10D5C000FF920F931F93CF93DF9300D000D0CDB77E
:10D5D000DEB78C01BC01CE0101960E948C89BE0190
:10D5E0006F5F7F4F85E69AE00E94058E85E69AE0A0
:10D5F0000E94F58BCE0101960E94568964E278E183
:10D60000CE0101960E945E89BE016F5F7F4FC80107
:10D610000E949487F82ECE0101960E945689FF2021
:10D6200069F0B801CE0101960E948C89CE01019665
:10D630000E94FDB8CE0101960E94568926960FB62B
:10D64000F894DEBF0FBECDBFDF91CF911F910F9138
:10D65000FF9008954F925F926F927F928F929F9268
:10D66000AF92BF92CF92DF92EF92FF920F931F93F0
:10D67000CF93DF93CDB7DEB7C859D1090FB6F89471
:10D68000DEBF0FBECDBF8E010F5B1F4FD8011D92B5
:10D690001C92FE01ED5BFF4F8EE1DF011D928A952A
:10D6A000E9F78091900990919109892B09F4CEC1F5
:10D6B0000E94A7A3882309F4C9C182E70E9492A30C
:10D6C0008091900990919109DC01ED91FC91008885
:10D6D000F189E02D60E270E019954FE150E0B8016A
:10D6E00080919009909191090E94ECA37C01809116
:10D6F000900990919109DC01ED91FC910488F589E4
:10D70000E02D1995E114F10409F4A0C1F801EE0D22
:10D71000FF1D108280919D091F928F9380919C091B
:10D720001F928F9380919B091F928F9380919A09EA
:10D730001F928F93809199091F928F9380919809DE
:10D740001F928F9383E395E09F938F931F9280E4C2
:10D750008F93FE0131966F01FF93EF930E949ADA47
:10D7600063E179E184EB99E00E94138EB80184EBC8
:10D7700099E00E946C8DB60184EB99E00E946C8D5B
:10D7800084EB99E00E94F58B7E01F1E6EF0EF11C2F
:10D79000D70113961C921E92129788EE93E0A0E098
:10D7A000B0E0F70184839583A683B78388E08487FC
:10D7B00088EE93E09687858786E693E09183808361
:10D7C000108A1786128B018B148A138A80E590E0E9
:10D7D000968B858B118E6BE278E185E69AE00E944C
:10D7E000138E62E979E0CE0185589F4F0E948C89A3
:10D7F000BE0165587F4F85E69AE00E94058E85E65A
:10D800009AE00E94F58BCE0185589F4F0E94568961
:10D8100062E675E0CE0183579F4F0E94958962E6CC
:10D8200075E0CE0185589F4F0E949589BE016558CD
:10D830007F4FCE018B579F4F0E948C8962E979E020
:10D84000CE018B579F4F0E94F288BE0163577F4FD6
:10D850000E94F288BC01CE018D569F4F0E948C8998
:10D86000CE018B579F4F0E945689CE0185589F4FFE
:10D870000E945689CE0183579F4F0E94568984E6A5
:10D8800095E0CB57DF4F99838883C558D040C75761
:10D89000DF4F19821882C958D040C557DF4F19820F
:10D8A0001882CB58D040CD56DF4F88819981C3591B
:10D8B000D040C957DF4F99838883C758D0406DE067
:10D8C00079E185E69AE00E94138E0E948C29AB01D3
:10D8D000BC0185E69AE00E94E2A685E69AE00E94F5
:10D8E000F58B64E670E080E090E00E9400B080EE8E
:10D8F0009AE6D70150969C938E931F976AE575E838
:10D900008FE792E90E9431CF8C010FB6F894DEBF09
:10D910000FBECDBF892B09F4F4C083E090E00E94D4
:10D92000EECBD8011D969C938E931C97FC01F1823F
:10D93000E0821282C7010E94D217882319F0C70122
:10D940000E94AF62D70153966D917C915497559682
:10D95000AD90BC906115710509F48FC0CE0185585A
:10D960009F4F0E94538EA501BE0165587F4FC7018E
:10D970000E94EA62181619060CF0C0C0D701519631
:10D98000BC9051975296AC90DF92CF9286E898E186
:10D990009F938F931F930F930E94B8CFDF92CF92E4
:10D9A00081E898E19F938F931F930F930E94B8CFC4
:10D9B000D8011C96ED91FC9181E08283DF92CF9299
:10D9C0008EE798E19F938F931F930F930E94B8CF98
:10D9D000D8011C96ED91FC911282AF92BF9288E41F
:10D9E00098E19F938F931F930F930E94B8CF0FB628
:10D9F000F894DEBF0FBECDBFB12C8FE3C82E88E1F7
:10DA0000D82E8B2D94E08902F0011124A5E8B0E016
:10DA1000AC0FBD1FEA0FFB1F808191810097A9F118
:10DA20002281338121153105C9F33F932F939F93B1
:10DA30008F93DF92CF921F930F930E94B8CFB3942E
:10DA40000FB6F894DEBF0FBECDBFDBCF40E250E093
:10DA500065E479E1C8010E945ECE67E279E184EB7A
:10DA600099E00E94138EB80184EB99E00E946C8DBE
:10DA700084EB99E00E94F58B4DCEF70161897289A4
:10DA8000A501C7010E94581875CF83E898E19F93BC
:10DA90008F931F930F930E94B8CFD70158961C9273
:10DAA0001E925797D8011C96ED91FC91C080D180B1
:10DAB0000F900F900F900F9043E3A42EB12CD6013E
:10DAC000ED91FC910084F185E02DC60119954197F7
:10DAD0005CF4B1E0AB1AB10839F064E170E080E0C9
:10DAE00090E00E9400B0EBCFD601ED91FC91008454
:10DAF000F185E02DC6011995419734F4C8010E94C3
:10DB0000589210E000E05AC06AE875E0CE018357F1
:10DB10009F4F0E949589912CA12CD601ED91FC91EB
:10DB20000688F789E02DC60119958823E1F1BDE04B
:10DB3000AB1201C0A92CD601ED91FC910688F789A2
:10DB4000E02DC60119958111B9C0D601ED91FC9166
:10DB50000084F185E02DC6011995892B09F4C0C018
:10DB6000D601ED91FC910284F385E02DC601199553
:10DB7000B82EBAE08B1709F4B5C0EDE08E1709F4A2
:10DB8000B1C0FFEF8F1709F4ABC0682FCE018357E8
:10DB90009F4F0E9481889A2CAB2CBFCFBAE0BB125A
:10DBA000FACFAB12F8CFCC24C394D12CCE0183573B
:10DBB0009F4F0E945689CD2809F4A3CFD7015796CD
:10DBC000ED90FC906FEF78E185E69AE00E94138E6D
:10DBD000B70185E69AE00E94ECA685E69AE00E94ED
:10DBE000F58B64E670E080E090E00E9400B00115E3
:10DBF000110509F463C1B8ECEB16F10409F03CC15E
:10DC000063EF78E184EB99E00E94138E64EF71E09A
:10DC100080E090E00E9400B0EF961FAE1EAEEF973E
:10DC2000C158DF4F19821882CF57D0408FEF9FEF36
:10DC3000CF57DF4F99838883C158D04083E992E062
:10DC4000ED969FAF8EAFED97CD57DF4F19830883C9
:10DC5000C358D040F8940E94E3B98111CEC067EE5A
:10DC600078E18EEB99E00E94138E8EEB99E00E9492
:10DC7000F58BC8010E94589224EFE22EFF24F39402
:10DC8000CE018D569F4F0E945689C701C856DF4F5F
:10DC90000FB6F894DEBF0FBECDBFDF91CF911F91BD
:10DCA0000F91FF90EF90DF90CF90BF90AF909F903B
:10DCB0008F907F906F905F904F900895D601ED9177
:10DCC000FC910084F185E02DC6011995892B09F09E
:10DCD0003CCF64E670E080E090E00E9400B02BCF83
:10DCE000BB24BA9462E775E088EC99E00E946C8DE1
:10DCF000BE0163577F4F88EC99E00E94058E88EC47
:10DD000099E00E94F58B66E378E1CE0185589F4F3C
:10DD10000E945E89BE0165587F4FCE0183579F4F99
:10DD20000E949487982ECE0185589F4F0E94568955
:10DD3000992099F1CF56DF4F28813981C159D040C0
:10DD400049E050E0BE0163577F4FCE0185589F4F99
:10DD50000E94A689ED968EAD9FADED97412C512C7A
:10DD60003201009719F00E94D9CD2B014201CE015A
:10DD700085589F4F0E9456894114510429F0D701BC
:10DD800058965C924E925797B40188EC99E00E94A5
:10DD9000ECA688EC99E00E94F58BF70187849088C7
:10DDA00081149104D1F0CF56DF4F88819981C159F8
:10DDB000D040892B91F0BE0163577F4FCE0185582B
:10DDC0009F4F0E948C89CE0185589F4FF401199571
:10DDD000CE0185589F4F0E9456896AE875E0CE01B2
:10DDE00083579F4F0E942689FFEFBF12D7CEC801ED
:10DDF0000E945892D12CC12CD9CECE0185589F4F6C
:10DE00000E9429AB9093900880938F087894C80162
:10DE10000E94589280918F0890919008892BD1F49C
:10DE20006AE875E0CE0183579F4F0E949589CE0125
:10DE300083579F4F0E94FDB8CE0183579F4F0E948A
:10DE4000568960ED78E18EEB99E00E94138EF12CFB
:10DE5000E12C16CF0E946D6380918808882329F0F9
:10DE60000E9406A670FF0E946E1B69EC78E184EBAD
:10DE700099E00E94138E04CFE0E3EE16E1E0FE0687
:10DE800051F465EB78E184EB99E00E94138EC801B0
:10DE90000E945892F5CE6DE978E18EEB99E00E94F0
:10DEA000138EC8010E945892B7018EEB99E00E9430
:10DEB000ECA68EEB99E00E94F58BE2CE6AE878E161
:10DEC00085E69AE00E94138EEE24EA94FE2CD8CECA
:10DED0005F926F927F928F929F92AF92BF92CF92FA
:10DEE000DF92EF92FF920F931F93CF93DF93CDB703
:10DEF000DEB7C157D1090FB6F894DEBF0FBECDBF54
:10DF00004C018B01F42E642F85E69AE00E94E5A671
:10DF100060ED7CE085E69AE00E94138EB801CE01A8
:10DF200001965C010E948C89B50185E69AE00E9409
:10DF3000058E85E69AE00E94F58BC5010E94568900
:10DF400092E0F9127EC26EEC7CE0C5010E945E890F
:10DF5000B501C8010E94C487F82EC5010E945689E8
:10DF6000FF2009F4E7C220E04DE251E0B4018FE563
:10DF700099E00E94BF8EE0907E08F0907F0867ECE9
:10DF80007CE0CE0184599F4F0E945E8960EC7CE06A
:10DF9000CE018A599F4F0E945E89CE01865A9F4FBB
:10DFA0000E94C521A0961FADA0976F960FAD6F97E9
:10DFB0006E96DFAC6E976D96CFAC6D976AE875E0A4
:10DFC000CE0181960E949589BE016F5D7F4FC5018C
:10DFD0000E948C896C2DC5010E94A78865E775E0B9
:10DFE0000E94D8886D2D0E94A78865E775E00E9481
:10DFF000D888602F0E94A78865E775E00E94D888BE
:10E00000612F0E94A788BC01CE01805A9F4F0E94B9
:10E010008C89C5010E945689CE0181960E9456893D
:10E020006BEB7CE0CE018C5A9F4F0E945E896AE8C0
:10E0300075E0CE01825B9F4F0E94958900E919E04F
:10E04000D80118966C9170E084E0759567958A9573
:10E05000E1F7C5010E9466A34D815E8169817A81E5
:10E06000CE01825B9F4F0E945588C5010E94568950
:10E07000F80160856F7070E0C5010E9466A34D8154
:10E080005E8169817A81CE01825B9F4F0E945588B3
:10E09000C5010E9456890F5F1F4FF9E006391F071F
:10E0A00079F665EB7CE0CE01885B9F4F0E945E892C
:10E0B00064E97CE0CE0181960E945E89BE016F5DBD
:10E0C0007F4FCE01805C9F4F0E948C89BE01685BB0
:10E0D0007F4FCE01805C9F4F0E94F288BE01625B41
:10E0E0007F4F0E94F288BE016C5A7F4F0E94F288D7
:10E0F000BE01605A7F4F0E94F288BE016A597F4F6D
:10E100000E94F2888C014AE0B50180E590E00E940F
:10E11000A3CEF50101900020E9F73197AF014A192C
:10E120005B09B501C8010E945588811103C0C8016F
:10E130000E949588BE0164597F4FC8010E94F288F1
:10E14000B7010E94D888BC01C4010E94058EC40199
:10E150000E94F58BCE01805C9F4F0E945689CE01B4
:10E1600081960E945689CE01885B9F4F0E945689F6
:10E17000CE01825B9F4F0E945689CE018C5A9F4FE1
:10E180000E945689CE01805A9F4F0E945689CE0127
:10E190008A599F4F0E945689CE0184599F4F0E94F1
:10E1A0005689C4010E94F58B64E670E080E090E03F
:10E1B0000E9400B0D401ED91FC910488F589E02D16
:10E1C000C401199501E010E098C02A966EAD7FADAC
:10E1D0002A97CE0181960E9409A8892B09F464C16F
:10E1E00024961CAE1DAE1EAE1FAE249728961CAE04
:10E1F0001DAE1EAE1FAE289722968FAD2297807F50
:10E2000022968FAF229740E053E0BE016F5D7F4FB3
:10E21000CE01805C9F4F0E944B3C00E020E033E049
:10E2200040E250E0B501CE01805C9F4F0E946A2E13
:10E23000BC01C6010E94308908EC10E137C1EE2014
:10E2400009F4FDC046E050E070E060E0C8010E94C3
:10E25000208740918C0850918D08D8016D917C9158
:10E26000CE0181960E94613ECE0181960E94583770
:10E2700000E911E08823E9F18BA5873061F4CE0134
:10E2800081960E943B4161E0892B09F462E0CE0156
:10E2900081960E94111E24961CAE1DAE1EAE1FAEAE
:10E2A000249728961CAE1DAE1EAE1FAE2897229650
:10E2B0008FAD2297807F22968FAF229740E053E068
:10E2C000BE016F5D7F4FCE01805C9F4F0E944B3C33
:10E2D00000E020E033E040E250E0B501CE01805C98
:10E2E0009F4F0E946A2EBC01C6010E94308908EC33
:10E2F00010E1CE0181960E94EB3EC801CF58DF4F5E
:10E300000FB6F894DEBF0FBECDBFDF91CF911F9146
:10E310000F91FF90EF90DF90CF90BF90AF909F90C4
:10E320008F907F906F905F900895F8016081718168
:10E330000E9446A27C01892B09F044C104E911E046
:10E34000DCCFEE2009F47BC049E050E070E060E0F3
:10E35000C8010E9420874AE0B401C5010E94728B67
:10E3600041E050E06DE574E0C8010E9455884D81A0
:10E370005E8169817A81C8010E94558860E77CE0EE
:10E3800085E69AE00E94138EB801CE0181960E9424
:10E390008C89BE016F5D7F4F85E69AE00E94058EF5
:10E3A00085E69AE00E94F58BCE0181960E945689FF
:10E3B00068E67CE0CE0181960E945E89F801848146
:10E3C00095812DA13EA182179307E1F4892BA1F13C
:10E3D000E080F18069A07AA0D7018D917D0188232A
:10E3E00059F1082E000C990B0E94D7D96C01F3014A
:10E3F00081913F01082E000C990B0E94D7D9C816B5
:10E40000D90651F3CE0181960E945689552041F0DC
:10E4100021E048EC50E0B4018FE599E00E94BF8E06
:10E42000D8018D919C910E94ED8E009711F484E9A2
:10E4300091E08C01C50141C055245394E3CF01E91B
:10E440007ECFB1E0FB1274C06DE87CE0C5010E9494
:10E450005E89B501C8010E949487582EC5010E94AB
:10E460005689552069F1EE2051F346E050E070E006
:10E4700060E0C8010E9420874AE0B401CE01885BB9
:10E480009F4F0E94728B40918C0850918D08F8012B
:10E4900060817181CE0181960E94613ECE0181969C
:10E4A0000E945837811191CE00E911E0CE0181968A
:10E4B0000E94EB3ECE01885B9F4F0E9456891DCF84
:10E4C00066E77CE0C5010E945E89B501C8010E9433
:10E4D0009487F82EC5010E945689F11032CF6BE562
:10E4E0007CE0C5010E945E89B501C8010E94948745
:10E4F000182FC5010E94568900E0112309F4FDCEB2
:10E5000080E00E94A4A663E37CE084EB99E00E9493
:10E51000138E84EB99E00E94F58B6AE875E0C501E3
:10E520000E949589C5010E94FDB8C5010E945689C7
:10E5300000E049CE66E87CE0C5010E945E89B50135
:10E54000C8010E949487F82EC5010E945689F110D7
:10E5500076CE60E87CE0C5010E945E89B501C80105
:10E560000E949487F82EC5010E945689FF2001F36E
:10E57000EE2009F464CF45E050E070E060E0C801AF
:10E580000E94208765E775E0C8010E94AF87882355
:10E5900039F0E0908C08F0908D08E114F10491F4CA
:10E5A0006AE875E0C8010E94AF87811107C08091B9
:10E5B0008C0890918D08009709F0B7CEE0908F08F5
:10E5C000F090900820E048EC50E2B4018FE599E02B
:10E5D0000E94BF8EC4010E94F58B1C821B8289EAB7
:10E5E00092E09A8389839E828D828FEF9FEF988736
:10E5F0008F83B701C5010E941690D6CD4F925F92CE
:10E600006F927F928F929F92AF92BF92CF92DF9242
:10E61000EF92FF920F931F93CF93DF93CDB7DEB7A7
:10E62000CF52D1400FB6F894DEBF0FBECDBF2091C0
:10E630008C0730918D07F9017196E532F10508F0EC
:10E6400011C78827E95DFC488F4F0C94F1D5D9801C
:10E65000C480327A327A327A327A0F800180327A0A
:10E66000327A327A327A327A327A327A327A327A4A
:10E670004C73EE760F78E879627BFD7EFC7F327A10
:10E68000327A327A327A327A2E80418084805B808C
:10E69000327A327A327A69800E94A322029709F490
:10E6A000E1C688EE93E0CC5DDE4F99838883C45247
:10E6B000D140CA5DDE4F188219821A821B82C6526F
:10E6C000D140C25EDE4F99838883CE51D140C05E77
:10E6D000DE4F188219821A821B82C052D140C85E56
:10E6E000DE4F99838883C851D140C65EDE4F1882C1
:10E6F00019821A821B82CA51D140CE5EDE4F9983A5
:10E700008883C251D140CC5EDE4F188219821A82B2
:10E710001B82C451D14060E37EE084EB99E00E940B
:10E72000138E84EB99E00E94F58B80919009909173
:10E730009109892B09F45CC00E94A7A3882309F4DE
:10E7400057C082E70E9492A380919009909191090D
:10E75000DC01ED91FC910088F189E02D60E170E031
:10E760001995BE016F5F7F4F80919009909191093B
:10E770000E9448A389819A81AB81BC81CA5DDE4F2A
:10E7800088839983AA83BB83C652D1408091900924
:10E7900090919109DC01ED91FC910488F589E02DBF
:10E7A0001995CA5DDE4F8881C652D140882301F198
:10E7B0008F3FA9F4C95DDE4F8881C752D1408F3F9A
:10E7C00071F4C85DDE4F8881C852D1408F3F39F463
:10E7D000C75DDE4F8881C952D1408F3F49F00E940A
:10E7E00006A671FF1DC18091C306833008F018C1D1
:10E7F00064E27EE084EB99E00E94138E0FB6F894F9
:10E80000A8958091600088618093600010926000FC
:10E810000FBE8091B80681112AC01092A0061092F6
:10E820009F0688EE93E0A0E0B0E08093A10690936D
:10E83000A206A093A306B093A4068EEB93E0909358
:10E840009E0680939D0688EE93E09093AC0680939D
:10E85000AB061092AD061092AE061092AF06109263
:10E86000B00688E08093B50681E08093B8068AE51B
:10E8700096E09093C2068093C1060E945C9610E0D9
:10E8800000E0882309F4AAC080E591E00E94D1AAA3
:10E8900046E050E068E979E089E090E00E94C093AA
:10E8A00088EE93E09A8389831B821C821D821E82DC
:10E8B000CE0103960E9429218091C1069091C20643
:10E8C000FC0112A213A214A215A2DC0116A217A227
:10E8D00010A611A612A613A614A615A640EE5EE277
:10E8E00060E070E046AB57AB60AF71AF40EA5FE00D
:10E8F00060E070E042AF53AF64AF75AF189626E0AA
:10E90000FD01322F11923A95E9F7AC01425F5F4F5A
:10E9100034E1FA0111923A95E9F7E8E9F9E001905A
:10E920000D922A95E1F7FC01EE5BFF4F10820E94E9
:10E930008E9D8C01019709F051C080E591E00E9405
:10E94000D1AA6091C1067091C206625F7F4FCE016D
:10E9500001960E94538ECE0103960E942921609158
:10E96000C1067091C2066A5E7F4FCE0101960E9479
:10E97000538ECE0103960E9437216091C10670919B
:10E98000C2066E5E7F4FCE0101960E94538ECE016D
:10E9900003960E9430216091C1067091C206625EAA
:10E9A0007F4FCE0101960E94538E8B819C81AD8159
:10E9B000BE818093210990932209A0932309B093EB
:10E9C00024090E94E8AE7F738091020290910302B5
:10E9D00068277927709303026093020288E199E225
:10E9E0000FB6F894A895809360000FBE90936000D6
:10E9F000A895012B09F085C26AEB7DE08EEB99E0CA
:10EA00000E94138E6BE87DE08EEB99E00E94138EDE
:10EA10008091C3068F5F8093C30686EF9FEFE0C1AE
:10EA20006EE07EE084EB99E00E94138E88EE93E026
:10EA30009A838983CA5DDE4F88819981AA81BB81CF
:10EA4000C652D1408B839C83AD83BE83CE01019699
:10EA50000E9487198091900990919109892B09F45E
:10EA60003BC20E94A7A3882309F436C282E70E9412
:10EA700092A38091900990919109DC01ED91FC9114
:10EA80000088F189E02D64E170E01995BE016F5FA7
:10EA90007F4F80919009909191090E9448A38981AC
:10EAA0009A81AB81BC81C05EDE4F88839983AA8343
:10EAB000BB83C052D1408091900990919109DC01B3
:10EAC000ED91FC910488F589E02D1995C05EDE4F2B
:10EAD0008881C052D140882309F4FEC18F3FB1F430
:10EAE000CF5DDE4F8881C152D1408F3F79F4CE5D3A
:10EAF000DE4F8881C252D1408F3F41F4CD5DDE4F61
:10EB00008881C352D1408F3F09F4E6C168E07EE0BE
:10EB100084EB99E00E94138E88EE93E09A838983B8
:10EB2000C05EDE4F88819981AA81BB81C052D140ED
:10EB30008B839C83AD83BE83CE0101960E9487198F
:10EB40008091900990919109892B09F496C10E94B6
:10EB5000A7A3882309F491C182E70E9492A3809120
:10EB6000900990919109DC01ED91FC910088F18967
:10EB7000E02D68E170E01995BE016F5F7F4F8091D5
:10EB80009009909191090E9448A389819A81AB8153
:10EB9000BC81C65EDE4F88839983AA83BB83CA513A
:10EBA000D1408091900990919109DC01ED91FC9107
:10EBB0000488F589E02D1995C65EDE4F8881CA511B
:10EBC000D140882309F459C18F3FB1F4C55EDE4FAF
:10EBD0008881CB51D1408F3F79F4C45EDE4F88816C
:10EBE000CC51D1408F3F41F4C35EDE4F8881CD517F
:10EBF000D1408F3F09F441C163E07EE084EB99E0AE
:10EC00000E94138E88EE93E09A838983C65EDE4F5E
:10EC100088819981AA81BB81CA51D1408B839C8311
:10EC2000AD83BE83CE0101960E9487198091900921
:10EC300090919109892B09F4D8C00E94A7A3882339
:10EC400009F4D3C082E70E9492A380919009909129
:10EC50009109DC01ED91FC910088F189E02D6CE1D6
:10EC600070E01995BE016F5F7F4F80919009909180
:10EC700091090E9448A389819A81AB81BC81CC5EB5
:10EC8000DE4F88839983AA83BB83C451D14080918E
:10EC9000900990919109DC01ED91FC910488F5892E
:10ECA000E02D1995CC5EDE4F8881C451D140882378
:10ECB00009F49BC08F3FB1F4CB5EDE4F8881C55114
:10ECC000D1408F3F79F4CA5EDE4F8881C651D14072
:10ECD0008F3F41F4C95EDE4F8881C751D1408F3FDD
:10ECE00009F483C06CEF7DE084EB99E00E94138E01
:10ECF00008EE13E01A830983CC5EDE4F8881998188
:10ED0000AA81BB81C451D1408B839C83AD83BE83D8
:10ED1000CE0101960E9487191A830983CC5EDE4FCB
:10ED200088819981AA81BB81C451D1408B839C8306
:10ED3000AD83BE83CF57DF4F19830883C158D040BE
:10ED4000C65EDE4F88819981AA81BB81CA51D140BC
:10ED5000CD57DF4F88839983AA83BB83C358D040A4
:10ED6000CE53DF4F19830883C25CD040C05EDE4FB4
:10ED700088819981AA81BB81C052D140CC53DF4F99
:10ED800088839983AA83BB83C45CD040CE5FDE4F67
:10ED900019830883C250D140CA5DDE4F88819981B2
:10EDA000AA81BB81C652D140CC5FDE4F8883998354
:10EDB000AA83BB83C450D1409E012F5F3F4FAE0159
:10EDC0004F575F4FBE016E537F4FCE018E5F9E4FF8
:10EDD0000E94B8AB84EB99E00E94F58B82E090E052
:10EDE00090938D0780938C073DC388EE93E09A83C0
:10EDF0008983C65EDE4F488159816A817B81CA5111
:10EE0000D1404B835C836D837E83CF57DF4F9983E3
:10EE10008883C158D040C05EDE4F488159816A81E5
:10EE20007B81C052D140CD57DF4F488359836A83DD
:10EE30007B83C358D040CE53DF4F99838883C25C15
:10EE4000D040CA5DDE4F88819981AA81BB81C652BC
:10EE5000D140CC53DF4F88839983AA83BB83C45CA2
:10EE6000D040AE014F5F5F4FBE016F577F4FCE0165
:10EE70008E539F4F0E94F7ABADCF88EE93E09A83FD
:10EE80008983C05EDE4F488159816A817B81C0528F
:10EE9000D1404B835C836D837E83CF57DF4F998353
:10EEA0008883C158D040CA5DDE4F88819981AA818C
:10EEB000BB81C652D140CD57DF4F88839983AA8347
:10EEC000BB83C358D040BE016F5F7F4FCE018F57C9
:10EED0009F4F0E9449AC7ECF88EE93E09A8389834E
:10EEE000CA5DDE4F88819981AA81BB81C652D1401B
:10EEF0008B839C83AD83BE83CE0101960E9494AC2C
:10EF000069CF6BE77DE084EB99E00E94138ECE0120
:10EF100001960E94C5218B819C81AD81BE81CA5D15
:10EF2000DE4F88839983AA83BB83C652D14008EE03
:10EF300013E01A830983CE0101960E94871984EB9E
:10EF400099E00E94F58BCE018C5D9E4F0E94B2A489
:10EF50008091210990912209A0912309B09124095F
:10EF60008B839C83AD83BE83C05EDE4F8883998391
:10EF7000AA83BB83C052D140CE01825E9E4F0E94C5
:10EF80005CA51A8309831B821C821D821E8280E578
:10EF900091E00E94D1AA44E050E0BE016D5F7F4F36
:10EFA00081E090E00E9435938B819C81AD81BE8190
:10EFB000C65EDE4F88839983AA83BB83CA51D14042
:10EFC000CE01885E9E4F0E94B1A51A8309831B82E1
:10EFD0001C821D821E8280E591E00E94D1AA44E03D
:10EFE00050E0BE016D5F7F4F85E090E00E94359359
:10EFF0008B819C81AD81BE81CC5EDE4F88839983FD
:10F00000AA83BB83C451D140CE018E5E9E4F0E9425
:10F0100007A581E00E949BA61092C306DFCE8091D7
:10F020008F078111D2C10E94E1216AEA71E185E670
:10F030009AE00E94138E85E69AE00E94F58B8091FB
:10F04000900990919109892B09F432C10E94A7A3DC
:10F05000882309F42DC182E70E9492A38091900930
:10F0600090919109DC01ED91FC910088F189E02DEE
:10F0700060E570E019954FE050E0BE016F5F7F4F93
:10F0800080919009909191090E94ECA38C0180914C
:10F09000900990919109DC01ED91FC910488F5892A
:10F0A000E02D19950115110509F402C1E1E0F0E028
:10F0B000EC0FFD1FE00FF11F1082BE016F5F7F4F4D
:10F0C00085E69AE00E946C8D85E69AE00E94F58BB9
:10F0D000CE01865D9E4F0E94C521C45DDE4F8881B2
:10F0E0009981AA81BB81CC52D14080936F099093C2
:10F0F0007009A0937109B093720967E775E08FE515
:10F1000099E00E942689BE016F5F7F4FCE01825E2B
:10F110009E4F0E94958966E87EE0CE01885E9E4FF4
:10F120000E945E8967E775E0CE018E5F9E4F0E9468
:10F130009589BE016E5F7E4FCE018E5E9E4F0E940E
:10F140008C89BE01685E7E4FCE018E5E9E4F0E940E
:10F15000F288BE01625E7E4F0E94F2888C016AE8EE
:10F1600075E0CE018C5D9E4F0E949589F8018481E7
:10F170009581880F991F880F991F63E070E00E94A6
:10F18000C9D5CE018C5D9E4F0E942D88F12CE12CBB
:10F19000D80114968D919C91E816F90608F0B7C035
:10F1A000B701C8010E948387E82F880FFF0BF595F0
:10F1B000E795F595E795EF73FF27E35CF14F6491D1
:10F1C000CE018C5D9E4F0E948188B701C8010E94CC
:10F1D0008387B0E18B0250011124E0E3AE22BB240F
:10F1E0006701FFEFCF1ADF0AD80114968D919C9129
:10F1F000C816D90608F078C0B601C8010E948387F6
:10F20000E82F880FFF0BB4E0F595E795BA95E1F785
:10F21000EF70FF27EA29FB29E35CF14F6491CE01EF
:10F220008C5D9E4F0E948188B601C8010E94838731
:10F23000B4E08B0250011124ECE3AE22BB24670141
:10F24000F2E0CF0ED11CD80114968D919C91C81676
:10F25000D90608F03EC0B601C8010E948387E82F96
:10F26000880FFF0BA6E0F595E795AA95E1F7E37007
:10F27000FF27EA29FB29E35CF14F6491CE018C5D05
:10F280009E4F0E948188B601C8010E948387E82FA3
:10F29000EF730E2E000CFF0BE35CF14F6491CE0177
:10F2A0008C5D9E4F0E948188B3E0EB0EF11C70CF05
:10F2B00061ED7EE0CE0101960E9430CE69E97EE0EC
:10F2C0008EEB99E00E94138E8EEB99E00E94F58BF5
:10F2D000F4CEF501E35CF14F6491CE018C5D9E4F5D
:10F2E0000E9481886DE3DBCFF501E35CF14F64910F
:10F2F000CE018C5D9E4F0E94818842E050E06FE716
:10F3000075E0CE018C5D9E4F0E945588CDCF6FE792
:10F310007EE0CE018F579F4F0E945E89BE016F57DE
:10F320007F4FCE018E539F4F0E948C89BE016C5D32
:10F330007E4FCE018E539F4F0E94F288BC0185E61E
:10F3400099E00E943F89CE018E539F4F0E945689BB
:10F35000CE018F579F4F0E945689CE018C5D9E4FE4
:10F360000E945689CE018E5E9E4F0E945689CE0124
:10F370008E5F9E4F0E945689CE01885E9E4F0E94EE
:10F380005689CE01825E9E4F0E9456898AEF98E090
:10F3900090936C0980936B098EE999E090936E09C4
:10F3A00080936D098BE799E00E943F2188E69FE6F4
:10F3B00090937A098093790968E87EE084EB99E07C
:10F3C0000E94138E81E080938F0783E090E008CD48
:10F3D00080918E0881115AC10E9406A664FD2DC03D
:10F3E00080917A0881111EC00E942A6B883C910589
:10F3F00019F484E090E0F4CC8091880863E871E12E
:10F40000811112C0CE0101960E94C5218B819C8181
:10F41000AD81BE81892B8A2B8B2B09F4FECA8FE02C
:10F4200090E0DECC63E771E184EB99E00E94138EFB
:10F4300084EB99E00E94F58BDCCF809188088823CB
:10F4400009F43DC184E090E090938D0780938C0790
:10F4500069E371E184EB99E00E94138E84EB99E0FB
:10F460000E94F58B0FB6F894A89580916000886192
:10F4700080936000109260000FBE80918C07909185
:10F480008D0702970CF4F4C08091C3068111BEC6AB
:10F490000091C1061091C2060115110509F4B6C606
:10F4A0000E9433B04B015C017801FEE3EF0EF11CCA
:10F4B000F70180819181A281B381A5019401281B6C
:10F4C000390B4A0B5B0BCA01B901683E33E0730785
:10F4D00081059105A0F128EE33E040E050E00E9464
:10F4E00066D5861A970AA80AB90AD7018D929D9205
:10F4F000AD92BC921397F80186A597A5A0A9B1A9D2
:10F5000069017A01CC0CDD1CEE1CFF1C8C159D05DD
:10F51000AE05BF0508F065C616A617A610AA11AA63
:10F52000F80182A993A9A4A9B5A98C159D05AE05DA
:10F53000BF0508F05FC612AA13AA14AA15AAF801FB
:10F5400086A597A5A0A9B1A9892B8A2B8B2B09F099
:10F550005AC6EE5BFF4F8081833009F054C684E0C9
:10F560008083C8010E948E9D01967C01F80182A9CA
:10F5700093A9A4A9B5A9892B8A2B8B2BA1F4EE5BA7
:10F58000FF4F8081833011F081110DC01082F8018E
:10F590003E9684E1DF011D928A95E9F7C8010E9439
:10F5A0008E9D03967C01B2E0EB16F10429F0E4E0B5
:10F5B000EE16F10409F044C080E591E00E94D1AA62
:10F5C0006091C1067091C206625F7F4FCE010196C5
:10F5D0000E94538ECE0103960E9429216091C1069C
:10F5E0007091C2066A5E7F4FCE0101960E94538ED3
:10F5F000CE0103960E9437216091C1067091C20628
:10F600006E5E7F4FCE0101960E94538ECE0103960F
:10F610000E9430216091C1067091C206625E7F4FE8
:10F62000CE0101960E94538E8B819C81AD81BE815B
:10F630008093210990932209A0932309B093240970
:10F640000E94A322029709F4EDC5F3E0EF16F1043E
:10F6500009F4FCC50CF0DDC531E0E316F10409F452
:10F66000F2C565E870E142E0E416F10409F4F3C57F
:10F6700088E199E20FB6F894A895809360000FBED8
:10F680009093600020918C0730918D07C901C15D76
:10F69000DE4F0FB6F894DEBF0FBECDBFDF91CF9126
:10F6A0001F910F91FF90EF90DF90CF90BF90AF90A0
:10F6B0009F908F907F906F905F904F9008958FE014
:10F6C00090E0C2CEA8958091800890918108009723
:10F6D00021F00E9449A7823068F466E271E184EB70
:10F6E00099E00E94138E84EB99E00E94F58B87E0ED
:10F6F00090E076CBC85EDE4F1882C851D140FE0143
:10F70000EE5FFE4F119211928EE0DF011D928A95FD
:10F71000E9F70E9464A2882319F085E090E060CBAD
:10F72000E0908008F0908108E114F10441F0C701F5
:10F730000E9449A7082F10E0023011055CF467EE23
:10F740007FE08EEB99E00E94138E8EEB99E00E9491
:10F75000F58B65CE70E060E0C7010E94A11D0097A7
:10F7600009F476C090937F0880937E086AED7FE06D
:10F7700084EB99E00E94138E60917E0870917F085F
:10F7800084EB99E00E946C8D84EB99E00E94F58BEC
:10F79000E0908008F090810861E070E0C7010E946D
:10F7A000A11D5C010230110509F455C062E0C701DA
:10F7B0000E94BEA2FC01C184D2840330110509F469
:10F7C00053C063E070E0C7010E94A11D7C018091DD
:10F7D000900990919109892B09F44BC00E94A7A32D
:10F7E000882309F446C082E70E9492A38091900981
:10F7F00090919109DC01ED91FC910088F189E02D57
:10F8000060E470E019954FE050E0BE016E5F7E4FFE
:10F8100080919009909191090E94ECA34C018091F4
:10F82000900990919109DC01ED91FC910488F58992
:10F83000E02D199581149104E1F0E2E0F1E0EC0F84
:10F84000FD1FE80DF91D10828E010E5F1E4F27C0AF
:10F8500085E792E087CFFBE5CF2EF7E0DF2E9E0114
:10F86000285E3E4F7901B3CFAE01485E5E4F7A010C
:10F87000AECF0530110544F364E070E0809180085C
:10F88000909181080E94A11D8C016AEB7FE084EBBE
:10F8900099E00E94138E84EB99E00E94F58BB09260
:10F8A0005309A0925209D0925509C092540989EF88
:10F8B0009EE390934B0980934A0940E150E06DEA42
:10F8C0007FE0CE018E539F4F0E945ECE30E020E05D
:10F8D00041E050E060E2CE018F579F4F0E945728D1
:10F8E00040E250E06DEF7FE1CE018F579F4F0E94C5
:10F8F00040CE6CE87FE084EB99E00E94138EB50166
:10F9000084EB99E00E946C8D6AE87FE084EB99E0DB
:10F910000E94138EB60184EB99E00E94ECA663E886
:10F920007FE084EB99E00E94138EB70184EB99E0AD
:10F930000E946C8D6EE77FE084EB99E00E94138E4D
:10F94000F7018081811104C010E000E0F12CE12C6E
:10F95000A0907E08B0907F080E9464A28111C5C16A
:10F960008091350990913609DC01ED91FC91068872
:10F97000F789E02D1995882309F497C081E090E07C
:10F980009093400980933F0987E0EAE2F2E0DE01CC
:10F99000119601900D928A95E1F7FE01319685E06E
:10F9A00090E02191A0913709B0913809A80FB91FB3
:10F9B0002C9301968C309105A1F786E3E114F104B4
:10F9C00029F086EB0115110509F086EFC090370983
:10F9D000D0903809F601848780913C098587809111
:10F9E0003B0986878090390990903A09B401C50196
:10F9F0000E9471CE41968816990608F08DC08091BC
:10FA0000350990913609DC01ED91FC910488F58966
:10FA1000E02D19956BE37FE08EEB99E00E94138E49
:10FA200060915809709159098EEB99E00E94ECA6FB
:10FA300063E27FE08EEB99E00E94138E8EEB99E0FB
:10FA40000E94F58B80917D08882379F0E0918008F1
:10FA5000F09181088281938190938108809380083E
:10FA6000892B09F0BBC10E944B190E9433B06093EF
:10FA7000C4067093C5068093C6069093C70680910E
:10FA8000C0068F5F8093C00683330CF4B2C165EF6C
:10FA90007EE08EEB99E00E94138E8EEB99E00E943F
:10FAA000F58B1092C0060C940D75609152097091FF
:10FAB00053098091350990913609DC01ED91FC9153
:10FAC00040915409509155096115710571F00088F4
:10FAD000F189E02D1995019709F450CF8EEF9FEF32
:10FAE000909359098093580995CF0684F785E02DA6
:10FAF00028EE33E03A83298340904E0950904F0915
:10FB000060905009709051094B825C826D827E82B8
:10FB1000BE016F5F7F4FDECF4FE050E0B601C50101
:10FB20000E949CA26C01A0903909B0903A09B501DD
:10FB3000CE018F579F4F0E9471CE8C0D9D1D029656
:10FB4000A816B90608F45BCF60913709709138099F
:10FB5000A601CE018F579F4F0E949CA26C01A090DE
:10FB60003909B0903A09B501CE018E539F4F0E94DA
:10FB700071CE8C0D9D1D0296A816B90608F43FCFD4
:10FB80006091370970913809A601CE018E539F4FBD
:10FB90000E949CA26C01E114F104B9F1A090390912
:10FBA000B0903A09B501C7010E9471CE96012E5F4F
:10FBB0003F4F820F931FA816B90608F420CF60911B
:10FBC000370970913809A601C7010E949CA26C01F7
:10FBD00001151105D1F0E0903909F0903A09B7010B
:10FBE000C8010E9471CE96012E5F3F4F820F931F76
:10FBF000E816F90608F403CF6091370970913809C7
:10FC0000A601C8010E949CA26C01A60145505109A1
:10FC1000609137097091380980E10E943FB00E94DD
:10FC200033B06093410970934209809343099093E4
:10FC3000440960934509709346098093470990935E
:10FC400048098091350990913609DC01ED91FC91CC
:10FC50000084F185E02D1995892B21F50E9433B0A0
:10FC600000914509109146092091470930914809B2
:10FC70006B017C01C01AD10AE20AF30A20913D0906
:10FC800030913E09A8EEB3E00E94BAD5C616D70659
:10FC9000E806F906B0F28CEF9FEF90935909809334
:10FCA0005809ADCECE018E5E9E4F0E94C2B4643024
:10FCB00071058105910509F0A2CEE0913709F09117
:10FCC0003809838190E08111E8CF0E9433B06093BE
:10FCD000450970934609809347099093480910920B
:10FCE000490910925909109258091092C00660E70C
:10FCF0007FE084EB99E00E94138E60917E08709102
:10FD00007F0884EB99E00E946C8D84EB99E00E945F
:10FD1000F58B81E080937A0830E020E043E050E00A
:10FD200061E4CE0101960E94572862E875E0CE0199
:10FD300001960E943CDACE0101960E9424B430E084
:10FD400020E042E050E061E4CE0101960E94572895
:10FD500066E875E0CE0101960E943CDABE016F5F55
:10FD60007F4F85E69AE00E949A8B85E69AE00E9492
:10FD7000F58BCE0101960E9424B430E020E041E0F2
:10FD800050E061E4CE0101960E94572866E875E0D4
:10FD9000CE0101960E943CDABE016F5F7F4F85E67F
:10FDA0009AE00E949A8B85E69AE00E94F58BCE013C
:10FDB00001960E9424B485E090E090938D07809393
:10FDC0008C070E9433B06093C4067093C50680937D
:10FDD000C6069093C7066DE47FE03CCB6AED7EE0FB
:10FDE00084EB99E00E94138E84EB99E00E94F58BDE
:10FDF0003CCE8CE090E00C94F0760E9433B09B01F6
:10FE0000AC016091C4067091C5068091C6069091C0
:10FE1000C706A12CB12C650110E4E12E1FE1F12EE3
:10FE200000E010E00E947627882309F41BCB30E025
:10FE300020E043E050E061E4CE018F579F4F0E94E5
:10FE4000572862E875E0CE018F579F4F0E943CDA39
:10FE50000091390910913A09B801CE018F579F4F8F
:10FE60000E9471CE09960817190790F10E9464A2AA
:10FE7000882371F180913F0990914009019609F41E
:10FE8000B8C09093400980933F09E0913709F09101
:10FE90003809809140098583E0913709F09138094C
:10FEA00080913F098683609137097091380947E056
:10FEB00050E0CE018F579F4F0E949CA2AC0145504D
:10FEC0005109609137097091380982EA0E943FB068
:10FED000FE01EE53FF4F119211928EE3DF011D924E
:10FEE0008A95E9F71A821982FE0133968EE7DF01BF
:10FEF0001D928A95E9F730E020E041E050E060E4AF
:10FF0000CE018E539F4F0E9457284FE350E06DEF74
:10FF10007FE1CE018E539F4F0E9440CE4FE750E0CD
:10FF200067EF7FE1CE0101960E945ECEBE016F5F5A
:10FF30007F4FCE018E539F4F0E9401B130E020E0F1
:10FF400041E050E060E4CE018E539F4F0E9457285D
:10FF50004FE350E060E570E1CE018E539F4F0E9469
:10FF600040CE4FE750E066E470E1CE0101960E947A
:10FF70005ECE4FE750E063E370E1CE0101960E9450
:10FF800040CEBE016F5F7F4FCE018E539F4F0E94C8
:10FF900001B130E020E041E050E060E4CE018E535A
:10FFA0009F4F0E9457284FE350E064E170E2CE017A
:10FFB0008E539F4F0E9440CE4FE750E063E270E1C6
:10FFC000CE0101960E945ECEBE016F5F7F4FCE01D3
:10FFD0008E539F4F0E9401B186E090E090938D0771
:10FFE00080938C0769E071E184EB99E00E94138EA5
:10FFF00039CA81E090E045CF0E9464A2811132CAE3
:020000021000EC
:10000000F8C90E9433B06093C4067093C50680930C
:10001000C6069093C70685EF9FEF0C94F0760E947A
:1000200033B09B01AC016091C4067091C50680910C
:10003000C6069091C706A12CB12C650118E8E12EE7
:1000400013E1F12E00E010E00E947627882309F4E6
:1000500009CA10928D0710928C0704CA0E9464A2EC
:1000600081110E9413B60E9433B06093C40670934E
:10007000C5068093C6069093C7068DE090E00C9469
:10008000F0760E9433B09B01AC016091C406709180
:10009000C5068091C6069091C706A12CB12C6501BA
:1000A00010E1E12E17E2F12E00E010E00E94762729
:1000B00081119FC9D7C90E9433B06093C406709361
:1000C000C5068093C6069093C7068EE090E00C9418
:1000D000F0760E9433B09B01AC016091C406709130
:1000E000C5068091C6069091C706A12CB12C65016A
:1000F00010ECE12E14EDF12E01E010E00E947627C5
:1001000081110C940D75AEC90E94B669009759F122
:100110008130910509F46DC9019609F0A3C90E94C7
:1001200033B09B01AC016091C4067091C50680910B
:10013000C6069091C706A12CB12C650110E3E12EF3
:1001400015E7F12E00E010E00E947627882309F4DD
:1001500089C966EE70E18EEB99E00E94138EF0E0A3
:10016000E0E019957FC983E190E090938D0780933B
:100170008C070E9433B06093C4067093C5068093C9
:10018000C6069093C7066EC90E9464A281110E94A0
:1001900013B60E944B190E9433B06093C40670934B
:1001A000C5068093C6069093C7068FEE9FEF0C940A
:1001B000F07680918E08811169CA82E190E0909377
:1001C0008D0780938C070E942A6B883C910509F467
:1001D00010C980918808882309F414C96FEB70E175
:1001E00023C9821B930BA40BB50B86A797A7A0ABC3
:1001F000B1AB96C9821B930BA40BB50B82AB93AB2F
:10020000A4ABB5AB9CC9F12CE12CB0C9F12CE12C0D
:1002100017CA54E0E516F104E1F085E0E816F104B0
:1002200009F026CA66EB70E18EEB99E00E94138E0E
:100230008EEB99E00E94F58B86EF9FEF90938D07F0
:1002400080938C0715CA62EA70E1EECF62E770E135
:10025000EBCF66E570E184EB99E00E94138ECE014E
:1002600001960E94C521CE0101960E94871984EB58
:1002700099E00E94F58BFCC9089508950895AF9206
:10028000BF92CF92DF92EF92FF920F931F93CF9383
:10029000DF936C017B018B01040F151FEB015E01E5
:1002A000AE18BF08C017D10759F06991D601ED917A
:1002B000FC910190F081E02DC6011995892B79F709
:1002C000C501DF91CF911F910F91FF90EF90DF90CB
:1002D000CF90BF90AF900895FC01538D448D252F92
:1002E00030E0842F90E0821B930B541710F0CF96D0
:1002F000089501970895FC01918D828D981761F002
:10030000A28DAE0FBF2FB11D5D968C91928D9F5F18
:100310009F73928F90E008958FEF9FEF0895FC01F7
:10032000918D828D981731F0828DE80FF11D858DAA
:1003300090E008958FEF9FEF0895FC01918D228D3D
:10034000892F90E0805C9F4F821B91098F739927C2
:10035000089588EC99E00E949D8121E0892B09F4A1
:1003600020E0822F0895FC01A48DA80FB92FB11DA4
:10037000A35ABF4F2C91848D90E001968F739927DB
:10038000848FA689B7892C93A089B1898C918370B9
:1003900080648C93938D848D981306C00288F389B2
:1003A000E02D80818F7D80830895EF92FF920F93DF
:1003B0001F93CF93DF93EC0181E0888F9B8D8C8D11
:1003C00098131AC0E889F989808185FF15C09FB705
:1003D000F894EE89FF896083E889F98980818370C8
:1003E000806480839FBF81E090E0DF91CF911F9177
:1003F0000F91FF90EF900895F62E0B8D10E00F5F98
:100400001F4F0F731127E02E8C8D8E110CC00FB66D
:1004100007FCFACFE889F989808185FFF5CFCE0105
:100420000E94B381F1CFEB8DEC0FFD2FF11DE35A4C
:10043000FF4FF0829FB7F8940B8FEA89FB89808188
:100440008062CFCFCF93DF93EC01888D8823B9F002
:10045000AA89BB89E889F9898C9185FD03C08081CF
:1004600086FD0DC00FB607FCF7CF8C9185FFF2CF4C
:10047000808185FFEDCFCE010E94B381E9CFDF916E
:10048000CF91089580E090E0892B29F00E94A98106
:1004900081110E94000080E090E0892B49F080E00B
:1004A00090E0892B29F00E94000081110E94000039
:1004B00080E090E0892B49F080E090E0892B29F0E2
:1004C0000E94000081110E94000080E090E0892BD2
:1004D00049F080E090E0892B29F00E940000811112
:1004E0000C9400000895DC01ED91FC910190F081E5
:1004F000E02D19948FEF9FEF0895FC0162897389B5
:10050000848995890895EF920F931F93CF93DF937A
:10051000FC01248D222341F0213051F1DF91CF9154
:100520001F910F91EF90089522893389448955894D
:1005300086899789A08DB18D821B930BA40BB50B77
:10054000892F9A2FAB2FBB278C010F5F1F4F628122
:10055000738184819581CFB7F894DCB7E1E0ECBF7B
:10056000EE24E394E2E0FEEF1995DCBFCFBFD6CFD7
:10057000F0E0E0E0DF91CF911F910F91EF9019949F
:10058000FC01138E128E41110CC082899389A489BB
:10059000B589868B978BA08FB18F148E81E090E008
:1005A000089590E080E00895CF92DF92EF92FF925D
:1005B000CF93DF93DC01CB01642FCFB7F8946D01AB
:1005C000EE24FF24CBBEDCB741E04CBFA901E1E043
:1005D000FEEF1995DCBFCFBFDF91CF91FF90EF9079
:1005E000DF90CF900895CF93DF93FC01248D2111EC
:1005F00010C0EC01828D938D892B49F06689778933
:10060000808D918D30E020E045E00E94D4821B8EE9
:100610001A8EDF91CF9108951F93CF93DF93FC0142
:10062000248D211145C0162FEC01828D938D892BCD
:1006300049F466897789808D918D30E020E043E030
:100640000E94D4824A8D5B8DCA0181709927FE0178
:10065000E80FF91F158F892B69F02D8D3E8D6E895E
:100660007F89888D998D640F751F811D911D41E0D3
:100670000E94D4828A8D9B8D01969B8F8A8F8115D3
:100680009140B1F46E897F89888D998D30E020E0AA
:1006900045E00E94D4821B8E1A8E8E899F89A88D78
:1006A000B98D9F5FAF4FBF4F8E8B9F8BA88FB98F38
:1006B00081E090E0DF91CF911F910895DC01ED91F1
:1006C000FC910280F381E02D40E01994FB0144810C
:1006D000558122813381215031094217530750F44B
:1006E000A081B181A40FB51F8C938481958101965F
:1006F0009583848380E00895CF93DF93EC01E881B4
:10070000F9810284F385E02DCE0119950196B9F7A0
:10071000DF91CF910895CF92DF92EF92FF920F93E6
:100720001F93CF93DF937C016A018B01D0E0C0E07F
:10073000CC15DD0581F0D701ED91FC910284F385A4
:10074000E02DC70119958F3F980729F0F801819393
:100750008F012196EDCFCE01DF91CF911F910F91A7
:10076000FF90EF90DF90CF900895CF93C62FDC01DC
:10077000ED91FC910088F189E02D1995DC01ED9156
:10078000FC910190F081E02D6C2FCF911994062EF1
:10079000000C770BFC01778366830895CF93DF937A
:1007A000EC018E819F81019611F5E881F981008825
:1007B000F189E02DCE011995DC01ED91FC910084C9
:1007C000F185E02D1995892BB1F0E881F98102843A
:1007D000F385E02DCE0119958132910534F3E8813E
:1007E000F9810684F785E02D682FCE01199581E007
:1007F000DF91CF91089580E0FBCFFC0120812EBDD9
:100800009B012150310941F051810DB407FEFDCF0C
:100810004EB55EBD4193F5CF61507109860F971FAC
:100820000DB407FEFDCF2EB5FC0120830895E091A5
:100830009107F0919207808190919007892B808396
:100840000895E0919107F09192079081809190072F
:1008500080958923808308958EBD00000DB407FE26
:10086000FDCF8EB5089590E020917908233339F4B7
:100870000C96982F990F990F990F80E0089548963C
:10088000F8CFCF93DF931F92CDB7DEB76983DC013A
:10089000ED91FC910280F381E02D41E050E0BE013A
:1008A0006F5F7F4F19950F90DF91CF910895EF9271
:1008B000FF920F931F93CF93DF93EC018B017A018B
:1008C0000E9433B0688B798B8A8B9B8B8C819D8146
:1008D000DC01ED91FC910280F381E02DA701B801CC
:1008E000DF91CF911F910F91FF90EF9019941F937B
:1008F000CF93DF93EC01162F0E9433B0688B798B76
:100900008A8B9B8B8C819D81DC01ED91FC91019008
:10091000F081E02D612FDF91CF911F911994CF923B
:10092000DF92EF92FF92CF93DF93EC018E819F8154
:100930008F3F980759F02FEF3FEF3F832E83DF91D2
:10094000CF91FF90EF90DF90CF9008950E9433B049
:100950006B017C01A4EFCA0EA1E0DA1EE11CF11CC0
:10096000E881F9810088F189E02DCE011995DC013B
:10097000ED91FC910084F185E02D1995892B39F4D6
:100980000E9433B06C157D058E059F0548F3E88104
:10099000F9810088F189E02DCE011995DC01ED91F6
:1009A000FC910284F385E02DDF91CF91FF90EF90D1
:1009B000DF90CF9019940E94D2D9AF92BF92CF927C
:1009C000DF92EF92FF920F931F93CF93DF93DC019F
:1009D000CD90DC901197C114D10439F01496CD91CB
:1009E000DC918C017601209761F4DF91CF911F910A
:1009F0000F91FF90EF90DF90CF90BF90AF90089550
:100A000075015701BFEFAB1ABB0AF7018081082EB1
:100A1000000C990B0E9400CE892B91F72197CC0DE9
:100A2000DD1D8881082E000C990B0E9400CE892BB9
:100A300029F0CE15DF0510F02197F3CFAE014F5FFF
:100A40005F4F4E195F09D80115965C934E9314972A
:100A5000CE14DF0420F4B701C6010E940EDAD801DB
:100A6000ED91FC91119714968D919C91E80FF91FCF
:100A70001082BBCF0F931F93CF93DF93D0E0C0E0E2
:100A8000009791F08C01C5EDD7E0688179816115FF
:100A9000710529F0C8010E9452DA892B29F00B80D8
:100AA000DC81C02D209789F7CE01DF91CF911F9176
:100AB0000F910895EF92FF920F931F93CF93DF93BF
:100AC000009751F4CFEFDFEFCE01DF91CF911F916F
:100AD0000F91FF90EF900895DC011C96ED90FC9033
:100AE000F70100811181D801ED91FC910688F78909
:100AF000E02DC8011995882329F3D801ED91FC91C7
:100B00000084F185E02DC8011995D801ED91FC9183
:100B1000892B61F30284F385E02DC8011995EC015E
:100B2000019681F2F801818D882329F06C2F88ECE1
:100B300099E00E94E5A6D70112968C91882321F2B4
:100B4000C532D10509F6D801ED91FC910084F185FB
:100B5000E02DC801199502975CF0D801ED91FC9148
:100B60000688F789E02DC80119958111ECCFAACF2D
:100B7000D1E0C0E0D801ED91FC910284F385E02D35
:100B8000C80119958F3F980709F49CCF9C01215407
:100B900031092A31310570F48D2F8295807F829F33
:100BA000C00D1124D11104C00C2E000CDD0B8CCF14
:100BB000D0E0E0CF9C01215631092A31310560F3A4
:100BC000C0978A30910570F79D2F9295907F989FDE
:100BD000C00D1124E7CFCF92DF92EF92FF920F93D7
:100BE0001F93CF93DF936C018B0186E090E00E940E
:100BF000EECBEC019093DB078093DA07F6010190CE
:100C00000020E9F7CF018C199D090E94EECB7C01F1
:100C1000B6010E945BDAF60101900020E9F73197F6
:100C2000EC19FD09EE0DFF1D1082F982E8821B838D
:100C30000A8380911808909119089D838C83D09322
:100C40001908C0931808DF91CF911F910F91FF9061
:100C5000EF90DF90CF900895FC01868197818F3FC0
:100C6000980729F02FEF3FEF37832683089580857B
:100C700091850C947CCFEF92FF921F93CF93DF93DB
:100C80001F921F92CDB7DEB7182F22E030E0AE01E1
:100C90004F5F5F4F60E270E00E941821E980FA80A8
:100CA000FE24EF24FE2422E030E0AE014F5F5F4FD0
:100CB00060E270E0812F0E94182189819A81982733
:100CC00089279827E816F90689F487E0189FF0012C
:100CD0001124EF5CF74FF582E482C7010F900F906B
:100CE000DF91CF911F91FF90EF9008957C01DBCFB2
:100CF000FF920F931F93CF93DF931F921F92CDB755
:100D0000DEB7F82E22E030E0AE014F5F5F4F66E2C3
:100D100070E00E94182109811A81102701271027ED
:100D200022E030E0AE014F5F5F4F66E270E08F2D52
:100D30000E94182189819A81982789279827081766
:100D4000190749F4C8010F900F90DF91CF911F91BF
:100D50000F91FF9008958C01E3CFCF92DF92EF9235
:100D6000FF920F931F93CF93DF93CDB7DEB7AF976B
:100D70000FB6F894DEBF0FBECDBF7C016A0108EE4E
:100D800013E01A8309831C861B8688EE93E0A0E09B
:100D9000B0E08D879E87AF87B88B8EEB93E09A8704
:100DA0008987188F0F8B198E1A8E1B8E1C8E88E0E8
:100DB00089A31BA70AA71CA61DA61EA61FA6809175
:100DC000210990912209A0912309B09124098EA3B1
:100DD0009FA3A8A7B9A78B839C83AD83BE831886E6
:100DE0001F82AE01465D5F4FCE0101960E944EB656
:100DF00081309105B1F4D701ED91FC910488F5891A
:100E0000E02D1DA30CA38CA59DA5AEA5BFA58EA30B
:100E10009FA3A8A7B9A7A601BE016C5D7F4FC7011C
:100E20001995AF960FB6F894DEBF0FBECDBFDF9118
:100E3000CF911F910F91FF90EF90DF90CF90089589
:100E4000CF93DF93DC011496ED91FC916E177F0731
:100E500028F54115510511F19F01261B370B42174B
:100E6000530708F49A01DB01EC0188819981E21BA8
:100E7000F30BFD83EC83AF01461B570B260F371F87
:100E8000BC01620F731F8A0F9B1F0E9480DAE881EA
:100E9000F9818C819D81E80FF91F1082DF91CF913C
:100EA0000895DF92EF92FF920F931F93CF93DF93FA
:100EB000FC01E480F580E114F10451F48FEF9FEF21
:100EC000DF91CF911F910F91FF90EF90DF900895E8
:100ED000EC010190F081E02DEE0DFF1DD08010821D
:100EE00008811981062E000C770BC8010E948FDA49
:100EF0000E0D1F1DF801D082009701F32881398162
:100F0000821B930BDDCFFC012481358162177307AF
:100F100048F480819181009729F0860F971FFC018A
:100F20008081089580E00895FB0144815581FC0192
:100F3000248135812417350778F0808191810097CD
:100F400059F0FB01608171816115710529F00E94E2
:100F500072DA21E0892B09F020E0822F0895FC014C
:100F600024813581232B39F421E0FB018081882302
:100F700049F020E007C0808191810E9452DA21E08F
:100F8000892BB9F7822F0895FC0124813581FB015B
:100F90004481558124173507E1F4FC01808191815A
:100FA000FB01608171810097D1F061157105A1F499
:100FB000232BC1F0FC01808190E008C0232B91F02D
:100FC000FB01808190E091958195910921E0892B29
:100FD00009F020E0822F08950E9452DAF7CF6115C0
:100FE000710561F721E0F6CF0F931F93CF93DF9345
:100FF0008C01EB01FC01808191810097E1F0688117
:10100000798161157105A9F0428153812C813D815F
:101010004217530770F00E945BDA8C819D81F801C2
:10102000958384831D821C82DF91CF911F910F9144
:1010300008950E948ACC88819981F80191838083E8
:101040008A819B81938382838C819D819583848314
:10105000198218821B821A82E5CF0F931F93CF93B8
:10106000DF93EC0188819981009759F02A813B81B7
:101070002617370730F081E0DF91CF911F910F9154
:1010800008958B016F5F7F4F0E94F1D8009759F050
:10109000998388831B830A832C813D81232B59F7F5
:1010A000FC011082E8CF80E0E7CFEF92FF920F9330
:1010B0001F93CF93DF936115710541F480E0DF91B9
:1010C000CF911F910F91FF90EF9008954115510519
:1010D000B1F07B01EC010C811D81040F151FB801DB
:1010E0000E942D88882351F3288139818C819D812C
:1010F000B701820F931F0E945BDA1D830C8381E08E
:10110000DECFCF93DF931F921F92CDB7DEB76983F7
:101110001A8241E050E0BE016F5F7F4F0E94558808
:101120000F900F90DF91CF910895CF93DF93EC0153
:1011300088819981009711F00E948ACC19821882C7
:101140001D821C821B821A82DF91CF910895EF923B
:10115000FF920F931F93CF93DF9300D01F92CDB7D1
:10116000DEB77C01862F4AE08E010F5F1F4FB8016A
:1011700090E00E94A3CEF80101900020E9F731979A
:10118000AF01401B510BB801C7010E945588811166
:1011900003C0C7010E949588C7010F900F900F9060
:1011A0000F90DF91CF911F910F91FF90EF900895D5
:1011B000CF93DF93EC016115710539F4CE010E94E4
:1011C0009588CE01DF91CF910895FB010190002019
:1011D000E9F73197AF01461B570B0E9455888823CA
:1011E00069F3EFCFCF93DF93EC01FB01448155818D
:1011F000608171810E945588811103C0CE010E94D7
:101200009588CE01DF91CF910895EF92FF920F93D1
:101210001F93CF93DF93EC017B018A01BA010E94F7
:101220002D8881110BC0CE010E949588CE01DF91DF
:10123000CF911F910F91FF90EF9008951D830C8324
:10124000B701888199810E945BDAF0CFFB010190A0
:101250000020E9F73197AF01461B570B0C94058925
:10126000CF93DF93EC016115710531F00E9426895F
:10127000CE01DF91CF9108950E949588F9CFCF9349
:10128000DF93EC01FB018617970749F060817181BC
:101290006115710541F0448155810E940589CE0197
:1012A000DF91CF9108950E949588F9CFFC0180814C
:1012B0009181009711F00C948ACC0895EF92FF92DF
:1012C0000F931F93CF93DF93EC018B011982188248
:1012D0001B821A821D821C82CB010E9437CE7C01A8
:1012E000BC01CE010E942D88811109C0CE01DF9181
:1012F000CF911F910F91FF90EF900C949588FD82F4
:10130000EC82B80188819981DF91CF911F910F9173
:10131000FF90EF900C9430CEFC011182108213826A
:101320001282158214820C943F89FC011182108272
:101330001382128215821482FB0101900020E9F7CA
:101340003197AF01461B570B0C940589AF92BF92A2
:10135000CF92DF92EF92FF920F931F93CF93DF9381
:101360005C016B017A0189012417350720F48F2D68
:101370007901042F182F6AE875E0C5010E9495894C
:10138000D6011496CD91DC91EC16FD06C8F40C172D
:101390001D0708F4E801D601ED91FC911197EC0FBF
:1013A000FD1F108110826D917C916E0D7F1DC50116
:1013B0000E943089F60180819181C80FD91F18835E
:1013C000C501DF91CF911F910F91FF90EF90DF90BA
:1013D000CF90BF90AF9008951F920F920FB60F92CB
:1013E00011240BB60F922F933F934F935F936F93FC
:1013F0007F938F939F93AF93BF93EF93FF93E0916E
:101400001202F09113021995FF91EF91BF91AF91E4
:101410009F918F917F916F915F914F913F912F910C
:101420000F900BBE0F900FBE0F901F9018951F923C
:101430000F920FB60F9211240BB60F922F933F937A
:101440004F935F936F937F938F939F93AF93BF93CC
:10145000EF93FF93E0911002F09111021995FF9123
:10146000EF91BF91AF919F918F917F916F915F911C
:101470004F913F912F910F900BBE0F900FBE0F9089
:101480001F9018951F920F920FB60F9211240BB652
:101490000F922F933F934F935F936F937F938F930D
:1014A0009F93AF93BF93EF93FF93E0910602F09168
:1014B00007021995FF91EF91BF91AF919F918F9185
:1014C0007F916F915F914F913F912F910F900BBE44
:1014D0000F900FBE0F901F9018951F920F920FB68E
:1014E0000F9211240BB60F922F933F934F935F935C
:1014F0006F937F938F939F93AF93BF93EF93FF93DC
:10150000E0910402F09105021995FF91EF91BF91CE
:10151000AF919F918F917F916F915F914F913F918B
:101520002F910F900BBE0F900FBE0F901F9018952C
:101530001F920F920FB60F9211240BB60F922F939A
:101540003F934F935F936F937F938F939F93AF934B
:10155000BF93EF93FF93E0910E02F0910F02199564
:10156000FF91EF91BF91AF919F918F917F916F917B
:101570005F914F913F912F910F900BBE0F900FBE37
:101580000F901F9018951F920F920FB60F92112473
:101590000BB60F922F933F934F935F936F937F936D
:1015A0008F939F93AF93BF93EF93FF93E0910C02C0
:1015B000F0910D021995FF91EF91BF91AF919F911D
:1015C0008F917F916F915F914F913F912F910F90EC
:1015D0000BBE0F900FBE0F901F9018951F920F9289
:1015E0000FB60F9211240BB60F922F933F934F9388
:1015F0005F936F937F938F939F93AF93BF93EF937B
:10160000FF93E0910A02F0910B021995FF91EF917F
:10161000BF91AF919F918F917F916F915F914F910A
:101620003F912F910F900BBE0F900FBE0F901F9008
:1016300018951F920F920FB60F9211240BB60F92AE
:101640002F933F934F935F936F937F938F939F93CA
:10165000AF93BF93EF93FF93E0910802F0910902DB
:101660001995FF91EF91BF91AF919F918F917F91CC
:101670006F915F914F913F912F910F900BBE0F9003
:101680000FBE0F901F9018950F931F93CF93DF936A
:10169000EC010E9433B0688779878A879B87E8814D
:1016A000F9810284F385E02DCE01199597FF15C0CD
:1016B0000E9433B0088519852A853B85601B710B14
:1016C000820B930B0C811D812E813F816017710766
:1016D0008207930720F38FEF9FEFDF91CF911F9148
:1016E0000F910895EF92FF920F931F93CF93DF9383
:1016F000EC017B01042F6AE875E00E949589C7011F
:101700000E94448B002E000C110B97FD0BC0081794
:10171000190741F0682FCE010E948188C7010E94FD
:10172000448BF3CFCE01DF91CF911F910F91FF90AA
:10173000EF900895FB0101900020E9F73197AF0188
:10174000461B570BDC01ED91FC910280F381E02DEB
:1017500019948F929F92AF92BF92EF92FF920F9344
:101760001F93CF93DF93CDB7DEB7A1970FB6F89451
:10177000DEBF0FBECDBF7C01FA01CB0119A2223022
:1017800008F42AE08E010F5D1F4F822E912CB12CA0
:10179000A12CBF01A50194010E9466D5F901CA01DF
:1017A0006A300CF5605DD8016E938D01232B242BDC
:1017B000252B79F790E080E0109721F0BD01C7015B
:1017C0000E949A8BA1960FB6F894DEBF0FBECDBFD4
:1017D000DF91CF911F910F91FF90EF90BF90AF904D
:1017E0009F908F900895695CDECF68E875E00C9457
:1017F0009A8BDC01ED91FC910190F081E02D199420
:101800002F923F924F925F926F927F928F929F9210
:10181000AF92BF92CF92DF92EF92FF921F93CF933E
:10182000DF93EC016A017B01722EAB019601CB01C3
:10183000B6010E9484D76BE875E0811126C046018D
:101840005701E894B7F82FEF3FEF4FE75FE7C50187
:10185000B4010E9484D781110CC02FEF3FEF4FE7F6
:101860005FE7C501B4010E941CD46FE875E018164B
:1018700064F02FEF3FEF4FE75FE4C701B6010E942E
:1018800024D71816B4F463E975E0CE01DF91CF9147
:101890001F91FF90EF90DF90CF90BF90AF909F90FF
:1018A0008F907F906F905F904F903F902F900C940F
:1018B0009A8B2FEF3FEF4FE75FECC701B6010E9415
:1018C0001CD487FDE0CF20E030E0A901C701B601BC
:1018D0000E941CD4312C212C87FF09C06DE2CE015F
:1018E0000E94F98B1C01F7FAF094F7F8F09410E0DD
:1018F00060E070E080E09FE3711641F020E030E0AE
:1019000040E251E40E947CD61F5FF6CFA70196010A
:101910000E9410D62B013C010E94F5D64B015C01C0
:101920002AE0BC01A401CE010E94A98B7C01E20C3B
:10193000F31C1123C1F1C501B4010E9421D49B0104
:10194000AC01C301B2010E940FD64B015C016EE2F3
:10195000CE010E94F98BE80EF91E115020F120E013
:1019600030E040E251E4C501B4010E9482D42B0171
:101970003C010E94F5D64B01B12CA12C2AE0B50107
:10198000A401CE010E94A98BE80EF91EC501B40185
:101990000E9421D49B01AC01C301B2010E940FD669
:1019A0004B015C01DACFC701DF91CF911F91FF900E
:1019B000EF90DF90CF90BF90AF909F908F907F90EF
:1019C0006F905F904F903F902F900895CF92DF924D
:1019D000EF92FF920F931F93CF93DF932115310561
:1019E00081F4DC01ED91FC910190F081E02D642FF8
:1019F000DF91CF911F910F91FF90EF90DF90CF90EB
:101A000019942A30310501F52AE077FF1DC06A01DB
:101A10007B01EC016DE20E94F98B8C014427552774
:101A2000BA014C195D096E097F092AE0CE010E94B6
:101A3000A98B800F911FDF91CF911F910F91FF9084
:101A4000EF90DF90CF900895DF91CF911F910F918C
:101A5000FF90EF90DF90CF900C94A98B8F929F9284
:101A6000AF92BF92CF92DF92EF92FF920F931F93AC
:101A7000CF93DF937C018B014C0182E0880E911C97
:101A80005701E5E0AE0EB11CD0E0C0E0F401619179
:101A90004F01C8010E94E5A66C016EE2C8010E94D8
:101AA000F98B8C0D9D1DC80FD91F8A149B0471F7EB
:101AB000F7016581C8010E94E5A68C0F9D1FDF918B
:101AC000CF911F910F91FF90EF90DF90CF90BF903B
:101AD000AF909F908F9008956115710511F00C944F
:101AE0009A8B90E080E008950F931F93CF93DF933C
:101AF000EC0167E975E088EC99E00E946C8D4A85FD
:101B00005B856C857D858A819B81AC81BD81481B0D
:101B1000590B6A0B7B0B8E859F85A889B989481B59
:101B2000590B6A0B7B0B2AE088EC99E00E94A98B89
:101B300088EC99E00E94F58B6A857B858C859D8574
:101B40000A811B812C813D81601B710B820B930BE1
:101B50000E851F8528893989601B710B820B930BB9
:101B6000DF91CF911F910F9108950F931F93CF9302
:101B7000DF93EC018B0162E675E00E946C8D01152C
:101B80001105C1F1F80161918F01662399F160326D
:101B900040F0623231F06C3521F0CE010E94F98BB9
:101BA000F1CF6CE5CE010E94F98BF801319780816D
:101BB0008C30D1F044F48930D9F08A30B9F08830D3
:101BC00009F762E6EACF823259F024F462E78D30F9
:101BD00021F3D8CF8F3231F06CE58C35F1F2D2CFD2
:101BE00062E2DBCF6FE2D9CF66E6D7CF6EE6D5CF24
:101BF00064E7D3CF62E2CE010E94F98B90E080E0EF
:101C0000DF91CF911F910F910895DB0114964D91B3
